:100000000C94C0100C94EF100C94EF100C94EF10A3
:100010000C94EF100C94EF100C94EF100C94EF1064
:100020000C94EF100C94EF100C94EF100C94EF1054
:100030000C94EF100C9437990C94EF100C94EF1073
:100040000C94EF100C9461AC0C9481E70C94EF10BD
:100050000C94C8270C94EF100C94EF100C94EF1034
:100060000C94EF100C94EF100C9465E40C94EF10CA
:100070000C94EF100C94EF100C94EF100C94EF1004
:100080000C94EF100C94EF100C94EF10BBACC8ACB8
:10009000E7ACF4AC0FAD12AD15AD18AD1BAD1EAD98
:1000A00021AD24AD27AD34AD62AD9BE8A0E8A5E855
:1000B000AFE8DDE8DDE8B9E8C1E8C9E8D3E8FAE887
:1000C000FDE8F0E8F4E814E914E901E905E90BE9D1
:1000D0000FE9084AD73B3BCE016E84BCBFFDC12F60
:1000E0003D6C74319ABD56833DDA3D00C77F11BE29
:1000F000D9E4BB4C3E916BAAAABE000000803F052C
:10010000A84CCDB2D44EB93836A9020C50B991865C
:1001100088083CA6AAAA2ABE000000803F004D38ED
:100120003420582059205A20450043616E6E6F7468
:1001300020656E746572207375626469723A20007E
:100140006175746F25692E67006572726F72207712
:10015000726974696E6720746F2066696C65004E01
:100160006F74205344207072696E74696E67005317
:1001700044207072696E74696E67206279746520BC
:100180000044656C6574696F6E206661696C6564B6
:100190002C2046696C653A200046696C65206465D0
:1001A0006C657465643A006F70656E206661696C99
:1001B00065642C2046696C653A2000577269746941
:1001C0006E6720746F2066696C653A20002E0A0005
:1001D0006F70656E206661696C65642C2046696C81
:1001E000653A20002E0A006F70656E206661696CAA
:1001F00065642C2046696C653A200046696C652070
:1002000073656C6563746564002053697A653A2090
:100210000046696C65206F70656E65643A20006FFA
:1002200070656E206661696C65642C2046696C653A
:100230003A20004E6F772066726573682066696C9D
:10024000653A20004E6F7720646F696E672066699B
:100250006C653A20002220706F730022207061725A
:10026000656E743A2200535542524F5554494E45DB
:100270002043414C4C207461726765743A22004BF4
:10028000494C4C45442E2000747279696E67207485
:100290006F2063616C6C207375622D67636F64659A
:1002A0002066696C6573207769746820746F6F20AD
:1002B0006D616E79206C6576656C732E204D4158AA
:1002C000206C6576656C2069733A004D3234004DC0
:1002D00032332025730053442063617264206F6BB6
:1002E000006F70656E526F6F74206661696C656433
:1002F00000766F6C756D652E696E69742066616934
:100300006C656400534420696E6974206661696C91
:100310000020204D383531205A005A2D50726F621E
:1003200065204F666673657420286D6D293A00203C
:10033000204D3230302044300020204D32303020EB
:1003400044002044697361626C65640046696C61B5
:100350006D656E742073657474696E67733A0020FE
:10036000440020490020204D333034205000204CE0
:100370000020430020440020490020204D3330312C
:100380002050005049442073657474696E67733A55
:100390000020460020420020204D313435205331CA
:1003A00020480020460020420020204D31343520D6
:1003B00053302048004D6174657269616C20686536
:1003C0006174757020706172616D65746572733AE5
:1003D00000205A0020590020204D3230362058008D
:1003E000486F6D65206F666673657420286D6D2992
:1003F0003A00204500205A00205800204200205496
:100400000020204D323035205300416476616E6308
:100410006564207661726961626C65733A20533D50
:100420004D696E20666565647261746520286D6D26
:100430002F73292C20543D4D696E207472617665AE
:100440006C20666565647261746520286D6D2F731C
:10045000292C20423D6D696E696D756D207365674D
:100460006D656E742074696D6520286D73292C206C
:10047000583D6D6178696D756D205859206A6572B7
:100480006B20286D6D2F73292C20205A3D6D6178CB
:10049000696D756D205A206A65726B20286D6D2F0D
:1004A00073292C2020453D6D6178696D756D20455F
:1004B000206A65726B20286D6D2F7329002054000F
:1004C00020520020204D32303420500041636365BB
:1004D0006C65726174696F6E733A20503D70726919
:1004E0006E74696E672C20523D726574726163741C
:1004F00020616E6420543D74726176656C00204505
:1005000000205A0020590020204D32303120580060
:100510004D6178696D756D20416363656C657261CD
:1005200074696F6E20286D6D2F7332293A00204553
:1005300000205A0020590020204D3230332058002E
:100540004D6178696D756D2066656564726174656D
:100550007320286D6D2F73293A00204500205A0022
:1005600020590020204D3932205800537465707393
:100570002070657220756E69743A00486172646318
:100580006F6465642044656661756C74205365749E
:1005900074696E6773204C6F6164656400206279D2
:1005A00074657329002073746F72656420736574B9
:1005B00074696E677320726574726965766564200C
:1005C0002800206279746573290053657474696E1C
:1005D00067732053746F7265642028004572726FD0
:1005E000722077726974696E6720746F2045455078
:1005F000524F4D210020496E76616C696420657808
:1006000074727564657220005072696E7465722030
:1006100068616C7465642E206B696C6C282920639A
:10062000616C6C656421004B494C4C45442E2000A4
:1006300020746F6F206C6F6E6720657874727573AD
:10064000696F6E2070726576656E746564002063F4
:100650006F6C6420657874727573696F6E20707248
:100660006576656E746564006F6B00526573656EC8
:10067000643A20003A20007A5F6D61783A20007A6F
:100680005F6D696E3A20005A204F6666736574008C
:100690004F666673657473206170706C6965640081
:1006A0004572723A20546F6F206661722100546F58
:1006B0006F206661722066726F6D2072656665726A
:1006C000656E636520706F696E740053657474693C
:1006D0006E672054726176656C20416363656C655A
:1006E000726174696F6E3A200053657474696E6745
:1006F000205265747261637420416363656C657236
:100700006174696F6E3A200053657474696E672076
:100710005072696E7420416363656C6572617469BF
:100720006F6E3A200053657474696E672050726969
:100730006E7420616E642054726176656C20416332
:1007400063656C65726174696F6E3A20004D313477
:100750003520533C696E6465783E206F7574206F58
:10076000662072616E67652028302D3129007A5F1E
:100770006D696E3A2000795F6D696E3A2000785F8E
:100780006D696E3A2000205A3A0020593A00204301
:100790006F756E7420583A200020453A00205A3A6E
:1007A0000020593A00583A004649524D57415245A7
:1007B0005F4E414D453A4D61726C696E20312E316C
:1007C0002E302D5243352046726F6D204172636882
:1007D00069766520534F555243455F434F44455F0B
:1007E00055524C3A68747470733A2F2F6769746865
:1007F00075622E636F6D2F4D61726C696E46697202
:100800006D776172652F4D61726C696E2050524F29
:10081000544F434F4C5F56455253494F4E3A312E39
:1008200030204D414348494E455F545950453A5058
:1008300072757361206933204558545255444552AE
:100840005F434F554E543A3120555549443A303064
:100850003030303030302D303030302D303030309E
:100860002D303030302D303030303030303030308E
:1008700030300A005072757361206933204F66660C
:100880002E0042656420646F6E652E004265642010
:1008900048656174696E672E0048656174696E67AA
:1008A00020646F6E652E003F0020573A005072752D
:1008B00073612069332072656164792E0048656137
:1008C00074696E672E2E2E006F6B004B494C4C45A1
:1008D000442E2000434F4D4D554E49434154494FFE
:1008E0004E0044525952554E004552524F525300F9
:1008F000494E464F004543484F007C006F666600F6
:1009000044454255473A005072757361206933205F
:1009100072656164792E0048656174696E672E2E78
:100920002E005374616E646172642044657669615F
:1009300074696F6E3A20004D65616E3A2000202088
:10094000207369676D613A2000206D65616E3A2001
:10095000002020207A3A2000206F66200020207A94
:100960003A2000793A2000783A2000202020616E59
:10097000676C653A20005374617274696E67207207
:1009800061646975733A2000506F736974696F6EA2
:10099000696E67207468652070726F62652E2E2EF6
:1009A0000A003F4E756D626572206F66206C656748
:1009B0007320696E206D6F76656D656E74206E6F45
:1009C0007420706C61757369626C652028302D31FC
:1009D00035292E0A00590058003F53616D706C652F
:1009E0002073697A65206E6F7420706C617573690D
:1009F000626C652028342D3530292E0A004D34389C
:100A0000205A2D50726F6265205265706561746165
:100A100062696C69747920746573740A003F566565
:100A200072626F7365204C6576656C206E6F742002
:100A3000706C61757369626C652028302D34292EC5
:100A40000A002569206D696E2C2025692073656375
:100A500000456E642066696C65206C6973740042A1
:100A60006567696E2066696C65206C697374004EF9
:100A70006F206D6F76652E0050727573612069333B
:100A80002072656164792E00526573756D696E67B9
:100A9000207072696E74005761697420666F7220ED
:100AA000757365722E2E2E00205A3A200020593A76
:100AB000200042656420583A2000205A3A20002045
:100AC000593A200042656420583A2000202B00202B
:100AD0000A436F72726563746564204265642048DE
:100AE00065696768742076732E2042656420546FB0
:100AF000706F6C6F67793A200A00202B0020283035
:100B00002C30290A002020204F2D2D2046524F4EF8
:100B100054202D2D2B0A002020207C202020202056
:100B20002020202020207C0A002020207C20202043
:100B300020282D29202020207C20540A0020542009
:100B40007C20202020202020202020207C20480ADB
:100B5000002046207C20282D29204E20282B2920CB
:100B60007C20470A002045207C20202020202020B7
:100B7000202020207C20490A00204C207C2020209E
:100B800020282B29202020207C20520A00202020F1
:100B90007C20202020202020202020207C0A0020D3
:100BA00020202B2D2D2D204241434B202D2D2B0A73
:100BB00000200A4265642048656967687420546FA4
:100BC000706F6772617068793A200A004D65616ED6
:100BD000206F662073616D706C656420706F696E44
:100BE00074733A200020643A200020623A200045C5
:100BF000716E20636F656666696369656E74733ACA
:100C000020613A200028422961636B00284629723E
:100C10006F6E74002852296967687400284C296532
:100C20006674003F4E756D626572206F662070724B
:100C30006F626564202850296F696E747320697330
:100C400020696D706C61757369626C652028322053
:100C50006D696E696D756D292E0A0052756E6E692B
:100C60006E6720696E204452592D52554E206D6F8B
:100C7000646500473239204175746F2042656420F5
:100C80004C6576656C696E670A003F285629657267
:100C9000626F7365204C6576656C20697320696DA1
:100CA000706C61757369626C652028302D34292E53
:100CB00000486F6D6520582F59206265666F726518
:100CC000205A00486F6D6520582F59206265666F65
:100CD0007265205A005761726E696E673A20486FDC
:100CE0006D696E672042756D702044697669736F17
:100CF00072203C2031005A2070726F6265206F753F
:100D0000742E20626564005A2070726F6265206FD5
:100D100075742E2062656400536C6565702E2E2EEE
:100D20000020403A002042403A00202F0020423A62
:100D300000202F0020543A0020706F736974696F8F
:100D40006E206F7574206F662072616E67652E006D
:100D50003F50726F62652000627573793A2070614E
:100D60007573656420666F7220696E7075740062B9
:100D70007573793A2070617573656420666F7220AF
:100D80007573657200627573793A2070726F63656E
:100D90007373696E6700220A00556E6B6E6F776E13
:100DA00020636F6D6D616E643A20220025692068B2
:100DB0006F757273202569206D696E757465730097
:100DC000446F6E65207072696E74696E6720666923
:100DD0006C65004B494C4C45442E200053544F50F9
:100DE0005045442E20005072696E746572207374F1
:100DF0006F707065642064756520746F2065727211
:100E00006F72732E2046697820746865206572724F
:100E10006F7220616E6420757365204D39393920F9
:100E2000746F20726573746172742E202854656D1E
:100E3000706572617475726520697320726573657F
:100E4000742E205365742069742061667465722065
:100E500072657374617274696E6729004E6F204CFD
:100E6000696E65204E756D626572207769746820C1
:100E7000636865636B73756D2C204C617374204CD3
:100E8000696E653A20004E6F20436865636B737529
:100E90006D2077697468206C696E65206E756D626F
:100EA00065722C204C617374204C696E653A200089
:100EB000636865636B73756D206D69736D617463D1
:100EC000682C204C617374204C696E653A20004C8C
:100ED000696E65204E756D626572206973206E6F54
:100EE00074204C617374204C696E65204E756D6280
:100EF00065722B312C204C617374204C696E653AFD
:100F000020004D31313000446F6E65207361766989
:100F10006E672066696C652E004D323900202050C6
:100F20006C616E6E65724275666665724279746553
:100F3000733A20002046726565204D656D6F7279A9
:100F40003A20004D6179202035203230313600437F
:100F50006F6D70696C65643A200050686973696BE5
:100F600000207C20417574686F723A200032303165
:100F7000362D30342D30312031323A303000204C93
:100F800061737420557064617465643A2000203187
:100F90002E312E302D524335004D61726C696E003A
:100FA00020536F66747761726520526573657400B3
:100FB000205761746368646F6720526573657400BD
:100FC0002042726F776E206F75742052657365745E
:100FD000002045787465726E616C2052657365748B
:100FE00000506F77657255700073746172740022DF
:100FF00000656E7175657565696E67202200FFFF7B
:10100000FF0000A0400000A0400000004000007A67
:10101000430000524300002A43000034C20000A0F5
:10102000C00000000000004D4300004D4300002AB6
:1010300043000034C20000A0C000000000656368E7
:101040006F3A004572726F723A0020746F6F206CB5
:101050006F6E6720657874727573696F6E20707239
:101060006576656E7465640020636F6C64206578D6
:1010700074727573696F6E2070726576656E7465D3
:1010800064007C3C3E5E2B3D3F2F5B5D3B2C2A2267
:101090005C004D383420582059205A204500656E98
:1010A0006473746F7073206869743A205A00205A10
:1010B0003A00656E6473746F7073206869743A20C7
:1010C000590020593A00656E6473746F707320681C
:1010D00069743A20580020583A00656E6473746F42
:1010E0007073206869743A200024F4D43050C38EA1
:1010F00020C2A24017828B7011127A910D816CD997
:101100000AA861E108C7586607615143061E4B5D96
:1011100005C145A7041A411104093D9803713931ED
:10112000034036DB0265339102D4305402802E1D19
:1011300002632CEE01752AC501B028A00110278199
:10114000018F2564012B244B01E0223401AC211FC7
:10115000018D200D01801FFC00841EED00971DDF16
:1011600000B81CD200E61BC600201BBC00641AB2EB
:1011700000B219A8000A19A0006A189900D11791A5
:101180000040178B00B516840031167E00B3157928
:10119000003A157300C7146F0058146A00EE136606
:1011A000008813630025135E00C7125B006C1257A2
:1011B0000015125400C111510070114F0021114B44
:1011C00000D61049008D104700461044000210421E
:1011D00000C00F4000800F3E00420F3C00060F3B56
:1011E00000CB0E3800930E37005C0E3500270E340E
:1011F00000F30D3200C10D3100900D3000600D2E56
:1012000000320D2D00050D2C00D90C2B00AE0C2941
:1012100000850C29005C0C2700350C27000E0C26DD
:1012200000E80B2400C40B2400A00B23007D0B233B
:10123000005A0B2100390B2100180B2000F80A1F5F
:1012400000D90A1E00BB0A1E009D0A1D00800A1D4F
:1012500000630A1C00470A1B002C0A1B00110A1A13
:1012600000F7091A00DD091900C4091900AB0919B2
:1012700000920917007B091800630917004C091632
:101280000036091600200916000A091500F5081590
:1012900000E0081400CC081400B8081400A40814D6
:1012A00000900813007D0812006B08130058081204
:1012B000004608120034081100230811001208111A
:1012C0000001081100F0071000E0071000D007101F
:1012D00000C0071000B0070F00A107100091070E13
:1012E0000083070F0074070F0065070E0057070EF5
:1012F0000049070E003B070D002E070E0020070DCA
:101300000013070D0006070D00F9060C00ED060D91
:1013100000E0060C00D4060C00C8060C00BC060C4D
:1013200000B0060C00A4060B0099060C008D060BFD
:101330000082060B0077060B006C060B0061060AA4
:101340000057060B004C060A0042060A0038060A3F
:10135000002E060A0024060A001A060A00100609D2
:101360000007060A00FD050900F4050900EB050960
:1013700000E2050900D9050900D0050900C70509E3
:1013800000BE050900B5050800AD050800A5050962
:10139000009C050800940508008C050800840508D9
:1013A000007C050800740508006C05070065050849
:1013B000005D050700560508004E050700470507B4
:1013C000004005080038050700310507002A050719
:1013D00000230507001C050600160507000F05077A
:1013E000000805060002050700FB040600F50407D7
:1013F00000EE040600E8040600E2040700DB040631
:1014000000D5040600CF040600C9040600C3040684
:1014100000BD040600B7040600B1040500AC0406D4
:1014200000A6040600A00405009B04060095040520
:1014300000900406008A0405008504050080040667
:10144000007A04050075040500700405006B0405AE
:101450000066040500610405005C040500570405EE
:1014600000520405004D040500480405004304052E
:10147000003E0404003A040500350405003004046D
:10148000002C04050027040400230405001E0404A6
:10149000001A04040016040500110404000D0404DD
:1014A00000090405000404040000040400FC030413
:1014B00000F8030400F4030400F0030400EC030448
:1014C00000E8030400E4030400E0030400DC030478
:1014D00000D8030400D4030400D0030400CC0304A8
:1014E00000C8030300C503030024F404D9201BC46F
:1014F0000C5C0E9804C4095F0265077101F405F9DC
:1015000000FB04B30048048700C103690058035579
:101510000003034500BE023A008402310053022A50
:10152000002902250004022000E4011C00C8011962
:1015300000AF01170098011400840113007101101D
:10154000006101100051010E0043010D0036010B36
:10155000002B010B0020010B00150109000C0109F3
:101560000003010800FB000800F3000800EB00077F
:1015700000E4000600DE000600D8000600D20006E7
:1015800000CC000500C7000500C2000500BD000436
:1015900000B9000400B5000400B1000400AD00046F
:1015A00000A9000400A5000300A20003009F00049E
:1015B000009B0003009800030095000200930003C5
:1015C00000900003008D0002008B000300880002E1
:1015D000008600020084000300810002007F0002F8
:1015E000007D0002007B000200790002007700010C
:1015F0000076000200740002007200010071000217
:10160000006F0002006D0001006C0002006A000122
:10161000006900020067000100660001006500012A
:10162000006400020062000100610001006000012E
:10163000005F0002005D0001005C0001005B000132
:10164000005A000100590001005800010057000134
:101650000056000100550001005400010053000035
:101660000053000100520001005100010050000130
:10167000004F0001004E0000004E0001004D00012F
:10168000004C0001004B0000004B0001004A00012B
:101690000049000100480000004800010047000127
:1016A0000046000000460001004500000045000122
:1016B000004400010043000000430001004200001C
:1016C0000042000100410000004100010040000113
:1016D000003F0000003F0001003E0000003E00010E
:1016E000003D0000003D0001003C0000003C000007
:1016F000003C0001003B0000003B0001003A0000FC
:10170000003A0001003900000039000100380000F3
:1017100000380000003800010037000000370001E9
:1017200000360000003600000036000100350000E1
:1017300000350000003500010034000000340000D6
:1017400000340001003300000033000000330001CA
:1017500000320000003200000032000100310000C1
:1017600000310000003100010030000000300000B6
:1017700000300001002F0000002F0000002F0000AB
:10178000002F0001002E0000002E0000002E00019E
:10179000002D0000002D0000002D0000002D000194
:1017A000002C0000002C0000002C0000002C000188
:1017B000002B0000002B0000002B0000002B00017C
:1017C000002A0000002A0000002A0000002A000170
:1017D0000029000000290000002900000029000065
:1017E0000029000100280000002800000028000057
:1017F000002800000028000100270000002700004A
:10180000002700000027000000270001002600003C
:10181000002600000026000000260000002600012F
:101820000025000000250000002500000025000024
:101830000025000000250001002400000024000015
:101840000024000000240000002400010023000008
:1018500000230000002300000023000000230000FC
:1018600000230000002300010022000000220000ED
:1018700000220000002200000022000000220001DF
:1018800000210000002100000021000000210000D4
:1018900000210000002100000021000100200000C4
:1018A00000200000002000000020000000200000B8
:1018B000002000000020000000200001001F0000A8
:1018C000001F0000001F0000001F0000001F00009C
:1018D000001F0000001F0001001E0000001E00008D
:1018E000001E0000001E0000004D494E54454D50A2
:1018F00020747269676765726564004572723A2088
:101900004D494E54454D5020424544004D41585498
:10191000454D502074726967676572656400457251
:10192000723A204D415854454D5020424544004D97
:10193000494E54454D5020747269676765726564FD
:10194000004572723A204D494E54454D5000626533
:1019500064002C2073797374656D2073746F7070DC
:10196000656421204865617465725F49443A2000CE
:101970004D415854454D50207472696767657265D2
:1019800064004572723A204D415854454D50004B09
:1019900064200023646566696E65202044454641E5
:1019A000554C545F004B69200023646566696E6581
:1019B000202044454641554C545F004B7020002385
:1019C000646566696E65202044454641554C545F08
:1019D00000504944204175746F74756E65206669C6
:1019E0006E69736865642120507574207468652081
:1019F0006C617374204B702C204B6920616E6420E5
:101A00004B6420636F6E7374616E74732066726FC3
:101A10006D2062656C6F7720696E746F20436F6E06
:101A200066696775726174696F6E2E68005049440B
:101A3000204175746F74756E65206661696C6564AC
:101A4000212074696D656F7574005049442041759B
:101A5000746F74756E65206661696C6564212054CD
:101A6000656D706572617475726520746F6F206842
:101A700069676800204B643A2000204B693A2000D7
:101A8000204B703A200020436C61737369632050CF
:101A9000494420002054753A2000204B753A20001C
:101AA000206D61783A2000206D696E3A2000206434
:101AB0003A200020626961733A20001000C902E0F8
:101AC000002C01000122013001180170010E01B04B
:101AD000010401F001FA005002F000F002E600906B
:101AE00003DC004004D2004005C8004006BE0000F0
:101AF00008B400B009AA00D00BA000600E960060E8
:101B0000118C000015820020197800C01D6E00A005
:101B1000226400B0275A00902C500000314600E0AB
:101B2000343C0010383200903A2800603C1E00A07F
:101B30003D1400803E0A00203F00004D3432380042
:101B4000312E312E302D524335002D2D2D2D2D2DA2
:101B5000007C4D61726C696E7C002D2D2D2D2D2D1C
:101B6000002D2D3A2D2D002D2D2D005344005A000F
:101B700020003F005A00590020003F00590020007B
:101B8000580020003F005800012000012000466C52
:101B90006F7700466C6F770046616E2073706565E5
:101BA000640046616E207370656564004265640080
:101BB000426564004E6F7A7A6C65004E6F7A7A6C7B
:101BC00065005370656564005370656564004D6120
:101BD000696E004D6F76652058004D6F766520590F
:101BE000004D6F7665205A00457874727564657291
:101BF000004578747275646572004D6F7665205A81
:101C0000004D6F7665205A004D6F76652059004D66
:101C10006F76652058004D6F766520617869730096
:101C20004D6F766520302E316D6D004D6F766520DD
:101C3000316D6D004D6F76652031306D6D005072E5
:101C40006570617265005072656865617420504C02
:101C50004120426564005072656865617420504C93
:101C6000410050726570617265005072656865610F
:101C7000742041425320426564005072656865617A
:101C80007420414253005072657061726500436F69
:101C90006F6C646F776E0050726568656174204187
:101CA0004253005072656865617420504C41004D8C
:101CB00038340044697361626C65207374657070B8
:101CC000657273004D6F76652061786973004732E5
:101CD00039004C6576656C2062656400536574203C
:101CE000686F6D65206F6666736574730047323880
:101CF000004175746F20686F6D65004D61696E00FD
:101D000053746F7265206D656D6F72790042656402
:101D100000426564004E6F7A7A6C65004E6F7A7A85
:101D20006C650046616E2073706565640046616E87
:101D30002073706565640054656D706572617475BB
:101D400072650053746F7265206D656D6F727900F6
:101D500042656400426564004E6F7A7A6C65004E9D
:101D60006F7A7A6C650046616E20737065656400F9
:101D700046616E2073706565640054656D706572B0
:101D800061747572650050726568656174204142C6
:101D90005320636F6E6600507265686561742050F1
:101DA0004C4120636F6E66005049442D43005049FA
:101DB000442D43005049442D44005049442D4400D3
:101DC0005049442D49005049442D49005049442D63
:101DD00050005049442D5000200220466163740099
:101DE00020022046616374002002204D61780020AB
:101DF00002204D6178002002204D696E00200220F3
:101E00004D696E004175746F74656D70004F666644
:101E1000004F6E200046616E207370656564004659
:101E2000616E20737065656400426564004265649C
:101E3000004E6F7A7A6C65004E6F7A7A6C6500435B
:101E40006F6E74726F6C004573746570732F6D6D77
:101E5000004573746570732F6D6D005A73746570EF
:101E6000732F6D6D005A73746570732F6D6D00590B
:101E700073746570732F6D6D005973746570732F73
:101E80006D6D005873746570732F6D6D00587374A9
:101E90006570732F6D6D00412D74726176656C00F5
:101EA000412D74726176656C00412D7265747261AA
:101EB000637400412D7265747261637400416D61D9
:101EC00078206500416D6178206500416D61782062
:101ED0007A00416D6178207A00416D617820790047
:101EE000416D6178207900416D6178207800416D05
:101EF00061782078005654726176206D696E0056C4
:101F000054726176206D696E00566D696E00566D73
:101F1000696E00566D6178206500566D61782065A8
:101F200000566D6178207A00566D6178207A0056EF
:101F30006D6178207900566D6178207900566D6169
:101F400078207800566D617820780056652D6A6596
:101F5000726B0056652D6A65726B00567A2D6A6544
:101F6000726B00567A2D6A65726B005678792D6A0D
:101F700065726B005678792D6A65726B00416363F8
:101F8000656C00416363656C005A204F666673653B
:101F900074005A204F666673657400436F6E7472E6
:101FA0006F6C0046696C2E204469612E0046696C96
:101FB0002E204469612E004520696E206D6D33002E
:101FC0004F6666004F6E2000436F6E74726F6C0038
:101FD000526573746F7265206661696C73616665C2
:101FE000004C6F6164206D656D6F72790053746F82
:101FF0007265206D656D6F72790046696C616D6503
:102000006E74004D6F74696F6E0054656D7065720B
:102010006174757265004D61696E00052E2E0004B5
:1020200052656672657368004D61696E004D3231AC
:1020300000496E69742E2053442063617264004E1F
:102040006F2053442063617264004D323100436855
:10205000616E676520534420636172640050726949
:102060006E742066726F6D2053440053746F70203D
:102070007072696E7400526573756D652070726957
:102080006E74005061757365207072696E740043E0
:102090006F6E74726F6C005072657061726500547F
:1020A000756E6500496E666F2073637265656E00BC
:1020B000207A3A200020793A200020783A20000047
:1020C00000000102000000000000000403080700F7
:1020D00000000000000000000000000000000001FF
:1020E00002040810204080010204081020408001F2
:1020F00002040810204080804020100804020102E1
:10210000020202020202020404040404040404039E
:1021100003030303030303010101010101010100A2
:1021200000200023002600290000002200250028AE
:10213000002B0000002100240027002A004E414E01
:10214000494E495459494E46CDCCCC3D0AD7233C43
:1021500017B7D13877CC2B329595E6241FB14F0AAB
:10216000000020410000C84200401C4620BCBE4C7C
:10217000CA1B0E5AAEC59D74E3634EBA38E4E763DA
:1021800011241FBECFEFD0E4DEBFCDBF14E0A0E02E
:10219000B1E0EEE3FCEE01E00BBF02C007900D9250
:1021A000A236B107D9F724E1A2E6B4E001C01D923E
:1021B000AE31B207E1F711E2CEE7D1E200E006C0AE
:1021C00022970109FE010BBF0E9454EFC837D107C7
:1021D00080E00807A9F70E94AEE90C940DF60C9474
:1021E0000000FC01148217821382128283ED93E0B7
:1021F00091838083089523ED33E0FC0131832083B4
:102200002781222319F004960C94198E0895CF92F9
:10221000DF92EF92FF920F931F93CF93DF93EC0126
:102220008F960E94F110CE01805B9F4F0E94F110AB
:102230007E012FE6E20EF11C87016E013BE5C31A19
:102240003EEFD30AC8010E94F110015E1F4F0C152A
:102250001D05C1F7FE01EA55FE4F89E18183148215
:102260003596178ACE0187539E4F0E94F110FE01CA
:10227000E658FD4F1082118212821382349610822A
:102280001182128213821A821B8218821982F8012B
:102290001082FE01E851FE4F108286E391E0F701C3
:1022A0009C01119221503040E1F7FE01EA57FD4FA9
:1022B00081E080831EA61DA60E94CBE7CE57DD4F8E
:1022C00068577C4E8F4F9F4F688379838A839B83A7
:1022D000DF91CF911F910F91FF90EF90DF90CF9002
:1022E0000895FC0120E03EE2DB014C91403241F0D8
:1022F000283011F430833196DB014C9140833196C4
:102300002F5F6F5F7F4F2B3079F7108208952F92E8
:102310003F924F925F926F927F928F929F92AF9275
:10232000BF92CF92DF92EF92FF920F931F93CF93C2
:10233000DF93CDB7DEB7C657D1090FB6F894DEBF2D
:102340000FBECDBF8C016B015A0129012DB73EB7DD
:10235000E3963FAF2EAFE397AD961FAEAD9734E057
:10236000A30EB11C4296E5969FAF8EAFE59718017C
:1023700099E7291A9DEF390AF801E757FD4FAF9603
:10238000FFAFEEAFAF973801F5E06F0E711C7E0125
:102390002FE5E20EF11C80E490E08C0F9D1F049667
:1023A000E7969FAF8EAFE797E5964EAD5FADE597A9
:1023B000BE016F5F7F4FC5010E947A8C18160CF02A
:1023C00048C12C85322F3871303109F0C1C0F1017C
:1023D000808191810197029708F4BAC02DB73EB76A
:1023E000E1963FAF2EAFE197BE016F5F7F4FC70110
:1023F0000E94711181E0F60190819111A1C0E1E08C
:10240000F0E0D7010D900020E9F7EE19FF09EA0F7F
:10241000FB1F31962DB73EB72E1B3F0B0FB6F8941E
:102420003EBF0FBE2DBFEDB7FEB731964F018823DB
:1024300019F062EA72E001C0B601C4010E9400F323
:10244000B701C4010E94E1F262EA72E0C4010E9495
:10245000E1F2CE01805C9F4F0E94F11021E0A701C4
:10246000B501E7968EAD9FADE7970E94229081114E
:1024700037C0F10180819181892B91F5EDE3F0E185
:102480008491882341F09091C00095FFFCCF809308
:10249000C6003196F5CFE4EAF2E08191882339F065
:1024A0009091C00095FFFCCF8093C600F6CF80913D
:1024B000C00085FFFCCF8AE08093C600F7018191C0
:1024C000882339F09091C00095FFFCCF8093C6001F
:1024D000F6CF8091C00085FFFCCF8AE08093C600D4
:1024E0008BE1FE01EC5BFF4FDE01959601900D92B2
:1024F0008A95E1F724968EAD9FAD24979CA38BA37C
:1025000083ED93E09AA389A320E030E0AE014F5D14
:102510005F4FB401C8010E948711CE0181960E94CD
:10252000FB10CE01805C9F4F0E94FB10E1962EAD08
:102530003FADE1970FB6F8943EBF0FBE2DBF34CF2D
:1025400080E001900020E9F73197EC19FD0959CF9F
:102550008981882309F47DC0853E09F425CF8E3218
:1025600009F422CFF80182898E3209F41DCF23FDB0
:102570001BCF81E0303109F080E0F80184838111C4
:1025800008C08985873409F00FCF8A858E3709F412
:102590000BCFF101808191818130910571F0823002
:1025A000910589F1892B09F0FFCEBE016F5F7F4F46
:1025B000C3010E947111F60110C0AF96EEADFFADE0
:1025C000AF9780819181019691838083EDCE909128
:1025D000C00095FFFCCF8093C60081918111F7CF99
:1025E000F3018191882339F09091C00095FFFCCFD1
:1025F0008093C600F6CF8091C00085FFFCCF8AE0B3
:102600008093C600D1CEBE016F5F7F4FC3010E9491
:1026100071114114510439F0B301C2010E94CEF28C
:10262000892B79F416C0AD96FFADAD972F2F30E012
:10263000AF96EEADFFADAF97808191812817390736
:1026400041F0AD96FFADAD97FF5FAD96FFAFAD9793
:10265000ABCEE3962EAD3FADE3970FB6F8943EBFF9
:102660000FBE2DBFCA58DF4F0FB6F894DEBF0FBEA6
:10267000CDBFDF91CF911F910F91FF90EF90DF9031
:10268000CF90BF90AF909F908F907F906F905F9012
:102690004F903F902F900895EF92FF920F931F93CA
:1026A000CF93DF93CDB7DEB76F970FB6F894DEBF49
:1026B0000FBECDBF8C01FC01E957FD4F1182108286
:1026C0007C0183E3E80EF11C40E050E0BA01C70151
:1026D0000E94338D8BE1F701DE01159601900D927A
:1026E0008A95E1F7F80181A992A99C838B8383EDF8
:1026F00093E09A83898320E030E0AE014F5F5F4F23
:102700006EEC72E0C8010E948711CE0101960E9412
:10271000FB106F960FB6F894DEBF0FBECDBFDF91F2
:10272000CF911F910F91FF90EF900895EF92FF923C
:102730000F931F93CF93DF93EC011B828EA9882305
:1027400021F0CE01C3960E94198E7E018AE5E81A17
:102750008EEFF80A4FE160E0C7010E946D88811199
:102760001FC0EDE3F0E18491882341F09091C00017
:1027700095FFFCCF8093C6003196F5CFE4E0F3E0FF
:102780008491882341F09091C00095FFFCCF809305
:10279000C6003196F5CF8091C00085FFFCCF76C092
:1027A0008E0105551E4F41E0B701C8010E944A96AF
:1027B000811126C040E0B701C8010E944A968111EC
:1027C0001FC0E3E4F0E18491882341F09091C000C0
:1027D00095FFFCCF8093C6003196F5CFE1EFF2E094
:1027E0008491882341F09091C00095FFFCCF8093A5
:1027F000C6003196F5CF8091C00085FFFCCF46C062
:10280000B801CE01C3960E941A8B81111FC0E3E468
:10281000F0E18491882341F09091C00095FFFCCFB6
:102820008093C6003196F5CFE1EEF2E084918823E3
:1028300041F09091C00095FFFCCF8093C600319687
:10284000F5CF8091C00085FFFCCF20C081E08B8355
:10285000EDE3F0E18491882341F09091C00095FF71
:10286000FCCF8093C6003196F5CFE6EDF2E084917F
:10287000882341F09091C00095FFFCCF8093C60063
:102880003196F5CF8091C00085FFFCCF8AE0809320
:10289000C600CE01805B9F4F2BE1FE01F396DC0169
:1028A000149601900D922A95E1F729A93AA9FC0105
:1028B000338322833297AF96D183C083DF91CF9148
:1028C0001F910F91FF90EF900895FC0112821382E7
:1028D0000895CF92DF92EF92FF920F931F93CF93C1
:1028E000DF93CDB7DEB7CDB6DEB6FB010190002099
:1028F000E9F7E61BF70B34968DB79EB78E1B9F0B3F
:102900000FB6F8949EBF0FBE8DBF0DB71EB70F5FF9
:102910001F4F7F936F938FEC92E09F938F931F9342
:102920000F930E9424F3780194E0E90EF11C0F90BC
:102930000F900F900F900F900F90F70180818823D8
:1029400049F0992787FD90950E946FF2F7018193D6
:102950007F01F3CF60E0C8010E94E52A8BEC92E092
:102960000E948C2B0FB6F894DEBE0FBECDBEDF9159
:10297000CF911F910F91FF90EF90DF90CF9008952E
:10298000FC012381222311F021E022830895FC0120
:102990002281211112820895AF92BF92CF92DF92CD
:1029A000EF92FF920F931F93CF93DF931F92CDB7B8
:1029B000DEB78C018FE2FB0181935F01D12C21E016
:1029C0007801FBE5EF1AFEEFFF0A8FE1C82EF70151
:1029D0008081D816C8F4B501C801CD9C800D911D29
:1029E00011248D589F4F29830E94BF8AC5012981D8
:1029F0005C010196F5013081332321F02D3810F46C
:102A00002F5FF6CFD394E3CF27FD11C0B501C801E6
:102A100083539E4F0F90DF91CF911F910F91FF90A5
:102A2000EF90DF90CF90BF90AF900C94BF8AF501EC
:102A300010820F90DF91CF911F910F91FF90EF9037
:102A4000DF90CF90BF90AF9008953F924F925F92EA
:102A50006F927F928F929F92AF92BF92CF92DF92AE
:102A6000EF92FF920F931F93CF93DF93CDB7DEB713
:102A7000AC970FB6F894DEBF0FBECDBF7C015B01F3
:102A8000FC018381882309F4EFC0C70183539E4F63
:102A90000E94198EF7011282CE0101966C010E94EC
:102AA000F11027019EE4490E511CC7018F96F201D7
:102AB00091838083F50180818F3209F077C06FE2C6
:102AC00070E0C5010E94ECF28C010F5F1F4F9AE08D
:102AD000392E0115110509F46FC06FE270E0C801CD
:102AE0000E94ECF24C01009709F467C0081719071F
:102AF00008F063C03C01601A710AA301B801CE015D
:102B000080960E9415F3E0E2F0E0EC0FFD1FE60D69
:102B1000F71D1082FE01B0968191882339F09091C3
:102B2000C00095FFFCCF8093C600F6CF8091C00017
:102B300085FFFCCF3092C600F20160817181611582
:102B4000710519F06C5F7F4F02C060E070E021E01A
:102B5000AE01405E5F4FCE0105960E94229081112A
:102B60001EC0E7EAF1E08491882341F09091C00013
:102B700095FFFCCF8093C6003196F5CFFE01B0964D
:102B80008191882339F09091C00095FFFCCF80930C
:102B9000C600F6CF8091C00085FFFCCF5FC0F20178
:102BA000D182C08284010F5F1F4F93CFC701805B2A
:102BB0009F4FF201918380838501F2018081918191
:102BC000009711F0049602C080E090E0B8010E94E6
:102BD0000291811103C0E1E8F1E02EC0E9E9F1E0E2
:102BE0008491882341F09091C00095FFFCCF8093A1
:102BF000C6003196F5CFF8018191882339F0909184
:102C0000C00095FFFCCF8093C600F6CF8091C00036
:102C100085FFFCCF8AE08093C600F701E258FD4FA4
:102C200010821182128213821CC09091C00095FF05
:102C3000FCCF8093C600319684918111F6CFF801C4
:102C40008191882339F09091C00095FFFCCF80934B
:102C5000C600F6CF8091C00085FFFCCF8EE2809346
:102C6000C600C6010E94FB10AC960FB6F894DEBFFA
:102C70000FBECDBFDF91CF911F910F91FF90EF90CD
:102C8000DF90CF90BF90AF909F908F907F906F908C
:102C90005F904F903F900895CF93DF93EC018B812D
:102CA000811103C0EFE5F1E039C0EFE6F1E0849176
:102CB000882341F09091C00095FFFCCF8093C6001F
:102CC0003196F5CFFE01E258FD4F4081518162817E
:102CD00073812AE030E082E694E00E9439298091F5
:102CE000C00085FFFCCF8FE28093C600C658DD4F41
:102CF000488159816A817B812AE030E082E694E054
:102D00000E9439298091C00085FFFCCF0EC09091B0
:102D1000C00095FFFCCF8093C6003196849181114D
:102D2000F6CF8091C00085FFFCCF8AE08093C6007B
:102D3000DF91CF910895AF92BF92CF92DF92EF9241
:102D4000FF920F931F93CF93DF935C01EB01FB0185
:102D500001900020E9F78F0101501109061B170BA4
:102D60006C01F3E3CF1AFEEFDF0AF60110826EE486
:102D700070E0CE010E94ECF27C01009729F4F8018A
:102D80003197EC0FFD1F0DC060E270E00E94ECF285
:102D9000EC0121966AE270E0C7010E94ECF2FC01AE
:102DA00031978DE081838AE082831382BE01C50161
:102DB00087539E4F0E94E892F6018081882309F193
:102DC000E3E4F0E18491882341F09091C00095FF05
:102DD000FCCF8093C6003196F5CFE9E4F1E0849111
:102DE000882341F09091C00095FFFCCF8093C600EE
:102DF0003196F5CF8091C00085FFFCCF8AE08093AB
:102E0000C600DF91CF911F910F91FF90EF90DF905F
:102E1000CF90BF90AF9008956F927F928F929F92C4
:102E2000AF92BF92CF92DF92EF92FF920F931F93D8
:102E3000CF93DF93CDB7DEB7AA970FB6F894DEBF76
:102E40000FBECDBF8C018A579D4F5C01611112C02E
:102E5000FC018081882309F498C03497C080D18018
:102E6000E280F3800E94CBE7C616D706E806F90693
:102E700008F48BC0F5011082F8018381811108C02C
:102E8000C8010E949613F8018381882309F47DC04C
:102E9000F80186A58F9385A58F9380E491E09F9399
:102EA0008F937E01F1E2EF0EF11CFF92EF920E94F0
:102EB00024F30F900F900F900F900F900F90B12C64
:102EC000F70101900020E9F73197EE19FF09BE16CE
:102ED00084F46701CB0CD11CB7FCDA94F601808135
:102EE000992787FD90950E946FF2F6018083B39435
:102EF000E7CF5801F3E3AF0EB11C40E050E0BA0158
:102F0000C5010E94338D612CCE0101966C0140E019
:102F100050E0B601C5010E947A8C181654F5712C48
:102F2000F60101900020E9F73197EC19FD097E16B2
:102F300074F44601870C911C77FC9A94F40180810B
:102F400090E00E946FF2F40180837394E9CF8A8548
:102F50008E37E9F245E050E0B701C6010E9407F361
:102F6000892BA9F6B701C8010E94691466246394ED
:102F7000CECF611004C08FEF9FEFF80104C0F801BD
:102F800085A596A5019696A785A7AA960FB6F8944B
:102F9000DEBF0FBECDBFDF91CF911F910F91FF908C
:102FA000EF90DF90CF90BF90AF909F908F907F90E9
:102FB0006F9008950F931F93CF93DF93EC018C01D3
:102FC00003531E4FC8010E94CD8DC8010E94198E67
:102FD00019821882DF91CF911F910F910895CF929E
:102FE000DF92EF92FF920F931F93CF93DF93CDB7B2
:102FF000DEB76F970FB6F894DEBF0FBECDBF8C0162
:103000006A017C018EE4E80EF11CC801805B9F4FD1
:10301000F70191838083E75CFD4F22E030E031834C
:10302000208332967183608340E050E0BA010496B9
:103030000E94338DF701808191812BE1FC01349650
:10304000DE01159601900D922A95E1F7FC0182812F
:1030500093819C838B8383ED93E09A83898396018C
:10306000AE014F5F5F4F6EEC72E0C8010E948711A6
:10307000CE0101960E94FB106F960FB6F894DEBF4A
:103080000FBECDBFDF91CF911F910F91FF90EF90B9
:10309000DF90CF9008952F923F924F925F926F9260
:1030A0007F928F929F92AF92BF92CF92DF92EF92D8
:1030B000FF920F931F93CF93DF93CDB7DEB7AC97FB
:1030C0000FB6F894DEBF0FBECDBF8C016B01342E5E
:1030D000FC018381882309F4CFC2E053FE4F808135
:1030E000882309F4FBC0211103C0EDE3F0E1CEC059
:1030F0007801F8E1EF1AFEEFFF0AF70180818111F4
:1031000003C0EDE3F0E135C0E3E4F0E1849188230E
:1031100041F09091C00095FFFCCF8093C60031969E
:10312000F5CFE8E8F2E08491882341F09091C00067
:1031300095FFFCCF8093C6003196F5CF4AE050E072
:1031400061E070E082E694E00E940A298091C0006C
:1031500085FFFCCF8AE08093C6008FE792E00E9453
:10316000E04B8AC29091C00095FFFCCF8093C600CF
:10317000319684918111F6CFE6E6F2E084918823BE
:1031800041F09091C00095FFFCCF8093C60031962E
:10319000F5CFF6018191882339F09091C00095FF19
:1031A000FCCF8093C600F6CFEBE5F2E08491882354
:1031B00041F09091C00095FFFCCF8093C6003196FE
:1031C000F5CFF70180813DE8B32EB801B89E600DC0
:1031D000711D112463517E4FC8010E94CC14F70168
:1031E0008081F801B89EE00DF11D1124E351FE4FDE
:1031F0008191882339F09091C00095FFFCCF809396
:10320000C600F6CFE5E5F2E08491882341F0909185
:10321000C00095FFFCCF8093C6003196F5CF5801D2
:10322000F2E8AF1AFDEFBF0AF501408151816281DA
:1032300073812AE030E082E694E00E94392980918F
:10324000C00085FFFCCF8AE08093C600F701208193
:10325000F80184E0289FE00DF11D1124AF014751D2
:103260005E4FF50180819181A281B381FA01808353
:103270009183A283B3832F5FF701208329C09091AC
:10328000C00095FFFCCF8093C600319684918111D8
:10329000F6CFE4E4F2E08491882341F09091C000FD
:1032A00095FFFCCF8093C6003196F5CFF601819152
:1032B000882339F09091C00095FFFCCF8093C60021
:1032C000F6CF8091C00085FFFCCF8AE08093C600D6
:1032D000C80183539E4F0E94198E30C0F801E851F7
:1032E000FE4F1082EDE3F0E18491882341F090914C
:1032F000C00095FFFCCF8093C6003196F5CFE3E385
:10330000F2E08491882341F09091C00095FFFCCFBA
:103310008093C6003196F5CFF6018191882339F06C
:103320009091C00095FFFCCF8093C600F6CF8091AE
:10333000C00085FFFCCF8AE08093C600F8011282AE
:10334000CE0101965C010E94F11028019EE4490E15
:10335000511CC8018F96F20191838083F601808110
:103360008F3209F077C07601FFEFEF1AFF0A2AE0EB
:10337000222EE114F10409F473C06FE270E0C7017A
:103380000E94ECF24C01009709F46BC0E816F906B4
:1033900008F067C03C016E187F08A301B701CE0199
:1033A00080960E9415F3E0E2F0E0EC0FFD1FE60DC1
:1033B000F71D1082FE01B0968191882339F090911B
:1033C000C00095FFFCCF8093C600F6CF8091C0006F
:1033D00085FFFCCF2092C600F201608171816115EA
:1033E000710519F06C5F7F4F02C060E070E021E072
:1033F000AE01405E5F4FCE0105960E942290811182
:1034000021C0EFE1F2E08491882341F09091C00067
:1034100095FFFCCF8093C6003196F5CFFE01B096A4
:103420008191882339F09091C00095FFFCCF809363
:10343000C600F6CF8091C00085FFFCCF8EE280935E
:10344000C60017C1F201B182A0827401FFEFEF1A2A
:10345000FF0A8FCFC801805B9F4FF2019183808369
:103460007601C80183539E4F4C01F2016081718146
:10347000332009F4A4C06115710519F06C5F7F4F0A
:1034800002C060E070E021E0A701C4010E94229028
:10349000811103C0E7EEF1E076C0980126583D4F58
:1034A000F40181899289A389B489F9018083918388
:1034B000A283B383E1E1F2E08491882341F090910B
:1034C000C00095FFFCCF8093C6003196F5CFF70181
:1034D0008191882339F09091C00095FFFCCF8093B3
:1034E000C600F6CFE9E0F2E08491882341F09091A4
:1034F000C00095FFFCCF8093C6003196F5CFF9014F
:1035000040815181628173812AE030E082E694E05B
:103510000E9439298091C00085FFFCCF8AE080930A
:10352000C600F801E258FD4F108211821282138208
:10353000EBEFF1E08491882341F09091C00095FF7A
:10354000FCCF8093C6003196F5CF8091C00085FFF7
:10355000FCCF8AE08093C600A70160E070E0C8015C
:103560000E94EF17F8018289882319F0C80142965A
:1035700001C0C70160E07BC09091C00095FFFCCF07
:103580008093C600319684918111F6CFF701819125
:10359000882339F09091C00095FFFCCF8093C6003E
:1035A000F6CFE4EEF1E08491882309F462C09091B3
:1035B000C00095FFFCCF8093C6003196F4CF611513
:1035C000710519F06C5F7F4F02C060E070E026E586
:1035D000A701C4010E942290811125C0E0EDF1E015
:1035E0008491882341F09091C00095FFFCCF809397
:1035F000C6003196F5CFF7018191882339F090917B
:10360000C00095FFFCCF8093C600F6CFEDECF1E053
:103610008491882371F19091C00095FFFCCF809335
:10362000C6003196F5CF81E0F8018083EBEBF1E045
:103630008491882341F09091C00095FFFCCF809346
:10364000C6003196F5CFF6018191882339F090912B
:10365000C00095FFFCCF8093C600F6CF8091C000DC
:1036600085FFFCCF8AE08093C60060E0C7010E941E
:1036700010B3C5010E94FB10AC960FB6F894DEBFE4
:103680000FBECDBFDF91CF911F910F91FF90EF90B3
:10369000DF90CF90BF90AF909F908F907F906F9072
:1036A0005F904F903F902F90089521E0FC0121837F
:1036B00020E040E00C944B18CF92DF92EF92FF9203
:1036C0000F931F93CF93DF93CDB7DEB76F970FB6EE
:1036D000F894DEBF0FBECDBF8C016C012EE4C20E8C
:1036E000D11C805B9F4FF60191838083E75CFD4F87
:1036F00021E030E0318320837801F7E7EF1AFDEF16
:10370000FF0AF7011182108240E050E0BA010496EE
:103710000E94338DF601808191812BE1FC0134966A
:10372000DE01159601900D922A95E1F7FC01828148
:1037300093819C838B8383ED93E09A83898320E03C
:1037400030E0AE014F5F5F4F6EEC72E0C8010E9447
:103750008711CE0101960E94FB10F70180819181B3
:103760006F960FB6F894DEBF0FBECDBFDF91CF913D
:103770001F910F91FF90EF90DF90CF900895AF923F
:10378000BF92CF92DF92EF92FF920F931F93CF934E
:10379000DF93CDB7DEB76F970FB6F894DEBF0FBEDD
:1037A000CDBF8C015B01CE0101960E94F110F801A2
:1037B000E95AFF4F80817801811104C02FE2E20EA7
:1037C000F11C03C030E5E30EF11C670144E0C40EB8
:1037D000D11C21E0A501B601CE0105960E942290E0
:1037E00081112DC0EDE3F0E18491882341F09091A7
:1037F000C00095FFFCCF8093C6003196F5CFEAE27A
:10380000F1E08491882341F09091C00095FFFCCFB6
:103810008093C6003196F5CFF5018191882339F068
:103820009091C00095FFFCCF8093C600F6CF8091A9
:10383000C00085FFFCCF8AE08093C60030C0F8014D
:10384000EB55FE4F80818A30D0F491E0980F908341
:10385000F8012FE1829FE00DF11D1124CF01815964
:103860009F4F2BE1F601DC01149601900D922A95F1
:10387000E1F7F70122813381FC0133832283005B6E
:103880001F4F8BE1FE013596D801149601900D92E1
:103890008A95E1F78B819C81F80193838283CE0125
:1038A00001960E94FB106F960FB6F894DEBF0FBE14
:1038B000CDBFDF91CF911F910F91FF90EF90DF90DF
:1038C000CF90BF90AF900895CF93DF93FC01EB555D
:1038D000FE4F20812223D1F021502083EC013FE1D3
:1038E000239FC00DD11D1124C159DF4F805B9F4F15
:1038F0002BE1FE013496DC01149601900D922A957D
:10390000E1F72A813B81FC0133832283DF91CF9150
:103910000895EF92FF920F931F93CF93DF93EC01E3
:103920000E948D9F8E0108511E4FF80180819E01DB
:1039300023533E4F79018823A9F1C9010E94198EB2
:10394000F801808181508083BE01FDE88F9F600D6A
:10395000711D112463517E4F21E041E0CE010E9490
:103960004B18F8018081FE0124E0829FE00DF11DDB
:103970001124E751FE4F4081518162817381FE0124
:10398000E258FD4F4083518362837383C7010E94D5
:10399000338DCE01DF91CF911F910F91FF90EF906A
:1039A0000C94C014C9010E94198E1A828EE191E014
:1039B0000E948C2B8091C60E8823F9F01092C60EBF
:1039C000C0916705D0E0CC0FDD1FC952DD4E688184
:1039D0007981882777FD8095982F0E94C9EB2091E7
:1039E0004C0130914D0140914E0150914F010E9488
:1039F0002AED181614F419821882DF91CF911F91C5
:103A00000F91FF90EF900895AF92BF92DF92EF92E7
:103A1000FF920F931F93CF93DF931F92CDB7DEB723
:103A20008C015B01460F8AE0D82E4A1509F43BC091
:103A30007501F50161915F01F801808191814983F0
:103A40000E9456F5F801808191810E944EF5F701A0
:103A500090814981891701F1EDE3F0E18491882398
:103A600041F09091C00095FFFCCF8093C600319645
:103A7000F5CFECEDF5E08491882341F09091C00002
:103A800095FFFCCF8093C6003196F5CF8091C000A2
:103A900085FFFCCFD092C600F8018081918101960C
:103AA00091838083C2CF0F90DF91CF911F910F91AF
:103AB000FF90EF90DF90BF90AF900895EF92FF924C
:103AC0000F931F93CF93DF931F92CDB7DEB78C0177
:103AD0007B01460FF8018081918149830E944EF558
:103AE000F70181937F01F801808191810196918393
:103AF000808349814E11EECF0F90DF91CF911F91BE
:103B00000F91FF90EF900895CF92DF92EF92FF9286
:103B10000F931F93CF93DF93CDB7DEB765970FB6A3
:103B2000F894DEBF0FBECDBF19861A861B861C8691
:103B300080E390E3A0E3B0E08D839E83AF83B887FA
:103B400084E690E09A8B898B44E0BE016B5F7F4FE7
:103B5000CE0141960E94041D40E167E07FE0CE0166
:103B600041960E94041D40E167E17FE0CE0141964D
:103B70000E94041D40E167EF7EE0CE0141960E9465
:103B8000041D44E06FEE7EE0CE0141960E94041DCC
:103B900044E06BEE7EE0CE0141960E94041D44E0BD
:103BA00067EE7EE0CE0141960E94041D44E063EF83
:103BB0007EE0CE0141960E94041D44E067ED7EE068
:103BC000CE0141960E94041D44E067E27FE0CE01F1
:103BD00041960E94041D44E063EE7EE0CE014196D2
:103BE0000E94041D44E06FED7EE0CE0141960E94EC
:103BF000041D44E06BED7EE0CE0141960E94041D61
:103C00004CE06AE675E0CE0141960E94041D83E017
:103C10008D8B8C8B1B8A19861A861B861C8641E02D
:103C2000BE016D5E7F4FCE0141960E94041D44E0AF
:103C3000BE01675F7F4FCE0141960E94041D41E0A7
:103C4000BE016B5E7F4FCE0141960E94041D41E094
:103C5000BE016C5E7F4FCE0141960E94041D10E0B4
:103C60009D898C89212F30E0989FC001112444E068
:103C7000281739074CF4BE01675F7F4FCE0141968C
:103C80000E94041D1F5FECCF65E171E0CE014196FB
:103C90000E94041D19861A861B861C861AE0115084
:103CA00049F044E0BE01675F7F4FCE0141960E941C
:103CB000041DF5CF42E06CE473E1CE0141960E9411
:103CC000041D42E06AE473E1CE0141960E94041DA6
:103CD00042E068E473E1CE0141960E94041D42E097
:103CE00066E473E1CE0141960E94041D42E064E463
:103CF00073E1CE0141960E94041D42E062E473E14B
:103D0000CE0141960E94041DC12C90E8D92E9BE360
:103D1000E92E95E4F92E11111DC044E063E971E02C
:103D2000CE0141960E94041D44E06FE871E0CE018F
:103D300041960E94041D44E06BE871E0CE0141967B
:103D40000E94041D44E067E871E0CE0141960E94A4
:103D5000041D1CC0C986DA86EB86FC8644E0BE01E1
:103D6000675F7F4FCE0141960E94041D19861A8617
:103D70001B861C8604E0015049F044E0BE01675FE9
:103D80007F4FCE0141960E94041DF5CF1F5F143076
:103D900011F642E062E171E0CE0141960E94041DFD
:103DA00044E06FE971E0CE0141960E94041D44E0B9
:103DB0006BE971E0CE0141960E94041D44E067E981
:103DC00071E0CE0141960E94041D80E290E0988B44
:103DD0008F8742E0BE01615F7F4FCE0141960E9416
:103DE000041D80E090E0A0E8BFE389879A87AB8755
:103DF000BC8744E0BE01675F7F4FCE0141960E94C1
:103E0000041D41E066E775E0CE0141960E94041D65
:103E100010E011110CC080913B0190913C01A091E8
:103E20003D01B0913E0189879A87AB87BC8744E00A
:103E3000BE01675F7F4FCE0141960E94041D1F5F48
:103E4000143039F786E592E3A3E3B0E089839A83DF
:103E5000AB83BC8384E690E09E878D8744E0BE01FF
:103E60006F5F7F4FCE010D960E94041DEDE3F0E1E0
:103E70008491882341F09091C00095FFFCCF8093FE
:103E8000C6003196F5CF49895A89662757FD609556
:103E9000762F8AEC95E00E94922AE2ECF5E084917C
:103EA000882341F09091C00095FFFCCF8093C6001D
:103EB0003196F5CF8091C00085FFFCCF8AE08093DA
:103EC000C60065960FB6F894DEBF0FBECDBFDF917A
:103ED000CF911F910F91FF90EF90DF90CF900895B9
:103EE000AF92BF92DF92EF92FF920F931F93CF9307
:103EF000DF93CDB7DEB7E0970FB6F894DEBF0FBE05
:103F0000CDBF80E1ECE0F2E0DE01919601900D92F0
:103F10008A95E1F780E1ECE1F2E0DE015196019053
:103F20000D928A95E1F780E1ECE2F2E0DE01119674
:103F300001900D928A95E1F77E0181E2E80EF11C75
:103F400007E01FE0BE016F5E7F4F47E15FE09E012B
:103F50002F5F3F4FE7EFAE2EEEE0BE2ED12CF701E4
:103F600081919191A191B1917F01F80181939193F8
:103F7000A193B1938F01FB0181919191A191B19195
:103F8000BF01FA0181939193A193B193AF01F9011C
:103F900081919191A191B1919F01F50181939193AB
:103FA000A193B1935F01D394F4E0DF12D8CF0E94C4
:103FB000997580E090E0AAE7B4E48093EF0E9093C7
:103FC000F00EA093F10EB093F20E40E050E86BE3D8
:103FD00075E44093EB0E5093EC0E6093ED0E7093EE
:103FE000EE0E8093E70E9093E80EA093E90EB09347
:103FF000EA0E1092F30E1092F40E1092F50E10923B
:10400000F60E80E29EE4A0E0B0E08093270F90934C
:10401000280FA093290FB0932A0F1092D70E109259
:10402000D80E1092D90E1092DA0E80E090E0A0EA3D
:10403000B1E48093E30E9093E40EA093E50EB09369
:10404000E60E8DEC9CECACECBEE38093DF0E90931F
:10405000E00EA093E10EB093E20E80E090E0A0EAC3
:10406000B0E48093DB0E9093DC0EA093DD0EB09352
:10407000DE0E109272051092730510927405109264
:10408000750510926E0510926F05109270051092D2
:10409000710510926A0510926B0510926C051092D2
:1040A0006D0586E696E6A6E8BFEB80931501909332
:1040B0001601A0931701B093180184EB90E0909340
:1040C0004D1380934C138CE390E090934B138093AB
:1040D0004A1310924913109248138CED90E090937C
:1040E00047138093461384E690E0909345138093A2
:1040F0004413109243131092421380E090E0A0E426
:10410000B1E48093930190939401A0939501B093AF
:1041100096016DEC7CEC8CEC9EE30E9401AE60930A
:104120008F0170939001809391019093920160E0D0
:1041300070E08CEA92E40E940FAE60938B01709362
:104140008C0180938D0190938E0180E090E0A8EC2B
:10415000B2E48093870190938801A0938901B09382
:104160008A0184E190E090931301809312010E94F0
:1041700099A181E79DE9A0EAB3E480939F01909320
:10418000A001A093A101B093A20162E578EB8AEBB4
:1041900091E40E9401AE60939B0170939C01809317
:1041A0009D0190939E0160E078E28AE894E40E9489
:1041B0000FAE60939701709398018093990190934B
:1041C0009A011092760580E090E0A0E4B0E480933C
:1041D0003B0190933C01A0933D01B0933E010E94AE
:1041E000154EEDE3F0E18491882341F09091C000F9
:1041F00095FFFCCF8093C6003196F5CFEBE7F5E055
:104200008491882341F09091C00095FFFCCF80936A
:10421000C6003196F5CF8091C00085FFFCCF8AE0C3
:104220008093C600E0960FB6F894DEBF0FBECDBFF8
:10423000DF91CF911F910F91FF90EF90DF90BF9092
:10424000AF900895CF93C82F882389F14091070F2D
:104250005091080F6091090F70910A0F83E695E065
:104260000E94802A40910B0F50910C0F60910D0F0E
:1042700070910E0F80E695E00E94802A40910F0F0A
:104280005091100F6091110F7091120F8DE595E014
:104290000E94802A4091130F5091140F6091150FC6
:1042A0007091160F8AE595E00E94802A2FC0EDE3F9
:1042B000F0E18491882341F09091C00095FFFCCFFC
:1042C0008093C6003196F5CFEBE6F5E08491882324
:1042D00041F09091C00095FFFCCF8093C6003196CD
:1042E000F5CF8091C00085FFFCCF8AE08093C600A7
:1042F000EDE3F0E18491882309F4A8CF9091C00008
:1043000095FFFCCF8093C6003196F4CF8091C0001A
:1043100085FFFCCF8AE08093C600CC2389F14091D1
:10432000170F5091180F6091190F70911A0F87E3B2
:1043300095E00E94802A40911B0F50911C0F6091C4
:104340001D0F70911E0F84E395E00E94802A40911A
:104350001F0F5091200F6091210F7091220F81E368
:1043600095E00E94802A4091230F5091240F609184
:10437000250F7091260F8EE295E00E94802A2FC0B3
:10438000EDE3F0E18491882341F09091C00095FF26
:10439000FCCF8093C6003196F5CFE0E4F5E0849140
:1043A000882341F09091C00095FFFCCF8093C60018
:1043B0003196F5CF8091C00085FFFCCF8AE08093D5
:1043C000C600EDE3F0E18491882309F4A8CF909131
:1043D000C00095FFFCCF8093C6003196F4CF80914A
:1043E000C00085FFFCCF8AE08093C600CC2389F112
:1043F0004091F70E5091F80E6091F90E7091FA0EFF
:1044000087E095E00E94922A4091FB0E5091FC0EAD
:104410006091FD0E7091FE0E84E095E00E94922A5C
:104420004091FF0E5091000F6091010F7091020FAB
:1044300081E095E00E94922A4091030F5091040F71
:104440006091050F7091060F8EEF94E00E94922A02
:104450002FC0EDE3F0E18491882341F09091C000FA
:1044600095FFFCCF8093C6003196F5CFE0E1F5E0F3
:104470008491882341F09091C00095FFFCCF8093F8
:10448000C6003196F5CF8091C00085FFFCCF8AE051
:104490008093C600EDE3F0E18491882309F4A8CF6E
:1044A0009091C00095FFFCCF8093C6003196F4CF69
:1044B0008091C00085FFFCCF8AE08093C600CC23AA
:1044C00029F14091EF0E5091F00E6091F10E709134
:1044D000F20E83EC94E00E94802A4091EB0E509102
:1044E000EC0E6091ED0E7091EE0E80EC94E00E9467
:1044F000802A4091E70E5091E80E6091E90E70918C
:10450000EA0E8DEB94E00E94802A2FC0EDE3F0E1EB
:104510008491882341F09091C00095FFFCCF809357
:10452000C6003196F5CFECECF4E08491882341F09D
:104530009091C00095FFFCCF8093C6003196F5CFD7
:104540008091C00085FFFCCF8AE08093C600EDE338
:10455000F0E18491882309F4B4CF9091C00095FFD5
:10456000FCCF8093C6003196F4CF8091C00085FFC8
:10457000FCCF8AE08093C600CC2309F449C0409167
:10458000F30E5091F40E6091F50E7091F60E81E0ED
:1045900094E00E94802A4091D70E5091D80E6091ED
:1045A000D90E7091DA0E8EEF93E00E94802A40912E
:1045B000270F5091280F6091290F70912A0F8BEFD0
:1045C00093E00E94922A4091E30E5091E40E609194
:1045D000E50E7091E60E88EF93E00E94802A4091EC
:1045E000DF0E5091E00E6091E10E7091E20E85EFCA
:1045F00093E00E94802A4091DB0E5091DC0E609186
:10460000DD0E7091DE0E82EF93E00E94802A2FC0B3
:10461000EDE3F0E18491882341F09091C00095FF93
:10462000FCCF8093C6003196F5CFEAE0F4E08491A8
:10463000882341F09091C00095FFFCCF8093C60085
:104640003196F5CF8091C00085FFFCCF8AE0809342
:10465000C600EDE3F0E18491882309F490CF9091B6
:10466000C00095FFFCCF8093C6003196F4CF8091B7
:10467000C00085FFFCCF8AE08093C600CC2329F1DF
:1046800040916A0550916B0560916C0570916D05C4
:1046900087ED93E00E94802A40916E0550916F054E
:1046A000609170057091710584ED93E00E94802AFD
:1046B0004091720550917305609174057091750574
:1046C00081ED93E00E94802A2FC0EDE3F0E1849118
:1046D000882341F09091C00095FFFCCF8093C600E5
:1046E0003196F5CFE0EEF3E08491882341F090918C
:1046F000C00095FFFCCF8093C6003196F5CF809126
:10470000C00085FFFCCF8AE08093C600EDE3F0E1B6
:104710008491882309F4B4CF9091C00095FFFCCF19
:104720008093C6003196F4CF8091C00085FFFCCF06
:104730008AE08093C600CC2329F140914C1350911C
:104740004D13662757FD6095762F89EA93E00E9406
:10475000922A40914A1350914B13662757FD60955A
:10476000762F86EA93E00E94922A40914813509156
:104770004913662757FD6095762F83EA93E00E94E0
:10478000922A2FC0EDE3F0E18491882341F09091CB
:10479000C00095FFFCCF8093C6003196F5CFE5EBC6
:1047A000F3E08491882341F09091C00095FFFCCF05
:1047B0008093C6003196F5CF8091C00085FFFCCF75
:1047C0008AE08093C600EDE3F0E18491882309F448
:1047D000B4CF9091C00095FFFCCF8093C600319676
:1047E000F4CF8091C00085FFFCCF8AE08093C600A3
:1047F000CC2329F14091461350914713662757FD6A
:104800006095762F87E993E00E94922A40914413A5
:1048100050914513662757FD6095762F84E993E004
:104820000E94922A4091421350914313662757FDEC
:104830006095762F81E993E00E94922A0DC0EDE306
:10484000F0E184918823B1F29091C00095FFFCCFF4
:104850008093C6003196F5CF8091C00085FFFCCFD4
:104860008AE08093C600CC2309F441C040919301B3
:104870005091940160919501709196018AE793E0BF
:104880000E94802A60918F01709190018091910126
:10489000909192010E9408AEAB01BC0187E793E0C2
:1048A0000E94802A60918B0170918C0180918D0112
:1048B00090918E010E9416AEAB01BC0184E793E09B
:1048C0000E94802A4091870150918801609189015E
:1048D00070918A0181E793E00E94802A6091120121
:1048E000709113018EE693E00E946E2A2FC0EDE3D3
:1048F000F0E18491882341F09091C00095FFFCCFB6
:104900008093C6003196F5CFE3E8F3E084918823E5
:1049100041F09091C00095FFFCCF8093C600319686
:10492000F5CF8091C00085FFFCCF8AE08093C60060
:10493000EDE3F0E18491882309F498CF9091C000D1
:1049400095FFFCCF8093C6003196F4CF8091C000D4
:1049500085FFFCCF8AE08093C600CC2369F14091AB
:104960009F015091A0016091A1017091A20185E683
:1049700093E00E94802A60919B0170919C0180913C
:104980009D0190919E010E9408AEAB01BC0182E6A0
:1049900093E00E94802A6091970170919801809124
:1049A000990190919A010E9416AEAB01BC018FE56E
:1049B00093E00E94802A0DC0EDE3F0E1849188230A
:1049C00071F29091C00095FFFCCF8093C6003196A4
:1049D000F5CF8091C00085FFFCCF8AE08093C600B0
:1049E000CC2369F040913B0150913C0160913D0125
:1049F00070913E0189E393E00E94802A45C0EDE377
:104A0000F0E18491882341F09091C00095FFFCCFA4
:104A10008093C6003196F5CFECE4F3E084918823CF
:104A200041F09091C00095FFFCCF8093C600319675
:104A3000F5CF80917605811103C0E2E4F3E00CC06C
:104A40008091C00085FFFCCF0EC09091C00095FF03
:104A5000FCCF8093C600319684918111F6CF80916E
:104A6000C00085FFFCCF8AE08093C600EDE3F0E153
:104A70008491882309F4B6CF9091C00095FFFCCFB4
:104A80008093C6003196F4CF8091C00085FFFCCFA3
:104A90008AE08093C60080917605811123C0C11100
:104AA0000DC0EDE3F0E107C09091C00095FFFCCF91
:104AB0008093C600319684918111F6CFEFE2F3E046
:104AC00007C09091C00095FFFCCF8093C60031963F
:104AD00084918111F6CF8091C00085FFFCCF8AE0E0
:104AE0008093C600CC2369F04091150150911601C6
:104AF000609117017091180181E193E00E94802A72
:104B00002EC0EDE3F0E18491882341F09091C00044
:104B100095FFFCCF8093C6003196F5CFEAE1F3E034
:104B20008491882341F09091C00095FFFCCF809341
:104B3000C6003196F5CF8091C00085FFFCCF8AE09A
:104B40008093C600EDE3F0E18491882369F29091AF
:104B5000C00095FFFCCF8093C6003196F5CF8091C1
:104B6000C00085FFFCCF8AE08093C600CF910895F6
:104B7000CF92DF92EF92FF920F931F93CF93DF9329
:104B8000CDB7DEB763970FB6F894DEBF0FBECDBFCB
:104B900084E690E0988B8F8786E592E3A3E3B0E00C
:104BA0008D839E83AF83B88744E0BE01675F7F4FEC
:104BB000CE010F960E945E1D43E050E0BE01675F8C
:104BC0007F4FCE0105960E9407F3892B19F00E94B2
:104BD000701FCCC119821A821B821C8240E167E0DF
:104BE0007FE0CE010F960E945E1D40E167E17FE00D
:104BF000CE010F960E945E1D40E167EF7EE0CE0180
:104C00000F960E945E1D0E94997544E06FEE7EE053
:104C1000CE010F960E945E1D44E06BEE7EE0CE0159
:104C20000F960E945E1D44E067EE7EE0CE010F9677
:104C30000E945E1D44E063EF7EE0CE010F960E946D
:104C40005E1D44E067ED7EE0CE010F960E945E1D82
:104C500044E067E27FE0CE010F960E945E1D44E0D3
:104C600063EE7EE0CE010F960E945E1D44E06FED84
:104C70007EE0CE010F960E945E1D44E06BED7EE06B
:104C8000CE010F960E945E1D4CE06AE675E0CE01F3
:104C90000F960E945E1D1B8A1A8A198A41E0BE0186
:104CA0006D5E7F4FCE010F960E945E1D44E0BE01F7
:104CB0006F5F7F4FCE010F960E945E1D41E0BE01E7
:104CC0006E5E7F4FCE010F960E945E1D41E0BE01D9
:104CD0006F5E7F4FCE010F960E945E1D10E09A8995
:104CE0008989212F30E0989FC001112444E02817C2
:104CF00039074CF4BE016F5F7F4FCE010F960E94C3
:104D00005E1D1F5FECCF65E171E0CE010F960E9442
:104D10005E1D19821A821B821C821AE0115049F012
:104D200044E0BE016F5F7F4FCE010F960E945E1D73
:104D3000F5CF42E06CE473E1CE010F960E945E1D58
:104D400042E06AE473E1CE010F960E945E1D42E0EC
:104D500068E473E1CE010F960E945E1D42E066E4B6
:104D600073E1CE010F960E945E1D42E064E473E1A0
:104D7000CE010F960E945E1D42E062E473E1CE0117
:104D80000F960E945E1D44E0BE016F5F7F4FCE0113
:104D90000F960E945E1D11110EC0C980DA80EB8053
:104DA000FC8020E030E84BE355E4C701B6010E94E7
:104DB00027EB811102C004E01EC0C0929301D09283
:104DC0009401E0929501F092960144E06FE871E061
:104DD000CE010F960E945E1D44E06BE871E0CE01AB
:104DE0000F960E945E1D44E067E871E0CE010F96C9
:104DF0000E945E1D0BC0015049F044E0BE016F5F90
:104E00007F4FCE010F960E945E1DF5CF1F5F1430BD
:104E100009F0B9CF42E062E171E0CE010F960E9445
:104E20005E1D44E0BE016F5F7F4FCE010F960E9472
:104E30005E1DC980DA80EB80FC8020E030E84BE327
:104E400055E4C701B6010E9427EB81110DC044E073
:104E5000BE016F5F7F4FCE010F960E945E1D44E042
:104E6000BE016F5F7F4F12C0C0929F01D092A00120
:104E7000E092A101F092A20144E06BE971E0CE0161
:104E80000F960E945E1D44E067E971E0CE010F9627
:104E90000E945E1D42E0BE01635F7F4FCE010F9610
:104EA0000E945E1D44E0BE016F5F7F4FCE010F96F2
:104EB0000E945E1D41E066E775E0CE010F960E94FC
:104EC0005E1D10E044E0BE016F5F7F4FCE010F9684
:104ED0000E945E1D11110CC089819A81AB81BC8139
:104EE00080933B0190933C01A0933D01B0933E0120
:104EF0001F5F143039F70E94154E0E9499A1EDE30F
:104F0000F0E18491882341F09091C00095FFFCCF9F
:104F10008093C6003196F5CFFE01359681918823A6
:104F200039F09091C00095FFFCCF8093C600F6CF7A
:104F30004F855889662757FD6095762F85EA95E05D
:104F40000E94922AEDE9F5E08491882341F0909146
:104F5000C00095FFFCCF8093C6003196F5CF8091BD
:104F6000C00085FFFCCF8AE08093C60080E00E94ED
:104F7000222163960FB6F894DEBF0FBECDBFDF913E
:104F8000CF911F910F91FF90EF90DF90CF900895F8
:104F90001F920F920FB60F9211240BB60F922F9300
:104FA0003F938F939F93EF93FF932091C6009FB7FA
:104FB000F894E091E30481E08E0F8F773091E40460
:104FC000831731F0F0E0ED59FB4F20838093E30429
:104FD0009FBFFF91EF919F918F913F912F910F90E4
:104FE0000BBE0F900FBE0F901F9018959A01AB014A
:104FF000211581EE38074105510549F182E0809382
:10500000C00060E079E08DE390E00E941CEF215049
:10501000310941095109CA01B90122E030E040E0FB
:1050200050E00E941CEF3093C5002093C400809193
:10503000C10080618093C1008091C100886080932D
:10504000C1008091C10080688093C10008951092D2
:10505000C00020E130E0E7CF3FB7F8942091E404AE
:105060008091E304821759F0E22FF0E0ED59FB4FF5
:10507000808190E02F5F2F772093E40402C08FEFB0
:105080009FEF3FBF08958FB7F8949091E4049093F9
:10509000E3048FBF08954F925F926F927F928F9239
:1050A0009F92AF92BF92CF92DF92EF92FF920F93B7
:1050B0001F93CF93DF93CDB7DEB7A0970FB6F894C9
:1050C000DEBF0FBECDBF5C01411551056105710505
:1050D000F1F420E030E040E350E060E070E0A096C2
:1050E0000FB6F894DEBF0FBECDBFDF91CF911F91F9
:1050F0000F91FF90EF90DF90CF90BF90AF909F9077
:105100008F907F906F905F904F900C94E3288E016A
:105110000F5F1F4FC12CD12C76014801422E512C1C
:10512000612C712C8FEFC81AD80AE80AF80ACB0153
:10513000BA01A30192010E94FAEECA01F80161933B
:105140008F01A901BC01411551056105710551F798
:10515000F1E0CF1AD108E108F108F401EC0DFD1DD2
:1051600080818A3010F440E301C047E3480F55279F
:1051700047FD5095652F752F20E030E0C5010E9456
:10518000E32881E0C81AD108E108F108EFEFCE1654
:10519000DE06EE06FE0609F7A0960FB6F894DEBF0F
:1051A0000FBECDBFDF91CF911F910F91FF90EF9078
:1051B000DF90CF90BF90AF909F908F907F906F9037
:1051C0005F904F9008952115310539F48091C0000A
:1051D00085FFFCCF4093C60008952A30310511F4B5
:1051E0000C9412290C944B28CF93DF93EC0120E010
:1051F00030E04DE050E060E070E00E94E32820E005
:1052000030E04AE050E060E070E0CE01DF91CF9105
:105210000C94E3289A01AB01662757FD6095762F21
:105220000C94E328CF92DF92EF92FF92CF93DF931B
:10523000EC016A017B0177FF10C020E030E04DE215
:1052400050E060E070E00E94E328F094E094D09495
:10525000C094C11CD11CE11CF11C2AE0B701A601BD
:10526000CE01DF91CF91FF90EF90DF90CF900C9423
:105270004B282115310539F48091C00085FFFCCF02
:105280004093C60008950C944B289A01462F50E095
:1052900060E070E00C943929CF93DF93EC019A0120
:1052A000AB0160E070E00E943929CE01DF91CF911F
:1052B0000C94F4288F929F92AF92BF92CF92DF927C
:1052C000EF92FF921F93CF93DF93EC016A017B0172
:1052D000122F20E030E0A901C701B6010E9427EBA0
:1052E00087FF0DC020E030E04DE250E060E070E06C
:1052F000CE010E94E328F7FAF094F7F8F094B12C6D
:1053000060E070E080E09FE3B11641F020E030E023
:1053100040E251E40E942EEBB394F6CF9B01AC0126
:10532000C701B6010E944EEA6B017C010E949BEB13
:105330004B015C010E94C7EB9B01AC01C701B601A8
:105340000E944DEA6B017C012AE0B501A401CE0167
:105350000E944B28112349F020E030E04EE250E05B
:1053600060E070E0CE010E94E328112321F120E0EB
:1053700030E040E251E4C701B6010E94FCED6B0150
:105380007C010E9496EB4B01AA2497FCA094BA2CB6
:10539000B501A401CE010E941229C501B4010E94E9
:1053A000C9EB9B01AC01C701B6010E944DEA6B013C
:1053B0007C011150DACFDF91CF911F91FF90EF90D8
:1053C000DF90CF90BF90AF909F908F9008950C94F6
:1053D0005A29FC0165917591859194910895809168
:1053E0007C11811103C081E080937C11089560E0FD
:1053F00083EC9CE00E945CB3EDE3F0E184918823B0
:1054000041F09091C00095FFFCCF8093C60031968B
:10541000F5CFE1EBFCE08491882341F09091C0004E
:1054200095FFFCCF8093C6003196F5CF8091C000E8
:1054300085FFFCCF8AE08093C600089580917C119F
:10544000811110927C1108950E94CBE760935B0557
:1054500070935C0580935D0590935E05089580913F
:10546000430190914401A0914501B0914601809380
:10547000350790933607A0933707B093380780918C
:10548000410190914201909378058093770584E6DD
:1054900090E090934201809341010E94242A81E090
:1054A0000C9486970E948E978091350790913607CD
:1054B000A0913707B091380780934301909344013E
:1054C000A0934501B09346018091770590917805AE
:1054D00090934201809341010C94242AFC01249171
:1054E000222341F03091C00035FFFCCF2093C6004D
:1054F0000196F4CF4AE050E082E694E00C940A2949
:10550000FC012491222341F03091C00035FFFCCFF3
:105510002093C6000196F4CF22E030E082E694E0CA
:105520000C94E729FC012491222341F03091C00022
:1055300035FFFCCF2093C6000196F4CF2AE030E07F
:1055400082E694E00C9439292091FF0630910007FF
:10555000F901E65BFA4F8083C901019664E070E0CF
:105560000E94E6EE909300078093FF068091FD066F
:105570009091FE0601969093FE068093FD06089595
:10558000CF93FC01C62F80818B33E1F02091FD0683
:105590003091FE0624303105ACF44091FF06509165
:1055A000000780E6849F9001859F300D1124BF0184
:1055B000C90183589A4F0E9400F38C2F0E94A42A9D
:1055C00081E001C080E0CF910895CF93DF93D82F81
:1055D000C92F0E94C02A882309F43CC0EDE3F0E102
:1055E0008491882341F09091C00095FFFCCF809377
:1055F000C6003196F5CFE1EFFFE08491882341F0BA
:105600009091C00095FFFCCF8093C6003196F5CFF6
:10561000ED2FFC2F8191882339F09091C00095FFE8
:10562000FCCF8093C600F6CFEFEEFFE08491882395
:1056300041F09091C00095FFFCCF8093C600319659
:10564000F5CF8091C00085FFFCCF8AE08093C60033
:1056500081E001C080E0DF91CF910895DF92EF9269
:10566000FF920F931F93CF93DF93CDB7DEB76E9763
:105670000FB6F894DEBF0FBECDBF60915F0570918D
:1056800060056115710561F14DE150E08E010F5F1C
:105690001F4FC8010E948FF21E8EF8017F01E01A91
:1056A000F10AD190DD2019F08AE0D812F7CFF80185
:1056B000EE0DFF1D108260E0C8010E94E52A8823DC
:1056C00079F0DD20B1F08FEFE81AF80A80915F05DC
:1056D000909160058E0D9F1D9093600580935F05EE
:1056E00081E020915F0530916005232B39F480E043
:1056F00005C01092600510925F05F2CF6E960FB64E
:10570000F894DEBF0FBECDBFDF91CF911F910F91F7
:10571000FF90EF90DF9008959093600580935F0570
:105720000C942E2B40E052EC61E070E082E694E0B5
:105730000E94F627E9EEFFE08491882341F09091E2
:10574000C00095FFFCCF8093C6003196F5CF8091C5
:10575000C00085FFFCCF8AE08093C600EDE3F0E156
:105760008491882341F09091C00095FFFCCF8093F5
:10577000C6003196F5CF84B780FF14C0E1EEFFE09C
:105780009491992341F02091C00025FFFCCF909384
:10579000C6003196F5CF9091C00095FFFCCF9AE0FE
:1057A0009093C60081FF14C0E1EDFFE0949199232E
:1057B00041F02091C00025FFFCCF9093C6003196A8
:1057C000F5CF9091C00095FFFCCF9AE09093C60072
:1057D00082FF14C0E0ECFFE09491992341F0209106
:1057E000C00025FFFCCF9093C6003196F5CF909175
:1057F000C00095FFFCCF9AE09093C60083FF14C0D1
:10580000E0EBFFE09491992341F02091C00025FF47
:10581000FCCF9093C6003196F5CF9091C00095FFD4
:10582000FCCF9AE09093C60085FF14C0E0EAFFE049
:105830008491882341F09091C00095FFFCCF809324
:10584000C6003196F5CF8091C00085FFFCCF8AE07D
:105850008093C60014BEE9E9FFE08491882341F0FB
:105860009091C00095FFFCCF8093C6003196F5CF94
:10587000EEE8FFE08491882341F09091C00095FF0D
:10588000FCCF8093C6003196F5CF8091C00085FF94
:10589000FCCF8AE08093C600EDE3F0E18491882399
:1058A00041F09091C00095FFFCCF8093C6003196E7
:1058B000F5CFEEE7FFE08491882341F09091C0009E
:1058C00095FFFCCF8093C6003196F5CFEDE6FFE063
:1058D0008491882341F09091C00095FFFCCF809384
:1058E000C6003196F5CFE1E6FFE08491882341F0D0
:1058F0009091C00095FFFCCF8093C6003196F5CF04
:10590000EAE5FFE08491882341F09091C00095FF83
:10591000FCCF8093C6003196F5CF8091C00085FF03
:10592000FCCF8AE08093C600EFE4FFE084918823F7
:1059300041F09091C00095FFFCCF8093C600319656
:10594000F5CFE3E4FFE08491882341F09091C0001B
:1059500095FFFCCF8093C6003196F5CF8091C000B3
:1059600085FFFCCF8AE08093C600EDE3F0E18491EF
:10597000882341F09091C00095FFFCCF8093C60032
:105980003196F5CFE4E3FFE08491882341F09091D4
:10599000C00095FFFCCF8093C6003196F5CF0E94E2
:1059A000BF924AE050E0BC0182E694E00E940A29DE
:1059B000EDE1FFE08491882341F09091C00095FFD4
:1059C000FCCF8093C6003196F5CF4AE050E060ED01
:1059D00074E082E694E00E940A298091C00085FF6D
:1059E000FCCF8AE08093C60081E080934A058093D3
:1059F0004B0580934C0580934D050E94B8250E946D
:105A0000FBC50E9414A60E94A8670E9495E30C940F
:105A10003B9F0F931F93CF93DF93009161051091EC
:105A2000620565E470E0C8010E94ECF2EC01C80177
:105A30000196209761F0188260E070E00E94C2EF4A
:105A400025E42883DF91CF911F910F91089560E0A5
:105A500070E0DF91CF911F910F910C94C2EF809174
:105A60006105909162054AE050E060E070E00196C7
:105A70000C9433F180916105909162054AE050E009
:105A800060E070E001960E9433F1CB0108950F931E
:105A90001F93CF93DF93082F112707FD1095C09117
:105AA0000307D0910407B801CE010E94ECF2909355
:105AB000620580936105892B51F4B801605E7F4FC8
:105AC000CE010E94ECF2909362058093610581E023
:105AD0002091610530916205232B09F480E0DF916C
:105AE000CF911F910F9108950F931F93CF93DF9341
:105AF00000D000D000D0CDB7DEB726E0ECE3F2E076
:105B0000DE01119601900D922A95E1F7FC01EE0F4E
:105B1000FF1F21E030E02C0F3D1FE20FF31F6081DB
:105B20007181161617061CF1EDE3F0E12491222392
:105B300041F03091C00035FFFCCF2093C600319674
:105B4000F5CFE5EDFCE02491222341F03091C00037
:105B500035FFFCCF2093C6003196F5CF2091C000D1
:105B600025FFFCCF2AE02093C6006AE070E08C019C
:105B7000000F111F000F111F01541C4F882777FDC4
:105B80008095982F0E94C9EB9B01AC01F8016081C0
:105B90007181828193810E942EEB60934301709307
:105BA0004401809345019093460126960FB6F894E0
:105BB000DEBF0FBECDBFDF91CF911F910F91089532
:105BC0008F929F92AF92BF92CF92DF92EF92FF920D
:105BD0000F931F9320E030E040E752E460914301CF
:105BE0007091440180914501909146010E942EEBF5
:105BF0004B015C01E0902D07F0902E0700912F07DC
:105C0000109130072091290730912A0740912B07E6
:105C100050912C07609125077091260780912707E6
:105C200090912807E0916705EF93E1E3CE2EE7E03E
:105C3000DE2E0E943F690F901F910F91FF90EF9011
:105C4000DF90CF90BF90AF909F908F9008954F922C
:105C50005F926F927F928F929F92AF92BF92EF92DC
:105C6000FF920F931F93CF93DF93CDB7DEB72897A3
:105C70000FB6F894DEBF0FBECDBF4B015C01809123
:105C8000430190914401A0914501B091460189835F
:105C90009A83AB83BC83412C512CF6E16F2EF4E444
:105CA0007F2E4092430150924401609245017092D0
:105CB0004601E0922D07F0922E0700932F071093D4
:105CC00030072D833E834F8358870E94E02D0E942A
:105CD0008D9F6091190170911A01882777FD809539
:105CE000982F0E94C9EB6093430170934401809305
:105CF0004501909346018092250790922607A09235
:105D00002707B09228072D813E814F815885209327
:105D1000290730932A0740932B0750932C070E94A2
:105D2000E02D0E948D9F89819A81AB81BC818093F7
:105D3000430190934401A0934501B09346012896F6
:105D40000FB6F894DEBF0FBECDBFDF91CF911F918C
:105D50000F91FF90EF90BF90AF909F908F907F90AA
:105D60006F905F904F9008954F925F926F927F92E5
:105D70008F929F92AF92BF92CF92DF92EF92FF925B
:105D80000F931F932B013C0120E030E040E752E4E9
:105D900060914301709144018091450190914601C9
:105DA0000E942EEB4B015C012091290730912A07BC
:105DB00040912B0750912C07609125077091260781
:105DC0008091270790912807E0916705EF93A1E361
:105DD000CA2EA7E0DA2E830172010E943F690F905C
:105DE0001F910F91FF90EF90DF90CF90BF90AF90F9
:105DF0009F908F907F906F905F904F9008958F92BB
:105E00009F92AF92BF92CF92DF92EF92FF920F9349
:105E10001F9320E030E040E752E40E942EEB4B015C
:105E20005C01E0901D07F0901E0700911F07109184
:105E300020072091190730911A0740911B075091B4
:105E40001C076091150770911607809117079091B4
:105E50001807E0916705EF93B1E2CB2EB7E0DB2E98
:105E60000E943F690F901F910F91FF90EF90DF907C
:105E7000CF90BF90AF909F908F9008956091430115
:105E80007091440180914501909146010C94FF2E40
:105E9000CF92DF92EF92FF920F931F93E0902D0726
:105EA000F0902E0700912F071091300720912907BD
:105EB00030912A0740912B0750912C0760912507BC
:105EC000709126078091270790912807E1E3CE2E55
:105ED000E7E0DE2E0E9488741F910F91FF90EF90F3
:105EE000DF90CF9008952F923F924F925F926F92E2
:105EF0007F928F929F92AF92BF92CF92DF92EF925A
:105F0000FF920F931F93CF93DF938C01FC01E2501C
:105F1000F04FF4902F2C332427FC3094EC01CC0F5D
:105F2000DD1FCC0FDD1FDE01AB5DB84F1D921D9252
:105F30001D921C9213970E94482F0230110519F4EC
:105F400037FC0E94EF29CE01835F9F4E0E94E92912
:105F50004B015C016F2D772767FD7095872F972F79
:105F60000E94C9EB2B013C019E012B5E384F790149
:105F700020E030E040EC5FE3C501B4010E94FCED9D
:105F8000A30192010E94FCEDF7016083718382837B
:105F90009383FE01E154FC4F80819181A281B38102
:105FA0008093430190934401A0934501B09346012F
:105FB0000E943E2F0E948D9F9E012B5D384F6901EC
:105FC000F90110821182128213820E94482F80E010
:105FD0000E9486979E012F5F3F4E5901C9010E9482
:105FE000E9299058A30192010E94FCEDF70160831A
:105FF0007183828393830E943E2F0E948D9F81E054
:106000000E948697C8010E94742DC5010E94E9294B
:106010009B01AC010E944EEAA30192010E94FCED9B
:10602000F70160837183828393830E943E2F0E94D5
:106030008D9FCE01875E9F4E0E94E9299E012659C1
:106040003A4F7901F90120813181428153810E94C7
:106050004EEAF6016083718382839383CE018F5C65
:106060009F4E0E94E9299E01255D3E4F6901F7017F
:1060700020813181428153810E944EEAF601608382
:10608000718382839383CE018B5D9F4E0E94E929A9
:106090009E01215E3E4F6901F701208131814281DD
:1060A00053810E944EEAF601608371838283938359
:1060B00002301105D1F42091150130911601409163
:1060C00017015091180160912D0770912E07809152
:1060D0002F07909130070E944DEA60932D0770932F
:1060E0002E0780932F07909330070E94482FFE01C0
:1060F000EB5EF84FCB5DD84F88819981AA81BB8137
:1061000080839183A283B383109243011092440150
:1061100010924501109246010E949397F801EE5E9D
:10612000F84F81E08083F801E15FF84F808302300F
:106130001105B1F437FE14C0DF91CF911F910F917B
:10614000FF90EF90DF90CF90BF90AF909F908F9097
:106150007F906F905F904F903F902F900C941E2AED
:10616000DF91CF911F910F91FF90EF90DF90CF9033
:10617000BF90AF909F908F907F906F905F904F9067
:106180003F902F9008958F929F92AF92BF92CF929F
:10619000DF92EF92FF920F931F930E94242A84E5CF
:1061A00091E00E9438E180E090E0A6E1B4E48093C1
:1061B000430190934401A0934501B093460160E0F0
:1061C00070E084E393EC0E94B42E0E948D9F82E0E5
:1061D00090E00E94F29F4B015C01209129073091D1
:1061E0002A0740912B0750912C0760912507709149
:1061F00026078091270790912807A1E3CA2EA7E0E0
:10620000DA2E850174010E94887489E090E10E9471
:10621000E9299B01AC01C501B4010E944EEA4B0182
:106220005C010E94B42E0E948D9F0E94939782E091
:1062300090E00E94742D89E090E10E94E9299B0181
:10624000AC010E944EEA9B01AC01C501B4010E9461
:106250004DEA0E94B42E0E948D9F0E94939782E087
:1062600090E00E94F29F60932D0770932E07809319
:106270002F07909330071F910F91FF90EF90DF90C1
:10628000CF90BF90AF909F908F900C94482F80E15B
:10629000E5E1F7E0A5E2B7E001900D928A95E1F71C
:1062A0000895EF92FF920F931F93E0902D07F090C7
:1062B0002E0700912F07109130070E94272E1F9163
:1062C0000F91FF90EF900895EF92FF920F931F931D
:1062D0007B018C012091290730912A0740912B07DF
:1062E00050912C0760912507709126078091270710
:1062F000909128070E94272E1F910F91FF90EF90F9
:1063000008954F925F926F927F928F929F92AF9279
:10631000BF92CF92DF92EF92FF920F931F93CF9392
:10632000DF9300D000D0CDB7DEB769837A838B834B
:106330009C8329013A01C801B70185010E9464319B
:1063400020E030E04CE252E4C301B2010E944EEA88
:106350004B015C0120E030E040EA51E469817A8140
:106360008B819C810E944EEAA50194010E945131CB
:10637000C0FC0E94EF290E94C33080902D079090AE
:106380002E07A0902F07B0903007C1FC0E941E2A54
:10639000033011050CF448C0E4ECFAE08491882342
:1063A00041F09091C00095FFFCCF8093C6003196DC
:1063B000F5CF23E030E049815A816B817C8182E610
:1063C00094E00E94E729EFEBFAE08491882341F002
:1063D0009091C00095FFFCCF8093C6003196F5CF19
:1063E00023E030E0B301A20182E694E00E94E729B5
:1063F000EAEBFAE08491882341F09091C00095FF88
:10640000FCCF8093C6003196F5CF23E030E0B50194
:10641000A40182E694E00E94E7298091C00085FFF4
:10642000FCCF8AE08093C600C501B4010F900F90A5
:106430000F900F90DF91CF911F910F91FF90EF90F0
:10644000DF90CF90BF90AF909F908F907F906F9094
:106450005F904F900895CF92DF92EF92FF920F934B
:106460001F93CF93DF93BBEBEB2EB3E0FB2E05E145
:1064700017E0C5E2D7E089E7C82E85E0D82EF701FE
:1064800081917F010E94472D8823D1F00E94092D20
:10649000F6012081211104C020916505222329F0F5
:1064A000288139814A815B8103C020E030E0A90165
:1064B0000E944EEAF801608371838283938309C04E
:1064C00088819981AA81BB81F80180839183A2830D
:1064D000B3830C5F1F4F2496FFEFCF1ADF0A8FEBB9
:1064E000E81683E0F80659F686E40E94472D8823D3
:1064F00099F00E94092D6B017C0120E030E0A90198
:106500000E942AED181644F4C0924301D09244012F
:10651000E0924501F0924601DF91CF911F910F91DA
:10652000FF90EF90DF90CF900895EDE3F0E184913C
:10653000882341F09091C00095FFFCCF8093C60066
:106540003196F5CFE9E9FDE08491882341F09091FF
:10655000C00095FFFCCF8093C6003196F5CFE09147
:106560000507F09106078191882339F09091C000CA
:1065700095FFFCCF8093C600F6CFE6E9FDE084915D
:10658000882341F09091C00095FFFCCF8093C60016
:106590003196F5CF08950F931F930E94CBE740915A
:1065A0004805509149054115510509F479C00091FC
:1065B0000E0110910F01209110013091110160170F
:1065C00071078207930708F479C04330510579F0C9
:1065D0003CF4413051050CF463C0EDE3F0E111C02F
:1065E0004430510509F05CC0EDE3F0E142C0EDE359
:1065F000F0E123C03091C00035FFFCCF2093C600EE
:10660000319624912111F6CFE5E8FDE02491222373
:1066100041F03091C00035FFFCCF2093C600319689
:10662000F5CF2091C00025FFFCCF37C03091C000CE
:1066300035FFFCCF2093C600319624912111F6CF6F
:10664000EFE6FDE02491222341F03091C00035FFB8
:10665000FCCF2093C6003196F5CF2091C00025FFD6
:10666000FCCF1BC03091C00035FFFCCF2093C6008B
:10667000319624912111F6CFE8E5FDE02491222303
:1066800041F03091C00035FFFCCF2093C600319619
:10669000F5CF2091C00025FFFCCF2AE02093C60053
:1066A000DC01CB01805F984DAF4FBF4F80930E014F
:1066B00090930F01A0931001B09311011F910F91BE
:1066C0000895E0E5FDE02491222379F03091C000A7
:1066D00035FFFCCF2093C6003196F5CF3091C00036
:1066E00035FFFCCF2093C6000196FC0124912111B7
:1066F000F5CFE8E3FDE08491882341F09091C0005C
:1067000095FFFCCF8093C6003196F5CF8091C000F5
:1067100085FFFCCF8AE08093C6000895BF92CF9298
:10672000DF92EF92FF920F931F93CF93DF9300D0EE
:1067300000D0CDB7DEB785E40E94472D811102C09D
:106740000E948D9F9BEBC92E93E0D92E25E2E22E6D
:1067500027E0F22E00E010E0B12CF60181916F01EC
:106760000E94472D8823A9F00E94092DF70160831C
:1067700071838283938369837A838B839C830330C1
:10678000110529F4CE0101960E947C7502C0BB243C
:10679000B3940F5F1F4FF4E0EF0EF11C04301105AE
:1067A000E1F6B1100E94482F0F900F900F900F90BC
:1067B000DF91CF911F910F91FF90EF90DF90CF90DD
:1067C000BF900895EFE5FAE08491882341F090911D
:1067D000C00095FFFCCF8093C6003196F5CF809125
:1067E000C00085FFFCCF8AE08093C6008AE397E073
:1067F0000E944C13E1E5FAE08491882341F09091E6
:10680000C00095FFFCCF8093C6003196F5CF8091F4
:10681000C00085FFFCCF8AE08093C60008950F93E7
:106820001F93CF93DF9383E50E94472D882389F13F
:106830000E943A2D8C018F3F910509F050F580E5BB
:106840000E94472D882331F00E943A2DEC0197FDDC
:1068500020C002C0CBE1D0E0E5E8F3E08191919166
:10686000C817D907B1F083E0EB3BF807B9F761E04F
:106870008C2F0E9415E9602F8C2F0E944EE9B801E1
:106880008C2F0E9475E8249721F4109369050093DA
:106890006805DF91CF911F910F910895E4E3FDE02A
:1068A0008491882341F09091C00095FFFCCF8093A4
:1068B000C6003196F5CFE0914E0584E0E89FF001E7
:1068C0001124E354FD4E408151816281738121E0A6
:1068D00030E082E694E00E94E729E1E3FDE0849164
:1068E000882341F09091C00095FFFCCF8093C600B3
:1068F0003196F5CFE0914E05F0E0EE0FFF1FE95223
:10690000FD4E60817181882777FD8095982F0E94C8
:10691000C9EBAB01BC0121E030E082E694E00E94CB
:10692000E729EDE2FDE08491882341F09091C000D9
:1069300095FFFCCF8093C6003196F5CF4091B712FA
:106940005091B8126091B9127091BA1221E030E002
:1069500082E694E00E94E729EAE2FDE08491882340
:1069600041F09091C00095FFFCCF8093C600319616
:10697000F5CF6091D5127091D612882777FD80955A
:10698000982F0E94C9EBAB01BC0121E030E082E608
:1069900094E00E94E729E5E2FDE08491882341F03C
:1069A0009091C00095FFFCCF8093C6003196F5CF43
:1069B0008FEF9FEF0E94CEA14AE050E0BC0182E63B
:1069C00094E00E940A29E1E2FDE08491882341F0ED
:1069D0009091C00095FFFCCF8093C6003196F5CF13
:1069E00080914E0590E00E94CEA14AE050E0BC01AB
:1069F00082E694E00C940A2983E50E94472D8823BF
:106A000019F00E943A2D01C080E080933907EDE330
:106A1000F0E18491882341F09091C00095FFFCCF74
:106A20008093C6003196F5CFE0E0F9E084918823A9
:106A300041F09091C00095FFFCCF8093C600319645
:106A4000F5CF8091390781110EC0ECEFF8E0849109
:106A5000882309F47EC09091C00095FFFCCF8093FD
:106A6000C6003196F4CF80E090E050E0482F2091AE
:106A7000390730E0082E02C0359527950A94E2F7D1
:106A800020FF62C0511113C0423009F140F4442389
:106A900009F1413009F057C0E0EFF8E030C0433071
:106AA00099F0443009F04FC0E4EDF8E049C0EAEF56
:106AB000F8E02491222341F33091C00035FFFCCF50
:106AC0002093C6003196F5CFE2EEF8E02EC0E9EE55
:106AD000F8E020C0E5EFF8E02491222309F433C068
:106AE0003091C00035FFFCCF2093C6003196F4CF23
:106AF0003091C00035FFFCCF2093C6003196249121
:106B00002111F6CF20C03091C00035FFFCCF20937B
:106B1000C600319624912111F6CF15C03091C000E6
:106B200035FFFCCF2093C600319624912111F6CF7A
:106B30000AC03091C00035FFFCCF2093C6003196CB
:106B400024912111F6CF51E001968830910509F08A
:106B50008DCF8091C00085FFFCCF8AE08093C60076
:106B6000089583E50E94472D882349F10E943A2D1C
:106B7000823010F1E3E4F0E18491882341F09091B8
:106B8000C00095FFFCCF8093C6003196F5CFEDE4B1
:106B9000F7E08491882341F09091C00095FFFCCFED
:106BA0008093C6003196F5CF8091C00085FFFCCF61
:106BB0008AE08093C6000895813009F444C088E4D7
:106BC0000E94472D882391F00E943A2D8639910525
:106BD0003CF0853021E092072CF084E091E002C087
:106BE00086E990E090934D1380934C1386E40E94C5
:106BF000472D882381F00E943A2D8F3F910519F08F
:106C000014F08FEF90E097FF02C080E090E0909347
:106C100049138093481382E40E94472D882309F486
:106C200054C00E943A2D8530910534F08A36910582
:106C30002CF089E690E002C085E090E090934B1341
:106C400080934A13089588E40E94472D882391F089
:106C50000E943A2D863991053CF0853021E092075B
:106C60002CF084E091E002C086E990E09093471315
:106C70008093461386E40E94472D882381F00E946A
:106C80003A2D8F3F910519F014F08FEF90E097FFA8
:106C900002C080E090E0909343138093421382E41B
:106CA0000E94472D882389F00E943A2D8530910556
:106CB00034F08A3691052CF089E690E002C085E038
:106CC00090E09093451380934413089583E50E94C8
:106CD000472D882399F00E94092D20E030E04AE7F3
:106CE00054E40E94FCED0E949BEB60931B017093A7
:106CF0001C0180931D0190931E01089588E50E9458
:106D0000472D811111C089E50E94472D81110CC0CA
:106D10008AE50E94472D811107C085E40E94472D16
:106D2000811102C00C9409A00E948D9F88E50E94E9
:106D3000472D882319F05E9A1092120789E50E9468
:106D4000472D882319F05E9A109213078AE50E9456
:106D5000472D882321F0159A10921407089508955D
:106D60003F924F925F926F927F928F929F92AF92DB
:106D7000BF92CF92DF92EF92FF920F931F93CF9328
:106D8000DF934BEB842E43E0942EC7E0DFE057E126
:106D9000A52E5FE0B52E07EC1EE0312CF4018191A9
:106DA0004F010E94472D882309F458C0F3E03F1299
:106DB0004FC00E94092D6B017C0120E030E040EAC9
:106DC00051E40E9427EB87FF3EC0A701960168812E
:106DD00079818A819B810E942EEB2B013C019B01D2
:106DE000AC016091DB0E7091DC0E8091DD0E909114
:106DF000DE0E0E94FCED6093DB0E7093DC0E809340
:106E0000DD0E9093DE0EA3019201F5016081718188
:106E1000828193810E94FCEDF501608371838283FE
:106E20009383F80160817181828193810E94C7EB15
:106E3000A30192010E94FCED0E949BEBF80160838C
:106E4000718382839383C882D982EA82FB8206C0DF
:106E50000E94092D688379838A839B8333942496C7
:106E6000F4E0AF0EB11C0C5F1F4F84E0381296CFD8
:106E7000DF91CF911F910F91FF90EF90DF90CF9016
:106E8000BF90AF909F908F907F906F905F904F904A
:106E90003F9008958F929F92AF92BF92CF92DF92D0
:106EA000EF92FF92E5EAF7E08491882341F0909118
:106EB000C00095FFFCCF8093C6003196F5CF40917E
:106EC000250750912607609127077091280722E037
:106ED00030E082E694E00E94E729E1EAF7E084915D
:106EE000882341F09091C00095FFFCCF8093C600AD
:106EF0003196F5CF4091290750912A0760912B07D1
:106F000070912C0722E030E082E694E00E94E729AD
:106F1000EDE9F7E08491882341F09091C00095FF5E
:106F2000FCCF8093C6003196F5CF40912D0750914C
:106F30002E0760912F077091300722E030E082E643
:106F400094E00E94E729E9E9F7E08491882341F081
:106F50009091C00095FFFCCF8093C6003196F5CF8D
:106F60004091310750913207609133077091340797
:106F700022E030E082E694E00E94E7298FB7F8949F
:106F8000409138115091391160913A1170913B1133
:106F900080903C1190903D11A0903E11B0903F1117
:106FA000C0904011D0904111E0904211F0904311F7
:106FB0008FBFEEE8F7E08491882341F09091C00004
:106FC00095FFFCCF8093C6003196F5CF2AE030E0E4
:106FD00082E694E00E94E328EAE8F7E084918823BF
:106FE00041F09091C00095FFFCCF8093C600319690
:106FF000F5CF2AE030E0B501A40182E694E00E94DA
:10700000E328E6E8F7E08491882341F09091C000FE
:1070100095FFFCCF8093C6003196F5CF2AE030E093
:10702000B701A60182E694E00E94E3288091C000A7
:1070300085FFFCCF8AE08093C600FF90EF90DF9041
:10704000CF90BF90AF909F908F9008958F929F9216
:10705000AF92BF92CF92DF92EF92FF920E948D9FEC
:1070600084E591E00E9438E10E942F2A80E1E5E268
:10707000F7E0A5E1B7E001900D928A95E1F7109253
:10708000430110924401109245011092460188E597
:107090000E94472DD82E89E50E94472DE82E8AE5CB
:1070A0000E94472DF82ED11005C0E11007C091E0D5
:1070B000982705C0EE2011F0982F01C090E0909322
:1070C0001401911102C0DD2021F080E090E00E94C7
:1070D000732F80911401811102C0EE2021F081E014
:1070E00090E00E94732F80911401882309F45BC003
:1070F0000E94482F80E090E0A4EFB2E4809315074F
:1071000090931607A0931707B093180780E090E0BC
:10711000A1E1B3E48093190790931A07A0931B078A
:10712000B0931C0780912D0790912E07A0912F07F7
:10713000B091300780931D0790931E07A0931F07FF
:10714000B093200780E090E4ACE9B5E4809343017C
:1071500090934401A0934501B09346010E943E2FB5
:107160000E948D9F8091150790911607A091170797
:10717000B09118078093250790932607A0932707BF
:10718000B09328078091190790911A07A0911B07C7
:10719000B0911C078093290790932A07A0932B078F
:1071A000B0932C0745C0FF2009F470C080910F07F1
:1071B000882309F469C080911007882309F464C00A
:1071C0008090250790902607A0902707B090280769
:1071D000C0902907D0902A07E0902B07F0902C0749
:1071E00020E030E040EA51E4C501B4010E942AEDFC
:1071F00087FD23C020E030E041E653E4C501B4013F
:107200000E9427EB1816CCF020E030E04CE252E46C
:10721000C701B6010E942AED87FD0FC020E030E0D3
:1072200048E753E4C701B6010E9427EB18162CF07B
:1072300082E090E00E94732F29C060E087E09DE02B
:107240000E945CB3EDE3F0E18491882341F09091DA
:10725000C00095FFFCCF8093C6003196F5CFE6EFD6
:10726000FCE08491882341F09091C00095FFFCCF11
:107270008093C6003196F5CF8091C00085FFFCCF8A
:107280008AE08093C60002C00E94F7290E94482F1E
:1072900080E00E9486978091350790913607A091F3
:1072A0003707B09138078093430190934401A0932E
:1072B0004501B093460180917705909178059093B0
:1072C0004201809341010E94242A0E949397FF90DB
:1072D000EF90DF90CF90BF90AF909F908F900C94E5
:1072E0004A370E94EF290E948D9F0E942F2A80E03A
:1072F00090E0A6E1B4E48093430190934401A0930D
:107300004501B09346010E94C330E2EBFAE084915C
:10731000882341F09091C00095FFFCCF8093C60078
:107320003196F5CF27E137EB41ED58E36091250722
:107330007091260780912707909128070E944EEAB6
:10734000AB01BC0122E030E082E694E00E94E72934
:10735000EDEAFAE08491882341F09091C00095FF16
:10736000FCCF8093C6003196F5CF27E137EB41ED96
:1073700058E36091290770912A0780912B0790911B
:107380002C070E944EEAAB01BC0122E030E082E60D
:1073900094E00E94E729E8EAFAE08491882341F02A
:1073A0009091C00095FFFCCF8093C6003196F5CF39
:1073B00027E137EB41ED58E360912D0770912E07DF
:1073C00080912F07909130070E944EEAAB01BC01DB
:1073D00022E030E082E694E00E94E7298091C0003C
:1073E00085FFFCCF8AE08093C6000E94522A0E944B
:1073F0001E2A0C944A372F923F924F925F926F92BF
:107400007F928F929F92AF92BF92CF92DF92EF9234
:10741000FF920F931F93CF93DF93CDB7DEB7C15F7A
:10742000D1090FB6F894DEBF0FBECDBF80910F0714
:10743000882341F080911007882321F08091110763
:1074400081111BC0CF50DF4F0FB6F894DEBF0FBEC7
:10745000CDBFDF91CF911F910F91FF90EF90DF9003
:10746000CF90BF90AF909F908F907F906F905F90E4
:107470004F903F902F900C94F72986E50E94472D5E
:107480008823F9F00E943A2DC753DF4F8883C95CE7
:10749000D040853070F0EDE1FAE08491882309F462
:1074A0001FC69091C00095FFFCCF8093C600319617
:1074B000F4CFC753DF4F2881C95CD0402223A1F00D
:1074C00006C031E0C753DF4F3883C95CD040EDEFD1
:1074D000F9E08491882341F09091C00095FFFCCFA2
:1074E0008093C6003196F5CF80E50E94472D882312
:1074F000C1F00E943A2DC952DF4F8883C75DD0404A
:1075000084508F32A0F0E9EDF9E08491882309F4EA
:10751000E7C59091C00095FFFCCF8093C6003196DF
:10752000F4CF8AE0C952DF4F8883C75DD0404090D6
:1075300025075090260760902707709028078090B5
:10754000290790902A07A0902B07B0902C07C09095
:107550002D07D0902E07E0902F07F090300785E49C
:107560000E94472DC851DF4F8883C85ED04088E510
:107570000E94472D882329F10E94092DC453DF4F13
:10758000688379838A839B83CC5CD04020E030E0A1
:1075900044E352EC0E9427EB87FD10C020E030E06E
:1075A00049E353E4C453DF4F688179818A819B8129
:1075B000CC5CD0400E942AED18169CF487ED99E02F
:1075C0003AC020E030E040EA51E4C301B2010E9439
:1075D0004DEAC453DF4F688379838A839B83CC5CF5
:1075E000D04089E50E94472D882309F43FC00E94BE
:1075F000092DC053DF4F688379838A839B83C05DE5
:10760000D04020E030E040EA50EC0E9427EB87FDBC
:1076100010C020E030E042E253E4C053DF4F688105
:1076200079818A819B81C05DD0400E942AED181625
:107630006CF585ED99E0CF50DF4F0FB6F894DEBFC3
:107640000FBECDBFDF91CF911F910F91FF90EF90B3
:10765000DF90CF90BF90AF909F908F907F906F9072
:107660005F904F903F902F900C94613320E030E07A
:107670004CE252E4C501B4010E944DEAC053DF4F11
:10768000688379838A839B83C05DD0408CE40E94A9
:10769000472D182F882329F10E943A2DCC52DF4F15
:1076A0008883C45DD040803170F0E2EAF9E08491D3
:1076B000882309F415C59091C00095FFFCCF8093F5
:1076C000C6003196F4CFCC52DF4F9881C45DD040D4
:1076D000913061F4A2E0CC52DF4FA883C45DD0406A
:1076E00005C0CC52DF4F1882C45DD04083E50E94B4
:1076F000472D882349F0112369F0B1E0C852DF4FCC
:10770000B883C85DD04012C0C852DF4F1882C85D30
:10771000D0400CC0E1E0C852DF4FE883C85DD040E4
:10772000F7E0CC52DF4FF883C45DD040C753DF4F42
:107730002881C95CD0402330E8F420E030E040E705
:1077400051E4C701B6010E944EEA6B017C0184E559
:1077500091E00E9438E120E030E040EF51E4C701C1
:10776000B6010E9427EB87FF12C0C701B6010E9435
:1077700064310DC0E8E8F9E084918823F1F290913A
:10778000C00095FFFCCF8093C6003196F5CF20E076
:1077900030E04CE252E4C053DF4F688179818A8146
:1077A0009B81C05DD0400E944EEAC652DF4F688385
:1077B00079838A839B83CA5DD04020E030E040EA31
:1077C00051E4C453DF4F688179818A819B81CC5C0D
:1077D000D0400E944EEAC252DF4F688379838A8389
:1077E0009B83CE5DD040C652DF4F288139814A81CC
:1077F0005B81CA5DD0400E9451310E942F2AC7533D
:10780000DF4F3881C95CD040232E312CC851DF4F67
:107810008881C85ED040882319F083E090E002C0E0
:1078200081E090E051016C01E12CF12C00E711E4C2
:10783000C053DF4F288139814A815B81C05DD040D0
:10784000C453DF4F688179818A819B81CC5CD040B1
:107850000E948131A801970160912D0770912E0738
:1078600080912F07909130070E944EEA0E94643168
:10787000DE011196CB52DF4FB983A883C55DD0409E
:10788000C653DF4F19821882CA5CD040CC52DF4FFA
:10789000F881C45DD040EF2FF0E03197CA51DF4F3F
:1078A000F983E883C65ED040C952DF4F3881C75D97
:1078B000D040232F30E0C251DF4F39832883CE5E82
:1078C000D04021503109C051DF4F39832883C05F38
:1078D000D040C653DF4F8881CA5CD040C751DF4FCC
:1078E0008883C95ED0400E94CBE70E9404EA64EF1F
:1078F00071E080E090E00E94FAE7CC52DF4F98817F
:10790000C45DD04091111FC0C652DF4F288139811C
:107910004A815B81CA5DD040C252DF4F6881798164
:107920008A819B81CE5DD0400E945131C851DF4F8A
:10793000A881C85ED040AA2309F4D6C15101F3E062
:10794000CF2ED12CE4C128E631E040E050E060E0E9
:1079500070E0CB010E9430EA0E94C9EB6B017C0110
:107960002AE030E040E050E060E070E0CB010E94AF
:1079700030EA0E94C9EB20E030E040EA50E40E9487
:107980002AED18161CF40FEF1FEF02C001E010E003
:107990002FE130E040E050E065E070E080E090E012
:1079A0000E9430EA0E94C9EBCE51DF4F6883798391
:1079B0008A839B83C25ED040C753DF4FB881C95CC6
:1079C000D040B43099F5AB01BC0186E799E00E9444
:1079D000802AB701A6018BE699E00E94802A64E61E
:1079E00070E080E090E00E94FAE70130110519F0A4
:1079F000E7EBF2E012C0EFECF2E08191882381F036
:107A00009091C00095FFFCCF8093C600F6CF909177
:107A1000C00095FFFCCF8093C60081918111F7CF04
:107A200064E670E080E090E00E94FAE7C752DF4F22
:107A30001882C95DD040C801AA2797FDA095BA2F2A
:107A4000C651DF4F88839983AA83BB83CA5ED04027
:107A5000C752DF4FF881C95DD0408F2F90E0CA51E7
:107A6000DF4F28813981C65ED040821793070CF022
:107A70004BCFC852DF4F9881C85DD040992399F011
:107A8000C651DF4F688179818A819B81CA5ED0406F
:107A90000E94C9EB9B01AC010E944EEA20E030E05D
:107AA00040E952E420C02DE230E040E050E069E1DE
:107AB00070E080E090E00E9430EA2B013C01C6516A
:107AC000DF4F688179818A819B81CA5ED0400E94A4
:107AD000C9EB4B015C01C301B2010E94C9EB9B01E0
:107AE000AC01C501B4010E94FCED9B01AC01C701D2
:107AF000B6010E944EEA6B017C0120E030E044EBCD
:107B000053E40E942AED18164CF420E030E044EBD8
:107B100053E4C701B6010E944DEAEDCF20E030E00A
:107B2000A901C701B6010E9427EB87FF0BC020E027
:107B300030E044EB53E4C701B6010E944EEA6B010A
:107B40007C01ECCF2BED3FE049E450E4C701B601E6
:107B50000E94FCED20E030E044E353E40E942EEB71
:107B60002B013C010E942BEBCE51DF4F2881398144
:107B70004A815B81C25ED0400E94FCED9B01AC015A
:107B8000C252DF4F688179818A819B81CE5DD0406E
:107B90000E944EEA4B015C01C301B2010E945FEEFC
:107BA000CE51DF4F288139814A815B81C25ED0404E
:107BB0000E94FCED9B01AC01C652DF4F68817981C8
:107BC0008A819B81CA5DD0400E944EEA2B013C0114
:107BD00020E030E044E352ECC501B4010E9427EB01
:107BE00087FD11C020E030E04DE453E4C501B4014D
:107BF0000E942AED18166CF4812C912C0DE4A02E15
:107C000003E4B02E06C0812C912C14E3A12E12ECBB
:107C1000B12E20E030E040EA50ECC301B2010E94F6
:107C200027EB87FD11C020E030E04DE453E4C301B1
:107C3000B2010E942AED18166CF4412C512CBDE4BF
:107C40006B2EB3E47B2E06C0412C512CA0EA6A2E89
:107C5000A0EC7A2EC753DF4FA881C95CD040A43076
:107C600089F5EFEEF2E08191882339F09091C00020
:107C700095FFFCCF8093C600F6CFB501A40187E63F
:107C800099E00E94802AB301A20183E699E00E9454
:107C9000802A40912D0750912E0760912F077091F7
:107CA00030078DE599E00E94802A8091C00085FF11
:107CB000FCCFBAE0B093C60067E370E080E090E0EC
:107CC0000E94FAE7A3019201C501B4010E9451315B
:107CD000C752DF4FE881C95DD040EF5FC752DF4F29
:107CE000E883C95DD040B4CEC653DF4FE881F98147
:107CF000CA5CD040C051DF4F28813981C05FD0407D
:107D00005101E217F30729F5E2E0CE2ED12CE12C48
:107D1000F12C00E711E4C053DF4F288139814A81FB
:107D20005B81C05DD040C453DF4F688179818A8117
:107D30009B81CC5CD0400E948131CB52DF4FA88127
:107D4000B981C55DD0406D937D938D939C931397BE
:107D500022C0C12CD12CE12CF12C00E711E4C0533E
:107D6000DF4F288139814A815B81C05DD040C45397
:107D7000DF4F688179818A819B81CC5CD0400E94F1
:107D80008131CB52DF4FE881F981C55DD0406083FE
:107D900071838283938310E0C12CD12C7601E1E0C2
:107DA000F0E0EC0FFD1F24E0129FE00DF11D112407
:107DB0002081318142815381C701B6010E944EEA80
:107DC0006B017C011F5FC751DF4F3881C95ED04016
:107DD000311728F7C653DF4F08811981CA5CD0409C
:107DE0000F5F1F4FB801882777FD8095982F0E945D
:107DF000C9EB4B015C019B01AC01C701B6010E94BC
:107E00002EEB2B013C01C653DF4F1882CA5CD040D9
:107E1000C12CD12C7601E1E0F0E0EC0FFD1FC65340
:107E2000DF4F9881CA5CD04084E0989FE00DF11D3F
:107E30001124A301920160817181828193810E944A
:107E40004DEA9B01AC010E94FCED9B01AC01C70116
:107E5000B6010E944EEA6B017C01C653DF4FA88138
:107E6000CA5CD040AF5FC653DF4FA883CA5CD04026
:107E7000C751DF4FB881C95ED040BA1760F6A5017F
:107E800094010E942EEB0E9469EE6B017C01C753A6
:107E9000DF4FE881C95CD040E23008F473C04AE0AB
:107EA00050E0B80182E694E00E940A29E8E5F9E092
:107EB0008491882341F09091C00095FFFCCF80937E
:107EC000C6003196F5CF4AE050E0C251DF4F6881DD
:107ED0007981CE5ED04082E694E00E940A29E1E5F5
:107EE000F9E08491882341F09091C00095FFFCCF88
:107EF0008093C6003196F5CF40912D0750912E0703
:107F000060912F077091300726E030E082E694E020
:107F10000E94E72962E370E080E090E00E94FAE7C7
:107F2000C753DF4FF881C95CD040F23091F1E9E4EA
:107F3000F9E08491882341F09091C00095FFFCCF37
:107F40008093C6003196F5CF26E030E0B301A20160
:107F500082E694E00E94E729EEE3F9E08491882329
:107F600041F09091C00095FFFCCF8093C600319600
:107F7000F5CF26E030E0B701A60182E694E00E944A
:107F8000E72907C0C753DF4F2881C95CD0402223AF
:107F900039F08091C00085FFFCCF3AE03093C600F5
:107FA00062E370E080E090E00E94FAE720E030E0D9
:107FB00040EA50E460912D0770912E0780912F07C1
:107FC000909130070E944EEA0E946431CB52DF4FFD
:107FD00088819981C55DD0400496CB52DF4F99834B
:107FE0008883C55DD040C952DF4F9881C75DD040BE
:107FF000091738F4C653DF4F19830883CA5CD04091
:1080000068CCC753DF4FA881C95CD040AA2311F1C7
:10801000E7E3F9E08491882341F09091C00095FF57
:10802000FCCF8093C6003196F5CF26E030E0B30157
:10803000A20182E694E00E94E7298091C00085FFBA
:10804000FCCF8AE08093C60069E170E080E090E0B8
:108050000E94FAE7E2E2F9E08491882341F09091EE
:10806000C00095FFFCCF8093C6003196F5CF26E087
:1080700030E0B701A60182E694E00E94E7298091F2
:10808000C00085FFFCCF8AE08093C6008091C000CD
:1080900085FFFCCF8AE08093C60069E170E080E054
:1080A00090E00E94FAE70E94522ACF50DF4F0FB6AD
:1080B000F894DEBF0FBECDBFDF91CF911F910F911E
:1080C000FF90EF90DF90CF90BF90AF909F908F90F8
:1080D0007F906F905F904F903F902F900C944A3715
:1080E000CF50DF4F0FB6F894DEBF0FBECDBFDF918C
:1080F000CF911F910F91FF90EF90DF90CF90BF90A5
:10810000AF909F908F907F906F905F904F903F9037
:108110002F900895E8E0F3E08191882339F0909161
:10812000C00095FFFCCF8093C600F6CF8091C000C1
:1081300085FFFCCF8AE08093C600EEE7F7E08491EC
:10814000882341F09091C00095FFFCCF8093C6003A
:108150003196F5CF329903C0E9EFF2E009C0E3E0D0
:10816000F3E006C09091C00095FFFCCF8093C6005D
:1081700081918111F7CF8091C00085FFFCCF8AE00B
:108180008093C600E6E7F7E08491882341F0909160
:10819000C00095FFFCCF8093C6003196F5CF339990
:1081A00003C0E9EFF2E009C0E3E0F3E006C090911C
:1081B000C00095FFFCCF8093C60081918111F7CF5D
:1081C0008091C00085FFFCCF8AE08093C600EEE678
:1081D000F7E08491882341F09091C00095FFFCCF97
:1081E0008093C6003196F5CF349B03C0E9EFF2E0EF
:1081F00009C0E3E0F3E006C09091C00095FFFCCF1A
:108200008093C60081918111F7CF8091C00085FFD6
:10821000FCCF8AE08093C600089583E50E94472D35
:108220008823F9F00E94092DAB01BC014093EF0EA9
:108230005093F00E6093F10E7093F20E4093E70EA0
:108240005093E80E6093E90E7093EA0E85E297E092
:108250000E94802A8091C00085FFFCCF8AE0809335
:10826000C60080E50E94472D8823B9F00E94092DA1
:10827000AB01BC014093EF0E5093F00E6093F10EF2
:108280007093F20E88E097E00E94802A8091C000EF
:1082900085FFFCCF8AE08093C60082E50E94472DCF
:1082A0008823B9F00E94092DAB01BC014093EB0E6D
:1082B0005093EC0E6093ED0E7093EE0E89EE96E007
:1082C0000E94802A8091C00085FFFCCF8AE08093C5
:1082D000C60084E50E94472D8823B9F00E94092D2D
:1082E000AB01BC014093E70E5093E80E6093E90E9A
:1082F0007093EA0E8BEC96E00E94802A8091C00079
:1083000085FFFCCF8AE08093C600089583E50E9434
:10831000472D882351F00E94092D6093F30E70932E
:10832000F40E8093F50E9093F60E84E50E94472D8F
:10833000882351F00E94092D6093D70E7093D80EB8
:108340008093D90E9093DA0E82E40E94472D882301
:1083500061F00E94092D0E949BEB6093270F7093A0
:10836000280F8093290F90932A0F88E50E94472DAC
:10837000882351F00E94092D6093E30E7093E40E60
:108380008093E50E9093E60E8AE50E94472D8823A0
:1083900051F00E94092D6093DF0E7093E00E8093E0
:1083A000E10E9093E20E85E40E94472D882351F060
:1083B0000E94092D6093DB0E7093DC0E8093DD0E1E
:1083C0009093DE0E089585E40E94472D811110C020
:1083D00080E50E94472D8823A9F00E94092D609313
:1083E00093017093940180939501909396010AC034
:1083F0000E94092D0E9496EB161617064CF7E3E42F
:10840000F0E1D5C089E40E94472D882361F00E94E5
:10841000092D0E9401AE60938F01709390018093AB
:1084200091019093920184E40E94472D882361F08A
:108430000E94092D0E940FAE60938B0170938C01F6
:1084400080938D0190938E0183E40E94472D8823B1
:1084500051F00E94092D60938701709388018093E9
:10846000890190938A018CE40E94472D882341F072
:108470000E94092D0E9496EB7093130160931201E4
:108480008091120190911301C39734F082E390E040
:1084900090931301809312010E9499A1EDE3F0E102
:1084A0008491882341F09091C00095FFFCCF809388
:1084B000C6003196F5CFE1E2F3E08191882339F0EF
:1084C0009091C00095FFFCCF8093C600F6CF4091FD
:1084D000930150919401609195017091960122E071
:1084E00030E082E694E00E94E729E5E2F3E0819142
:1084F000882339F09091C00095FFFCCF8093C6008F
:10850000F6CF60918F0170919001809191019091CF
:1085100092010E9408AEAB01BC0122E030E082E68D
:1085200094E00E94E729E9E2F3E08191882339F0A1
:108530009091C00095FFFCCF8093C600F6CF60916C
:108540008B0170918C0180918D0190918E010E9420
:1085500016AEAB01BC0122E030E082E694E00E945E
:10856000E729EDE2F3E08191882339F09091C00092
:1085700095FFFCCF8093C600F6CF409187015091C4
:1085800088016091890170918A0122E030E082E6E1
:1085900094E00E94E7298091C00085FFFCCF1AC0BB
:1085A0009091C00095FFFCCF8093C60031968491D6
:1085B0008111F6CFE1E3F3E08191882339F09091C6
:1085C000C00095FFFCCF8093C600F6CF8091C0001D
:1085D00085FFFCCF8AE08093C600089580E50E9465
:1085E000472D882351F00E94092D60939F017093BD
:1085F000A0018093A1019093A20189E40E94472DDC
:10860000882361F00E94092D0E9401AE60939B01B6
:1086100070939C0180939D0190939E0184E40E943D
:10862000472D882361F00E94092D0E940FAE6093B0
:108630009701709398018093990190939A010E94F9
:1086400099A1EDE3F0E18491882341F09091C0007D
:1086500095FFFCCF8093C6003196F5CFE1E2F3E0C1
:108660008191882339F09091C00095FFFCCF8093D1
:10867000C600F6CF40919F015091A0016091A101E9
:108680007091A20122E030E082E694E00E94E729A6
:10869000E5E2F3E08191882339F09091C00095FFE5
:1086A000FCCF8093C600F6CF60919B0170919C0136
:1086B00080919D0190919E010E9408AEAB01BC018A
:1086C00022E030E082E694E00E94E729E9E2F3E06C
:1086D0008191882339F09091C00095FFFCCF809361
:1086E000C600F6CF60919701709198018091990131
:1086F00090919A010E9416AEAB01BC0122E030E0DD
:1087000082E694E00E94E7298091C00085FFFCCFBB
:108710008AE08093C6000895EF92FF920F93CF9363
:10872000DF9385E40E94472D882321F00E943A2D93
:10873000EC0102C0C0E0D0E083E40E94472D882312
:1087400021F00E943A2D7C0103C095E0E92EF12C26
:1087500085E50E94472D882329F00E943A2D01E0EB
:10876000892B09F400E083E50E94472D882319F046
:108770000E94092D06C0D7FD09C060E070E086E1C7
:1087800093E4209739F410924E0504C060E070E045
:108790008CE892E410924905109248059701AE01C9
:1087A0000E947CA781E090E0909349058093480562
:1087B000DF91CF910F91FF90EF9008952F923F920C
:1087C0004F925F926F927F928F929F92AF92BF92E1
:1087D000CF92DF92EF92FF920F931F93CF93DF938D
:1087E000CDB7DEB768970FB6F894DEBF0FBECDBF2A
:1087F0008CE0E5E2F7E0DE01119601900D928A959A
:10880000E1F78CE0EAE6F5E0DE011D9601900D92BD
:108810008A95E1F72FE0222E27E0322E4E018DE0DF
:10882000880E911CFE0131965F0100E010E0F1011D
:1088300081911F01882309F480C0F5014080518097
:1088400062807380F801E15EFE4F208131814281B8
:108850005381F801E55DFE4F6081718182819381D2
:108860000E944EEA20E030E040E05FE30E94FCED31
:108870009B01AC01C301B2010E942AED181644F419
:10888000C801875E9F4E0E94E9296B017C0103C0ED
:10889000C12CD12C7601A7019601C301B2010E941F
:1088A0004DEA2B013C0120E030E040EA51EC0E940F
:1088B0002AED18161CF0E3E4F0E125C020E030E0DA
:1088C00040EA51E4C301B2010E9427EB87FFF3CFD6
:1088D000A3019201F40160817181828193810E94E0
:1088E0004DEAF4016083718382839383F501C08232
:1088F000D182E282F38221C09091C00095FFFCCF2B
:108900008093C600319684918111F6CFEEEAF6E0AD
:108910008491882341F09091C00095FFFCCF809313
:10892000C6003196F5CF8091C00085FFFCCF8AE06C
:108930008093C60080EA96E022C0F4E08F0E911C7E
:108940000C5F1F4F84E0A80EB11C0C30110509F01C
:108950006ECF8CE0FE013196A5E2B7E001900D925A
:108960008A95E1F78CE0FE013D96AAE6B5E001901C
:108970000D928A95E1F70E94482F80E996E068966B
:108980000FB6F894DEBF0FBECDBFDF91CF911F9120
:108990000F91FF90EF90DF90CF90BF90AF909F909E
:1089A0008F907F906F905F904F903F902F900C949E
:1089B00075B3CF92DF92EF92FF92EDE3F0E18491F5
:1089C000882341F09091C00095FFFCCF8093C600B2
:1089D0003196F5CFE7E8F6E08491882341F0909155
:1089E000C00095FFFCCF8093C6003196F5CF8091F3
:1089F000C00085FFFCCF80E28093C6008AE50E941C
:108A0000472D882309F452C00E94092D6B017C0177
:108A100020E030E040EA51EC0E942AED87FD0AC0D8
:108A200020E030E040EA51E4C701B6010E9427EBA4
:108A300018161CF4EFE7F6E018C0C0921501D092AA
:108A40001601E0921701F092180122E030E0B70120
:108A5000A60182E694E00E94E72934C09091C0000C
:108A600095FFFCCF8093C600319684918111F6CF9B
:108A70004AE050E06CEE7FEF82E694E00E940A2923
:108A8000E7E7F6E08491882341F09091C00095FFDC
:108A9000FCCF8093C6003196F5CF4AE050E064E108
:108AA00070E082E694E00E940A290CC04091150112
:108AB00050911601609117017091180184E796E0BA
:108AC0000E94802A8091C00085FFFCCF8AE08093BD
:108AD000C600FF90EF90DF90CF900895CF92DF9285
:108AE000EF92FF92882361F1EDE3F0E194919923F5
:108AF00041F02091C00025FFFCCF9093C600319635
:108B0000F5CF9091C00095FFFCCF94E59093C600FF
:108B10004AE050E0682F82E694E00E944529E1E3B4
:108B2000F3E08191882339F09091C00095FFFCCF4C
:108B30008093C600F6CF8091C00085FFFCCF40C077
:108B400010924E0586E40E94472D882399F00E94DA
:108B5000092D6B017C0120E030E0A9010E942AED83
:108B6000181644F4C0924301D0924401E0924501AA
:108B7000F0924601EDE3F0E18491882341F0909179
:108B8000C00095FFFCCF8093C6003196F5CFE2E49C
:108B9000F3E08191882339F09091C00095FFFCCFDC
:108BA0008093C600F6CF6091670570E04AE050E020
:108BB00082E694E00E940A298091C00085FFFCCFE4
:108BC0008AE08093C600FF90EF90DF90CF900895E9
:108BD0000E94242AE0910107F0910207E65BFA4F18
:108BE00080818823A1F0E8E6F6E08491882341F0B3
:108BF0009091C00095FFFCCF8093C6003196F5CFD1
:108C00008091C00085FFFCCF8AE08093C600089564
:108C100082E694E00E944328EBE6F6E08491882304
:108C200041F09091C00095FFFCCF8093C600319633
:108C3000F5CF40910707509108076091090770919F
:108C40000A074F5F5F4F6F4F7F4F2AE030E082E6A9
:108C500094E00E94E3288091C00085FFFCCF8AE069
:108C60008093C6000C94E845CF93C62FE3E4F0E16F
:108C70002491222379F03091C00035FFFCCF20935E
:108C8000C6003196F5CF3091C00035FFFCCF209360
:108C9000C6000196FC0124912111F5CF40910707F0
:108CA000509108076091090770910A072AE030E0A7
:108CB00082E694E00E94E3288091C00085FFFCCF0B
:108CC0008AE08093C600C1110E9408461092640594
:108CD00010926305CF9108958F929F92AF92BF92A9
:108CE000CF92DF92EF92FF92CF93DF93EC01C0908F
:108CF0002B01D0902C01E0902D01F0902E01A701C6
:108D00009601688179818A819B810E9427EB87FF88
:108D100004C0C882D982EA82FB82C0902F01D09021
:108D20003001E0903101F0903201A70196016C8191
:108D30007D818E819F810E9427EB87FF04C0CC82BA
:108D4000DD82EE82FF82C0901501D0901601E09086
:108D50001701F090180120E030E0A901C701B60129
:108D60000E9427EB87FF0AC020E030E0A901C7017D
:108D7000B6010E944EEA6B017C0103C0C12CD12CCC
:108D800076018090720590907305A0907405B09064
:108D9000750520E030E0A901C501B4010E9427EB70
:108DA00087FF08C0A5019401C701B6010E944EEAE1
:108DB0006B017C01209133013091340140913501E8
:108DC00050913601C701B6010E944EEA6B017C0149
:108DD0009B01AC01688579858A859B850E9427EB7C
:108DE00087FF04C0C886D986EA86FB86C0901F012B
:108DF000D0902001E0902101F0902201A70196017E
:108E0000688179818A819B810E942AED181624F459
:108E1000C882D982EA82FB82C0902301D0902401CB
:108E2000E0902501F0902601A70196016C817D81DB
:108E30008E819F810E942AED181624F4CC82DD8257
:108E4000EE82FF82C0902701D0902801E090290196
:108E5000F0902A01A7019601688579858A859B850E
:108E60000E942AED181624F4C886D986EA86FB8665
:108E7000DF91CF91FF90EF90DF90CF90BF90AF90B8
:108E80009F908F9008958F929F92AF92BF92CF92B2
:108E9000DF92EF92FF920F931F93CF93DF93EC013A
:108EA0008B018091390783FD90C0FB018080918008
:108EB000A280B380288139814A815B81C501B401D8
:108EC0000E944DEA6B017C0120E030E0A9010E9484
:108ED00027EB882309F479C0E091670524E0E29F3D
:108EE000F0011124E354FD4E20910A0130910B0151
:108EF00040910C0150910D016081718182819381BB
:108F00000E9427EB87FF25C088829982AA82BB82B4
:108F1000EDE3F0E18491882341F09091C00095FF4A
:108F2000FCCF8093C6003196F5CFEEE4F6E0849155
:108F3000882341F09091C00095FFFCCF8093C6003C
:108F40003196F5CF8091C00085FFFCCF8AE08093F9
:108F5000C600C701B6010E9496EB97FF07C0909527
:108F60008095709561957F4F8F4F9F4F6D3C7140FD
:108F70008105910554F1F80180819181A281B3812D
:108F800088839983AA83BB83EDE3F0E184918823EE
:108F900041F09091C00095FFFCCF8093C6003196C0
:108FA000F5CFE0E3F6E08491882341F09091C00092
:108FB00095FFFCCF8093C6003196F5CF8091C0001D
:108FC00085FFFCCF8AE08093C600DF91CF911F918F
:108FD0000F91FF90EF90DF90CF90BF90AF909F9058
:108FE0008F90089585E197E00E946C460E94242AA4
:108FF00061E277E081E397E00E9443472091150703
:109000003091160740911707509118076091250776
:109010007091260780912707909128070E9427EBDF
:10902000811117C02091190730911A0740911B0731
:1090300050911C076091290770912A0780912B0796
:1090400090912C070E9427EB811103C00E943E2FB4
:109050001CC06091410170914201882777FD809585
:10906000982F0E94C9EB2091430130914401409117
:109070004501509146010E94FCED20E030E048ECB3
:1090800052E40E942EEB0E94FF2E0C9447312F9247
:109090003F924F925F926F927F928F929F92AF9288
:1090A000BF92CF92DF92EF92FF920F931F93CF93D5
:1090B000DF93CDB7DEB7C654D1090FB6F894DEBF43
:1090C0000FBECDBF1C017EA76DA7142FDB01149628
:1090D0008D909D90AD90BC901797CD90DD90ED90C8
:1090E000FC90A5019401C701B6010E9437ED2396BB
:1090F0006CAF7DAF8EAF9FAF239780912507909186
:109100002607A0912707B09128078D8F9E8FAF8FDC
:10911000B8A3A7019601BC01CD010E944EEA6FAB36
:1091200078AF89AF9AAF8091290790912A07A091D3
:109130002B07B0912C0789A39AA3ABA3BCA3A501CD
:109140009401BC01CD010E944EEA6BAF7CAF8DAFA4
:109150009EAF80912D0790912E07A0912F07B0917F
:1091600030078D8B9E8BAF8BB88F9C01AD01D101E9
:1091700018966D917D918D919C911B970E944DEA5F
:109180006DA37EA38FA398A7D1011C968D919D916D
:109190000D90BC91A02D27968CAF9DAFAEAFBFAF09
:1091A00027978091310790913207A0913307B091B2
:1091B000340789A79AA7ABA7BCA7D701C601B058A7
:1091C000898F9A8FAB8FBC8FD501C401B058898B22
:1091D0009A8BAB8BBC8BD1018D919D910D90BC91E5
:1091E000A02D8FA798ABA9ABBAAB2FA938AD49ADCD
:1091F0005AADBC01CD010E944DEA6B017C01D10149
:1092000014968D919D910D90BC91A02D8BAB9CAB34
:10921000ADABBEAB2BAD3CAD4DAD5EADBC01CD013C
:109220000E944DEA4B015C01A7019601698D7A8D80
:109230008B8D9C8D0E94FCED2B013C01A5019401BE
:1092400069897A898B899C890E94FCED9B01AC011C
:10925000C301B2010E944EEA2B013C01A501940119
:10926000698D7A8D8B8D9C8D0E94FCED4B015C018C
:10927000A701960169897A898B899C890E94FCEDF6
:109280009B01AC01C501B4010E944DEAA30192010A
:109290000E94C1EA6B017C0120E030E0A9010E943C
:1092A00027EB87FF0AC02BED3FE049EC50E4C701F4
:1092B000B6010E944EEA6B017C01112351F02BEDA7
:1092C0003FE049EC50E4C701B6010E944DEA6B0152
:1092D0007C012FA538A949A95AA96D8D7E8D8F8D46
:1092E00098A10E9427EB81111FC02BA93CA94DA971
:1092F0005EA969A17AA18BA19CA10E9427EB811193
:1093000013C020E030E0A901C701B6010E9427EB9D
:1093100081110AC02BED3FE049EC50E4C701B601D2
:109320000E944EEA6B017C0123962CAD3DAD4EAD03
:109330005FAD2397C701B6010E94FCED2DA13EA1B0
:109340004FA158A55F770E9437ED4B015C012FE6D6
:1093500032E143E85AE30E9427EB87FDC3C1C50110
:10936000B4010E9404EC0E949BEB7E8F6D8FFB0189
:10937000EF2B21F421E030E03E8F2D8FAD8DBE8D9F
:10938000BD0180E090E00E94C7EB4B015C019B01B6
:10939000AC01C701B6010E942EEB2B013C01A501D7
:1093A00094016DA17EA18FA198A50E942EEB6FA7BD
:1093B00078AB89AB9AAB29A53AA54BA55CA52796B6
:1093C0006CAD7DAD8EAD9FAD27970E944DEAA50196
:1093D00094010E942EEB6BAB7CAB8DAB9EAB20E07F
:1093E00030E040E05FE3C301B2010E94FCEDA30165
:1093F00092010E94FCED9B01AC0160E070E080E80E
:109400009FE30E944DEA6DA37EA38FA398A78D8949
:109410009E89AF89B88D89879A87AB87BC8789A5D4
:109420009AA5ABA5BCA58D879E87AF87B88B6091A9
:10943000410170914201882777FD8095982F0E9405
:10944000C9EB209143013091440140914501509175
:1094500046010E94FCED20E030E040E752E40E942B
:109460002EEB20E030E048EC52E40E942EEB69A79E
:109470007AA78BA79CA71D8AA1E0B0E0BAA3A9A3F5
:1094800089A19AA1AD8DBE8D8A179B0708F00DC1E9
:10949000BD89B9310CF042C02DA13EA14FA158A504
:1094A00069897A898B899C890E94FCED6B017C011A
:1094B000A3019201698D7A8D8B8D9C8D0E94FCEDAC
:1094C000A70196010E944EEA6B017C012DA13EA1ED
:1094D0004FA158A5698D7A8D8B8D9C8D0E94FCEDD6
:1094E0004B015C01A301920169897A898B899C896E
:1094F0000E94FCED9B01AC01C501B4010E944DEA44
:10950000698F7A8F8B8F9C8FED89EF5FED8BA60132
:10951000B701498B5A8B6B8B7C8B6BC029A13AA10D
:10952000B90180E090E00E94C7EBA30192010E9484
:10953000FCED6B017C010E942BEB698B7A8B8B8B92
:109540009C8BC701B6010E945FEE4B015C01ADA58B
:10955000BEA5CD90DD90ED90FC901397F7FAF094B6
:10956000F7F8F09414968D919D910D90BC91A02DDB
:109570008D8B9E8BAF8BB88F29893A894B895C89FB
:10958000C701B6010E94FCED698F7A8F8B8F9C8F8B
:10959000A50194016D897E898F89988D0E94FCEDCB
:1095A0009B01AC01698D7A8D8B8D9C8D0E944EEA5A
:1095B000698F7A8F8B8F9C8FA5019401C701B601AB
:1095C0000E94FCED6B017C0129893A894B895C89F9
:1095D0006D897E898F89988D0E94FCED9B01AC017D
:1095E000C701B6010E944DEA698B7A8B8B8B9C8BED
:1095F0001D8A298D3A8D4B8D5C8D6FA978AD89AD13
:109600009AAD0E944EEA69837A838B839C83298971
:109610003A894B895C896BAD7CAD8DAD9EAD0E9466
:109620004EEA6D837E838F8398872FA538A949A939
:109630005AA969857A858B859C850E944EEA69873F
:109640007A878B879C872BA93CA94DA95EA96D853C
:109650007E858F8598890E944EEA6D877E878F87E9
:10966000988BCE0101960E946C46E984FA840B85A2
:109670001C852D813E814F81588569817A818B813E
:109680009C81E0916705EF9389A49AA4ABA4BCA444
:10969000FE013D966F010E943F6929A13AA12F5F0B
:1096A0003F4F3AA329A30F90EBCE6101BCE0CB0E54
:1096B000D11CF101E084F184028513852481358178
:1096C000468157816081718182819381E091670534
:1096D000EF9389A49AA4ABA4BCA40E943F690E9402
:1096E00047310F90CA5BDF4F0FB6F894DEBF0FBE55
:1096F000CDBFDF91CF911F910F91FF90EF90DF9041
:10970000CF90BF90AF909F908F907F906F905F9021
:109710004F903F902F9008951F93CF93DF93CDB735
:10972000DEB728970FB6F894DEBF0FBECDBF182F57
:1097300080914701882351F10E942B3289E40E94D5
:10974000472D882319F00E94092D03C060E070E0C6
:10975000CB0169837A838B839C838AE40E94472DA3
:10976000882319F00E94092D03C060E070E0CB014E
:109770006D837E838F839887412FBE016F5F7F4FFC
:1097800085E197E00E9447480E94242A28960FB658
:10979000F894DEBF0FBECDBFDF91CF911F9108952A
:1097A0005E985E9815985E9808955E9A10921207DA
:1097B0005E9A10921307159A109214075E9A0895F4
:1097C0000E9475B3F8940E94F0A60E94D54BE3E482
:1097D000F0E18491882341F09091C00095FFFCCF87
:1097E0008093C6003196F5CFE8E0F6E084918823B7
:1097F00041F09091C00095FFFCCF8093C600319658
:10980000F5CF8091C00085FFFCCF8AE08093C60031
:109810007894C6E0D0E0219749F068EC70E080E0F1
:1098200090E00E94FAE70E943EB9F5CFF894A8951F
:10983000FECF8F929F92AF92BF92CF92DF92EF9224
:10984000FF920F931F93CF93DF933AE0F32E809113
:10985000FD069091FE0604970CF034C12FB7F894E2
:109860008091E3049091E4042FBF891B8F7709F462
:1098700029C182E694E00E942C2820916305309152
:1098800064058A3019F08D3009F0E9C0109247055F
:1098900021153105E1F2F901E951FB4F10821092D7
:1098A00064051092630587EE94E06C01FC01208151
:1098B00001962032D1F3E6012E3411F0C12CD12CC7
:1098C0006AE270E0CE010E94ECF28C01C114D10476
:1098D00009F474C062E07FE0CE010E949EF2EE24A3
:1098E000E394892B11F4E12C09C06EE470E0CE0101
:1098F00004960E94ECF2009709F06C014AE050E0F7
:1099000060E070E0C60101960E9433F160930B079E
:1099100070930C0780930D0790930E0780900707B4
:1099200090900807A0900907B0900A07FFEF8F1AE0
:109930009F0AAF0ABF0A681579058A059B0531F0B1
:10994000E11004C061E08FEC9EE03DC001151105FF
:1099500001F180E0D12CFE01E80FF11D90819A32D7
:1099600019F08F5FD926F7CF4AE050E060E070E051
:10997000C80101960E9433F10D2D10E020E030E087
:10998000601771078207930741F061E080EB9EE06A
:109990001AC061E086E89EE016C080910B079091A6
:1099A0000C07A0910D07B0910E07809307079093C5
:1099B0000807A0930907B0930A0713C0009789F01E
:1099C00060E08CE59EE0DF91CF911F910F91FF90B9
:1099D000EF90DF90CF90BF90AF909F908F900C94BE
:1099E000344680914701811129C067E470E0CE01BF
:1099F0000E94ECF2009711F14AE050E060E070E064
:109A000001960E9433F164307105C0F4E6EEFDE08A
:109A10008491882341F09091C00095FFFCCF809302
:109A2000C6003196F5CF8091C00085FFFCCFF09243
:109A3000C60060E08CED9DE00E945CB364E573E0DD
:109A4000CE010E94F7F2892B21F483ED9DE00E9464
:109A5000E04B61E087EE94E00E94C02AF8CE2F35FB
:109A600031050CF0F4CE8C35C1F42FB7F894809109
:109A7000E3049091E4042FBF891B8F7709F4E7CEAC
:109A800082E694E00E942C28909147059111DFCE48
:109A9000209163053091640509C08B3319F491E07E
:109AA00090934705909147059111D1CEA9014F5F41
:109AB0005F4F5093640540936305F901E951FB4FF3
:109AC0008083C5CEDF91CF911F910F91FF90EF90D2
:109AD000DF90CF90BF90AF909F908F900895CF93DD
:109AE000DF93EC018091670580934E0584E50E9429
:109AF000472D811102C080E03FC00E943A2D809323
:109B00004E058823C1F3EDE3F0E18491882341F011
:109B10009091C00095FFFCCF8093C6003196F5CFA1
:109B20008091C00085FFFCCF8DE48093C6004AE0A1
:109B300050E0BE0182E694E00E940A29E5EFF5E0DC
:109B40008491882341F09091C00095FFFCCF8093D1
:109B5000C6003196F5CF60914E0570E04AE050E0C6
:109B600082E694E00E940A298091C00085FFFCCF24
:109B70008AE08093C60081E0DF91CF91089589E665
:109B800090E00E946F4D811116C0E8ECF8E08491DE
:109B9000882341F09091C00095FFFCCF8093C600D0
:109BA0003196F5CF0E944E348091C00085FFFCCFE6
:109BB0008AE08093C6000895CF92DF92EF92FF92E1
:109BC0006B017C0180917605882331F120E030E043
:109BD000A901C701B6010E9427EB8823E9F020E024
:109BE00030E040E05FE3C701B6010E94FCED6B018D
:109BF0007C012BED3FE049E450E40E94FCEDA7011D
:109C000096010E94FCED9B01AC0160E070E080E8F1
:109C10009FE30E942EEB04C060E070E080E89FE3C9
:109C2000FF90EF90DF90CF90089560913B0170918D
:109C30003C0180913D0190913E010E94DC4D60937A
:109C40003701709338018093390190933A01089558
:109C5000CF92DF92EF92FF92CF9388EC90E00E9438
:109C60006F4D811145C084E40E94472D882309F47B
:109C70003FC00E94092D6B017C01C1E020E030E073
:109C8000A9010E9427EB811101C0C0E0C0937605B5
:109C9000CC2339F1E0914E0584E0E89FF0011124D6
:109CA000E55CFE4FC082D182E282F38220E030E0A8
:109CB000A90160913B0170913C0180913D0190911F
:109CC0003E010E9427EB81110CC080E090E0A0E4EF
:109CD000B0E480933B0190933C01A0933D01B0938D
:109CE0003E01CF91FF90EF90DF90CF900C94154EF6
:109CF000CF91FF90EF90DF90CF900895CF92DF92B9
:109D0000EF92FF926B017C016091D7127091D81293
:109D1000882777FD8095982F0E94C9EB20E030E0DE
:109D2000A9010E942AED1816E4F0C114D104E1043F
:109D3000F10419F40E94CBE702C0B601C701609399
:109D400053057093540580935505909356051092D2
:109D50004F0510925005109251051092520581E066
:109D600001C080E0FF90EF90DF90CF9008951F93A7
:109D7000CF93DF9380913C0781110E948D9FC0910A
:109D80000307D091040761E270E0CE010E94ECF27B
:109D9000009711F0EC01219680E50E94472D882361
:109DA00041F011E080916105909162058C179D074B
:109DB00008F010E080913D078823A9F1212F41E0B0
:109DC000BE018AE397E00E944B1883E50E94472D6D
:109DD000882339F080916105909162058C179D0769
:109DE00070F08AE397E00E94C01411111CC060E07B
:109DF00070E0CB01DF91CF911F910C947E4E0E94B9
:109E00003A2DAC01662757FD6095762F4093B8092F
:109E10005093B9096093BA097093BB0987E099E040
:109E20000E94338DDECFDF91CF911F910895409135
:109E30005305509154056091550570915605452B79
:109E4000462B472BF9F0811111C06091D712709108
:109E5000D812882777FD8095982F0E94C9EB20E0C3
:109E600030E0A9010E942AED181664F00E94CBE7A9
:109E700060934F0570935005809351059093520560
:109E800081E0089580E00895CF92DF92EF92FF92F3
:109E90000F931F93CF93DF9388E690E00E946F4D5E
:109EA000811146C08091390783FD42C060E070E0B7
:109EB000CB010E947E4E83E50E94472D882331F11D
:109EC0000E94092D6B017C0100914E0510E0E80114
:109ED000CC0FDD1FC952DD4E0E9496EB798368835B
:109EE000F801EE0FFF1FEE0FFF1FE354FD4E208120
:109EF000318142815381C701B6010E942AED1816B3
:109F00002CF460E087E199E00E945CB380E00E945D
:109F1000174F882369F060E087E099E0DF91CF91E7
:109F20001F910F91FF90EF90DF90CF900C945CB356
:109F3000DF91CF911F910F91FF90EF90DF90CF9025
:109F400008950F931F93009153051091540520918C
:109F5000550530915605011511052105310529F1E9
:109F600080914F0590915005A0915105B0915205F7
:109F7000081719072A073B0718F00E94CBE702C011
:109F8000BC01CD0100915305109154052091550558
:109F900030915605601B710B820B930B28EE33E05A
:109FA00040E050E00E94FAEE03C020E030E0A9015A
:109FB000CA01B9011F910F9108952F923F924F92BC
:109FC0005F926F927F928F929F92AF92BF92CF9249
:109FD000DF92EF92FF920F931F93CF93DF93CDB752
:109FE000DEB7A0970FB6F894DEBF0FBECDBF80914D
:109FF0003C07882309F42AC18091FD069091FE0652
:10A00000892B11F41092E60421E028A34091B809AD
:10A010005091B9096091BA097091BB098091B40956
:10A020009091B509A091B609B091B70948175907A1
:10A030006A077B0708F418A200E010E06CE3C62E64
:10A04000D12CE12CF12C70E1272E7EE0372E412C13
:10A05000512CCE0101963C018091FD069091FE06A7
:10A0600004970CF0F3C028A12111F0C08091E60400
:10A070008111ECC080910F0990911009A0911109F4
:10A08000B09112098093B8099093B909A093BA09C5
:10A09000B093BB0987E099E00E94638C8F8FA1E0A9
:10A0A000A8A38090B8099090B909A090BA09B0907F
:10A0B000BB094091B4095091B5096091B6097091FE
:10A0C000B70984169506A606B70630F418A28F3F86
:10A0D000BFEF9B0721F479C0E0ECFDE018C02F8DA5
:10A0E0002A3009F478C02D3009F475C0233219F0F4
:10A0F0002A3309F08BC02091E504211187C065C087
:10A100009091C00095FFFCCF8093C600319684915A
:10A110008111F6CF8091C00085FFFCCF4AE04093CB
:10A12000C60081E00E94174F0E94A14F4B015C01C5
:10A13000A70196010E94FAEECA01B901A701960192
:10A140000E94FAEE7F936F93C501B401A2019101C1
:10A150000E94FAEE3F932F93ACEABDE0BF93AF931A
:10A160007F926F920E9424F30FB6F894DEBF0FBE69
:10A17000CDBFEDE3F0E18491882341F09091C000E0
:10A1800095FFFCCF8093C6003196F5CFF301819106
:10A19000882339F09091C00095FFFCCF8093C600D2
:10A1A000F6CF8091C00085FFFCCF9AE09093C60067
:10A1B00061E0C3010E9410B38AE397E00E94891C0A
:10A1C00061E08AE397E00E940C17AF8DA33219F487
:10A1D000B1E0B093E6041092E5040115110509F40D
:10A1E0003BCF8091FF069091000720E6289FF00169
:10A1F000299FF00D1124E00FF11FE358FA4F108250
:10A2000080E00E94A42A00E010E026CF0F3511055F
:10A2100008F022CF4F8D4B3319F4A1E0A093E50451
:10A220002091E504211118CF2091FF0630910007FD
:10A23000B0E6B29FF001B39FF00D1124E00FF11FC3
:10A24000E358FA4F80830F5F1F4F06CFA0960FB6DB
:10A25000F894DEBF0FBECDBFDF91CF911F910F915C
:10A26000FF90EF90DF90CF90BF90AF909F908F9036
:10A270007F906F905F904F903F902F9008950E9435
:10A280002E2B811104C00E94194C0C94DD4F0895AF
:10A29000CF92DF92EF92FF920F931F93CF93C82F2D
:10A2A0008091FD069091FE06049714F40E943F51A0
:10A2B0000E94CBE7C0905705D0905805E090590513
:10A2C000F0905A05C114D104E104F104A9F0009101
:10A2D0005B0510915C0520915D0530915E050C0DCC
:10A2E0001D1D2E1D3F1D061717072807390720F4CF
:10A2F00087E296E00E94E04BC0901B01D0901C01C9
:10A30000E0901D01F0901E01C114D104E104F1049C
:10A31000C9F000915B0510915C0520915D053091BD
:10A320005E050C0D1D1D2E1D3F1D06171707280766
:10A33000390740F4C11106C09091F5098091F409E4
:10A34000981749F0CF911F910F91FF90EF90DF90F8
:10A35000CF900C94ED685E9A109212075E9A10925C
:10A360001307159A109214075E9AECCF0E9496A5D7
:10A3700080E00E9448510E94CB320C943EB98F92EB
:10A380009F92AF92BF92CF92DF92EF92FF9280E5C1
:10A390000E94472D882329F00E942F2D4B015C013C
:10A3A00003C0812C912C540183E50E94472D882302
:10A3B00061F00E94092D20E030E04AE754E40E9459
:10A3C000FCED0E949BEB4B015C010E948D9F0E9463
:10A3D000242AC0905B05D0905C05E0905D05F0906C
:10A3E0005E05C80CD91CEA1CFB1C0E9409B3811134
:10A3F00005C060E088E19DE00E945CB30E94CBE76D
:10A400006C157D058E059F0518F40E94B651F6CF98
:10A41000FF90EF90DF90CF90BF90AF909F908F9084
:10A4200008952F923F924F925F926F927F928F92F8
:10A430009F92AF92BF92CF92DF92EF92FF920F93D3
:10A440001F93CF93DF93CDB7DEB7C259D1090FB6B3
:10A45000F894DEBF0FBECDBF2DB73EB7E7963FAF36
:10A460002EAFE79780910F07882321F08091100786
:10A47000811104C00E94F7290C94E85A86E50E94D5
:10A48000472D882339F00E943A2D6F969FAF8EAFEB
:10A490006F9706C041E050E06F965FAF4EAF6F9789
:10A4A0006F968EAD9FAD6F970597B0F0EAE8FCE030
:10A4B0008491882341F09091C00095FFFCCF809358
:10A4C000C6003196F5CF8091C00085FFFCCF8AE0B1
:10A4D0008093C6000C94E85A84E40E94472DAA9603
:10A4E0008FAFAA9785E40E94472DCC57DF4F888312
:10A4F000C458D0406F96AEADBFAD6F9713977CF444
:10A5000084E50E94472DCF57DF4F8883C158D04044
:10A510006F96EEADFFAD6F97EF2B69F106C0F1E0DE
:10A52000CF57DF4FF883C158D040E3E7FCE0849178
:10A53000882341F09091C00095FFFCCF8093C60026
:10A540003196F5CFAA962FADAA972223A1F0EBE57D
:10A55000FCE08491882341F09091C00095FFFCCFEE
:10A560008093C6003196F5CF8091C00085FFFCCF67
:10A570008AE08093C60080E50E94472D8823A9F0D9
:10A580000E943A2D1C018230910594F4E3E2FCE034
:10A590008491882311F40C94E85A9091C00095FF9F
:10A5A000FCCF8093C6003196F3CF63E0262E312C8A
:10A5B00083E50E94472D882319F00E943A2D02C09E
:10A5C00088E893E190931A01809319018CE40E942A
:10A5D000472D882339F00E943A2D6B969FAF8EAF9E
:10A5E0006B9706C04EE150E06B965FAF4EAF6B9736
:10A5F00082E50E94472D882321F00E943A2D7C019C
:10A6000003C050EAE52EF12C86E40E94472D8823F2
:10A6100021F00E943A2D8C0102C00EE110E082E48C
:10A620000E94472D882321F00E943A2D6C0103C01F
:10A6300040EAC42ED12C6B968EAD9FAD6B9731E066
:10A64000833D9F4F54F0C70109976B96EEADFFAD68
:10A650006B97E817F9070CF430E021E0FAEBEF16FE
:10A66000F1044CF46B968EAD9FAD6B9709968E15E9
:10A670009F050CF420E0AA24A3940B3F4FEF14078E
:10A6800034F0C6010997081719070CF4A12CBB2454
:10A69000B39453EAC516D10434F4C80109968C1555
:10A6A0009D050CF4B12C31110CC0222329F084E15A
:10A6B0009CE00E94613315C0A11013C0B11017C0F7
:10A6C0001EC08CE19CE0CE56DF4F2883C259D0409B
:10A6D0000E946133CE56DF4F2881C259D0402111EC
:10A6E000E6CFAA2021F08CE09CE00E946133BB20E1
:10A6F00009F46EC785E09CE00E94613369C70E943F
:10A700008D9FAA968FADAA9781112EC084E591E006
:10A710000E9438E1CE0101960E940E7489819A81CF
:10A72000AB81BC818093250790932607A0932707D0
:10A73000B09328078D819E81AF81B88580932907CA
:10A7400090932A07A0932B07B0932C0789859A85AD
:10A75000AB85BC8580932D0790932E07A0932F0780
:10A76000B09330070E94482F0E942F2A80E090E08B
:10A77000A6E1B4E48093430190934401A093450182
:10A78000B0934601D10111976596BFAFAEAF659703
:10A79000C7016B96EEADFFAD6B978E1B9F0BBD0196
:10A7A0000E94E6EECE57DF4F79836883C258D040CF
:10A7B000229C9001239C300D300D1124A3963FAFB5
:10A7C0002EAFA397220F331FE3963FAF2EAFE39731
:10A7D000C901A3964EAD5FADA397840F951F880F57
:10A7E000991F880F991FADB7BEB7A81BB90B0FB63D
:10A7F000F894BEBF0FBEADBFEDB7FEB73196A796BA
:10A80000FFAFEEAFA797440F551F440F551FE996B2
:10A810005FAF4EAFE9972DB73EB7241B350B0FB690
:10A82000F8943EBF0FBE2DBF4DB75EB74F5F5F4F71
:10A83000AC965FAF4EAFAC978DB79EB7A396AEAD5B
:10A84000BFADA3978A1B9B0B0FB6F8949EBF0FBE9C
:10A850008DBFEDB7FEB73196E596FFAFEEAFE5974A
:10A86000F22DF170E196FFAFE197C601801B910BCD
:10A8700065966EAD7FAD65970E94E6EEC757DF4FD8
:10A8800079836883C958D040E0961FAF0EAFE09738
:10A890002CEFE3964EAD5FADE3972403C001259FF7
:10A8A000900D1124CB57DF4F99838883C558D04032
:10A8B0006D961FAE1EAE6D9769961FAE1EAE699760
:10A8C000412C512C3201E096AEADBFADE097BD01F9
:10A8D000882777FD8095982F0E94C9EBED966CAF85
:10A8E0007DAF8EAF9FAFED97E196BFADE197BB23F4
:10A8F00079F0AE963FAE2EAEAE97E1E0F0E0A996CD
:10A90000FFAFEEAFA997A5961FAE1EAEA59714C0D8
:10A9100065962EAD3FAD6597A5963FAF2EAFA59737
:10A920004FEF5FEFA9965FAF4EAFA9978FEF9FEF05
:10A93000AE969FAF8EAFAE97E1969FADE197A1E047
:10A940009A27E1969FAFE1976996EEADFFAD6997C3
:10A95000E3962EAD3FADE397E20FF31FEE0FFF1F1F
:10A96000EE0FFF1FA7964EAD5FADA7974E0F5F1F6F
:10A9700067965FAF4EAF6797A996AEADBFADA9978B
:10A98000CE57DF4FE881F981C258D040AE9FC00159
:10A99000AF9F900DBE9F900D1124C957DF4F998333
:10A9A0008883C758D040A5964EAD5FADA5974E9F02
:10A9B00090014F9F300D5E9F300D11246B968EAD30
:10A9C0009FAD6B97820F931FA1969FAF8EAFA197FC
:10A9D0004A01AE96EEADFFADAE97EA1BFB0BC55735
:10A9E000DF4FF983E883CB58D040E5962EAD3FADDD
:10A9F000E5976D964EAD5FAD6D97240F351FC3572C
:10AA0000DF4F39832883CD58D040AE962EAD3FAD71
:10AA1000AE978216930609F402C1A196AEADBFAD02
:10AA2000A197BD01882777FD8095982F0E94C9EBDB
:10AA3000C358DF4F688379838A839B83CD57D04087
:10AA40006996EEADFFAD6997EF2B79F020E030E02D
:10AA500040EA50E460912D0770912E0780912F07F6
:10AA6000909130070E944EEA04C060E070E080E7F9
:10AA700091E4CC57DF4FF881C458D040F11127C082
:10AA80006D962EAD3FAD6D97232B61F421E0D12C57
:10AA9000A5964EAD5FADA5978416950609F020E00A
:10AAA000C22E1DC06D96AEADBFAD6D976596EEAD75
:10AAB000FFAD6597AE17BF0769F4C557DF4F288113
:10AAC0003981CB58D0408216930621F405C013E09B
:10AAD000C12E04C0C12C02C0B2E0CB2ED12C6F9687
:10AAE000AEACBFAC6F977B018C01ED962CAD3DAD4C
:10AAF0004EAD5FADED97C358DF4F688179818A8194
:10AB00009B81CD57D0400E9481316B017C019B011C
:10AB1000AC01C301B2010E944EEA2B013C016996CF
:10AB2000EEADFFAD6997EE0FFF1FEE0FFF1FAC9666
:10AB30004EAD5FADAC97E40FF51FC082D182E282CB
:10AB4000F3826796EEADFFAD6797CB57DF4F8881F5
:10AB50009981C558D040E80FF91FC358DF4F2881AD
:10AB600039814A815B81CD57D04020833183428334
:10AB70005383E9964EAD5FADE997E40FF51FED966F
:10AB80008CAD9DADAEADBFADED9780839183A283BB
:10AB9000B3836796AEADBFAD679720E030E040E885
:10ABA0005FE32D933D934D935D936796BFAFAEAF3B
:10ABB0006797829CF001839CF00D929CF00D11240C
:10ABC000C357DF4F28813981CD58D040E20FF31FA2
:10ABD00068963FAD6897308369964EAD5FAD6997D3
:10ABE0004F5F5F4F69965FAF4EAF69970E94B65156
:10ABF000A9968EAD9FADA997880E991EA196AEAD70
:10AC0000BFADA197C957DF4FE881F981C758D04040
:10AC1000AE0FBF1FA196BFAFAEAFA197F6CE6D9698
:10AC20004EAD5FAD6D974F5F5F4F6D965FAF4EAFAF
:10AC30006D97E0968EAD9FADE097C757DF4FA88127
:10AC4000B981C958D0408A0F9B1FE0969FAF8EAF45
:10AC5000E097421553050CF436CE0E94522AAC966A
:10AC60000EAD1FADAC97A7962EAD3FADA79743E0B5
:10AC700050E0A3966EAD7FADA397CE0149960E949A
:10AC8000BD86A396EEADFFADA397BF01882777FDE4
:10AC90008095982F0E94C9EB9B01AC01C301B201C2
:10ACA0000E942EEB2B013C016F962EAD3FAD6F97AE
:10ACB000232B09F46FC0EFEEFBE08491882341F071
:10ACC0009091C00095FFFCCF8093C6003196F5CFE0
:10ACD000498D5A8D6B8D7C8D28E030E082E694E0C2
:10ACE0000E94E729EAEEFBE08491882341F09091ED
:10ACF000C00095FFFCCF8093C6003196F5CF4D8DF7
:10AD00005E8D6F8D78A128E030E082E694E00E94AD
:10AD1000E729E5EEFBE08491882341F09091C000A3
:10AD200095FFFCCF8093C6003196F5CF49A15AA17B
:10AD30006BA17CA128E030E082E694E00E94E72944
:10AD40008091C00085FFFCCF8AE08093C6006F969B
:10AD50004EAD5FAD6F9743305105E4F0ECECFBE096
:10AD60008491882341F09091C00095FFFCCF80939F
:10AD7000C6003196F5CF28E030E0B301A20182E6AB
:10AD800094E00E94E7298091C00085FFFCCF8AE013
:10AD90008093C600AA965FADAA9751115DC00D8D34
:10ADA0001E8D2F8D38A13058498D5A8D6B8D7C8D1D
:10ADB0007058C12CD12CE0E8EE2EEFE3FE2ECE0130
:10ADC0000D960E94EEDE69E573E0CE010D960E94BD
:10ADD0006CE0CD84DE84EF84F88809891A892B8998
:10ADE0003C894D895E896F89788DCE0189960E9454
:10ADF00062E184E2FE01B996A4E5B1E001900D9212
:10AE00008A95E1F7CE0101960E940E7489819A819C
:10AE1000AB81BC818093250790932607A0932707D9
:10AE2000B09328078D819E81AF81B88580932907D3
:10AE300090932A07A0932B07B0932C0789859A85B6
:10AE4000AB85BC8580932D0790932E07A0932F0789
:10AE5000B09330070E94482FCF57DF4F8881C158E9
:10AE6000D040882309F4E3C2E1EBFBE0849188231E
:10AE700041F09091C00095FFFCCF8093C6003196C1
:10AE8000F5CFEFE9FBE08491882341F09091C00079
:10AE900095FFFCCF8093C6003196F5CFEDE8FBE03F
:10AEA0008491882341F09091C00095FFFCCF80935E
:10AEB000C6003196F5CFE9E7FBE08491882341F0A5
:10AEC0009091C00095FFFCCF8093C6003196F5CFDE
:10AED000E5E6FBE08491882341F09091C00095FF66
:10AEE000FCCF8093C6003196F5CFE1E5FBE084917D
:10AEF000882341F09091C00095FFFCCF8093C6005D
:10AF00003196F5CFEDE3FBE08491882341F09091F9
:10AF1000C00095FFFCCF8093C6003196F5CFE9E2E3
:10AF2000FBE08491882341F09091C00095FFFCCF15
:10AF30008093C6003196F5CFE7E1FBE0849188234A
:10AF400041F09091C00095FFFCCF8093C6003196F0
:10AF5000F5CFE5E0FBE08491882341F09091C000BB
:10AF600095FFFCCF8093C6003196F5CFEDEFFAE068
:10AF70008491882341F09091C00095FFFCCF80938D
:10AF8000C6003196F5CF65960EAD1FAD6597912C35
:10AF900090EC892E99E766969FAF6697A4E4689631
:10AFA000AFAF6897FE0131962F96FFAFEEAF2F97A8
:10AFB0009E01235F3F4F61963FAF2EAF6197AE0179
:10AFC0004B5D5F4F63965FAF4EAF63976A969FAEE0
:10AFD0006A976C968FAE6C9766968FAD6697A096C3
:10AFE0008FAFA09768969FAD6897A4969FAFA497E0
:10AFF000A12CB12CE596AEADBFADE597A00FB11F6A
:10B00000A996BFAFAEAFA997A29CF001A39CF00D8B
:10B01000B29CF00D1124A996AEADBFADA997EA0F71
:10B02000FB1F8080992487FC9094F401EE0FFF1F92
:10B03000EE0FFF1F6996FFAFEEAF6997AC962EAD8E
:10B040003FADAC972E0F3F1F67963FAF2EAF679770
:10B05000A30192016796AEADBFAD67976D917D91EB
:10B060008D919C910E944DEA6B017C01A796EEADFB
:10B07000FFADA79769962EAD3FAD6997E20FF31F1D
:10B0800080819181A281B3818DA39EA3AFA3B8A734
:10B09000A396EEADFFADA397E80DF91DEE0FFF1FD0
:10B0A000EE0FFF1FA7964EAD5FADA797E40FF51FFC
:10B0B00080819181A281B3818D879E87AF87B88B74
:10B0C00019821A821B821C822F965FAD2F975F9385
:10B0D0002E968FAD2E978F9361969FAD61979F931C
:10B0E0006096AFAD6097AF936396BFAD6397BF9324
:10B0F0006296EFAD6297EF932DB73EB724523109B8
:10B100000FB6F8943EBF0FBE2DBFADB7BEB71196B8
:10B11000E4E5F1E084E201900D928A95E1F70E9466
:10B12000CAE029813A814B815C816796AEADBFADA3
:10B1300067976D917D918D919C910E944DEA962E1D
:10B14000872E66968FAF669768969FAF6897EDB724
:10B15000FEB7BA960FB6F894FEBF0FBEEDBF262F0E
:10B16000372FAC016A966FAD6A976C967FAD6C977E
:10B17000A0968FADA097A4969FADA4970E942AEDAC
:10B18000181694F06A969FAC6A976C968FAC6C9781
:10B19000A096FFADA0976696FFAF6697A4962FADD9
:10B1A000A49768962FAF689720E030E0A901C70107
:10B1B000B6010E942AED87FD0DC0EAEFFAE0849106
:10B1C000882379F09091C00095FFFCCF8093C60052
:10B1D0003196F5CF8091C00085FFFCCF30E23093EF
:10B1E000C60025E030E0B701A60182E694E00E94A7
:10B1F000E7294FEFA41AB40AA214B3049CF46A9688
:10B200009FAE6A976C968FAE6C9766965FAD6697A9
:10B21000A0965FAFA09768968FAD6897A4968FAF02
:10B22000A497F2CE8091C00085FFFCCF5AE05093E6
:10B23000C6000150110917FFC9CE8091C00085FFDB
:10B24000FCCF8AE08093C6006F96EEADFFAD6F979E
:10B25000349709F0ECC0EFECFAE08491882341F0D8
:10B260009091C00095FFFCCF8093C6003196F5CF3A
:10B270009E012F5F3F4F2F963FAF2EAF2F975E015E
:10B280003DE0A30EB11C2E0145E2440E511C00E02E
:10B2900010E0E5966EAC7FACE5976596AEADBFADC0
:10B2A00065976A0E7B1E029DF001039DF00D129DB5
:10B2B000F00D1124E60DF71D8081992787FD9095EB
:10B2C0007C01EE0CFF1CEE0CFF1CA796EEADFFAD53
:10B2D000A797EE0DFF1D40815181628173814DA3BF
:10B2E0005EA36FA378A7A396EEADFFADA397E80F7B
:10B2F000F91FEE0FFF1FEE0FFF1FA7968EAD9FAD3C
:10B30000A797E80FF91F80819181A281B3818D8772
:10B310009E87AF87B88B19821A821B821C822F9658
:10B320009FAD2F979F932E96AFAD2E97AF93BF9261
:10B33000AF925F924F92EDB7FEB7B4970FB6F89405
:10B34000FEBF0FBEEDBFADB7BEB71196E4E5F1E0AD
:10B3500084E201900D928A95E1F70E94CAE0AC96D2
:10B36000EEADFFADAC97EE0DFF1D29813A814B810B
:10B370005C8160817181828193810E944DEA292DD7
:10B38000382D66964FAD669768965FAD68970E94B8
:10B390004DEA6B017C012DB73EB7265D3F4F0FB6DE
:10B3A000F8943EBF0FBE2DBF20E030E0A9010E94FF
:10B3B0002AED87FD0DC0ECECFAE08491882379F04A
:10B3C0009091C00095FFFCCF8093C6003196F5CFD9
:10B3D0008091C00085FFFCCF30E23093C60025E0AD
:10B3E00030E0B701A60182E694E00E94E7290F5FF2
:10B3F0001F4F021513050CF456CF8091C00085FF36
:10B40000FCCF4AE04093C60065968EAD9FAD659730
:10B41000019765969FAF8EAF659797FF38CF809164
:10B42000C00085FFFCCF8AE08093C60006C06F96FF
:10B43000EEADFFAD6F97EF2B31F065E673E084E57D
:10B4400091E00E9427E3AA96FFADAA97F1119EC052
:10B4500020E030E040EA51E4609125077091260732
:10B4600080912707909128070E944DEA6DA37EA343
:10B470008FA398A720E030E04CE252E460912907C6
:10B4800070912A0780912B0790912C070E944DEA1A
:10B490006D877E878F87988B80912D0790912E07DF
:10B4A000A0912F07B091300789839A83AB83BC8327
:10B4B00082E090E00E94F29F9B01AC01CE010196D8
:10B4C0009F938F930C969F938F9348969F938F9300
:10B4D0008DB79EB784970FB6F8949EBF0FBE8DBFF1
:10B4E000ADB7BEB7119684E2E4E5F1E001900D92AC
:10B4F0008A95E1F7CE56DF4F2883C259D040C15715
:10B50000DF4F3883CF58D040C057DF4F4883C059F2
:10B51000D040CF56DF4F5883C159D0400E94CAE077
:10B52000CE56DF4F2881C259D040C157DF4F3881F6
:10B53000CF58D040C057DF4F4881C059D040CF5678
:10B54000DF4F5881C159D04069817A818B819C81BC
:10B550000E944DEA2091150130911601409117018A
:10B56000509118010E944DEA60932D0770932E07A9
:10B5700080932F0790933007ADB7BEB79A960FB65A
:10B58000F894BEBF0FBEADBF0E94482F20E030E050
:10B5900040E751E460912D0770912E0780912F07AD
:10B5A000909130070E944EEA0E94643181E090E061
:10B5B00090934905809348050E944A37E796EEAD7F
:10B5C000FFADE7970FB6F894FEBF0FBEEDBF09C001
:10B5D000E7962EAD3FADE7970FB6F8943EBF0FBE8E
:10B5E0002DBFE7964EAD5FADE7970FB6F8945EBFFF
:10B5F0000FBE4DBFCE56DF4F0FB6F894DEBF0FBE65
:10B60000CDBFDF91CF911F910F91FF90EF90DF9011
:10B61000CF90BF90AF909F908F907F906F905F90F2
:10B620004F903F902F9008958F929F92AF92BF922C
:10B63000CF92DF92EF92FF921F93CF93DF93C0914F
:10B640000307D091040780E50E94472D882379F0F5
:10B650000E943A2D6C01EE24D7FCE094FE2C11E000
:10B66000C114D104E104F10431F410E004C010E08D
:10B67000C12CD12C760183E50E94472D8823D9F077
:10B680000E94092D20E030E04AE754E40E94FCEDDE
:10B690000E949BEB6B017C0111110FC061157105BC
:10B6A0008105910551F48881882339F061E0CE014C
:10B6B0000E9410B307C01123B1F360E087E99AE05C
:10B6C0000E945CB381E00E94DFB20E948D9F0E94C5
:10B6D000242AC114D104E104F104F1F080905B0547
:10B6E00090905C05A0905D05B0905E058C0C9D1C53
:10B6F000AE1CBF1C83E090E0909349058093480501
:10B700000E94CBE7681579058A059B0598F50E948C
:10B710007FB381112FC038C00E947DB38823B9F157
:10B7200083E090E090934905809348050E947FB3A1
:10B73000811103C00E94B651F9CF81E090E090934F
:10B7400049058093480580913C0760E0882319F003
:10B7500088E89AE002C088E79AE0DF91CF911F91D4
:10B76000FF90EF90DF90CF90BF90AF909F908F9021
:10B770000C945CB381E090E0909349058093480578
:10B7800080E00E94DFB2DFCF0E94B651B9CFDF91D7
:10B79000CF911F91FF90EF90DF90CF90BF90AF902F
:10B7A0009F908F9008954F925F926F927F928F92A9
:10B7B0009F92AF92BF92CF92DF92EF92FF921F9330
:10B7C000CF93DF938DE690E00E946F4D81117BC196
:10B7D0008091390783FD77C160E070E0CB010E9462
:10B7E0007E4E83E50E94472D182F811105C082E50A
:10B7F0000E94472D882331F10E94092D6B017C01A5
:10B80000A0904E05B12CE501CC0FDD1FC952DD4ED5
:10B810000E9496EB79836883F501EE0FFF1FEE0F10
:10B82000FF1FE354FD4E2081318142815381C701C6
:10B83000B6010E942AED18162CF460E08DEB98E01A
:10B840000E945CB380E00E94174F882329F060E0DB
:10B850008DEA98E00E945CB386E40E94472D8093B5
:10B86000C60E882351F00E94092D60934801709301
:10B87000490180934A0190934B0183E50E94472D33
:10B88000882351F00E94092D60934C0170934D0163
:10B8900080934E0190934F0182E40E94472D8823AC
:10B8A00051F00E94092D60935001709351018093D3
:10B8B000520190935301D0904E051123F9F0ED2CD5
:10B8C000F12CE701CC0FDD1FC952DD4E6881798173
:10B8D000882777FD8095982F0E94C9EBD701AA0F82
:10B8E000BB1FAA0FBB1FA354BD4E2D913D914D917F
:10B8F0005C910E942AED18160CF0E5C0ED2DF0E0E9
:10B90000EE0FFF1FE952FD4E60817181882777FDA0
:10B910008095982F0E94C9EB20E030E046E952E480
:10B920000E9427EB87FDCFC0109266050E94CBE7EF
:10B930006B017C012B013C0188EE480E83E0581E10
:10B94000611C711C88248A94982C54011AE08091FF
:10B9500066058111A4C0B7FE96C00E94CBE76B01BB
:10B960007C01461657066806790608F049C02B0187
:10B970003C0188EE480E83E0581E611C711C0E9439
:10B980004E34E9EAF8E08491882341F09091C000B8
:10B9900095FFFCCF8093C6003196F5CFB7FE03C06C
:10B9A000E7EAF8E024C0C501B401605F784D8F4F2D
:10B9B0009F4F6C197D098E099F0928EE33E040E006
:10B9C00050E00E94FAEEBA01A9012AE030E082E6D6
:10B9D00094E00E94E3288091C00085FFFCCF0EC058
:10B9E0009091C00095FFFCCF8093C6003196849162
:10B9F0008111F6CF8091C00085FFFCCF1093C60067
:10BA00000E94B6510E94242AE0914E05F0E0EF0119
:10BA1000CC0FDD1FCC0FDD1FC354DD4EEE0FFF1F1B
:10BA2000E952FD4E60817181882777FD8095982FBE
:10BA30000E94C9EB9B01AC01688179818A819B815D
:10BA40000E944DEA0E9496EB97FF07C09095809563
:10BA5000709561957F4F8F4F9F4FB7FE05C021E0D6
:10BA600030E040E050E004C023E030E040E050E04F
:10BA700026173707480759070CF069CF0E94CBE714
:10BA80004B015C0164CFD501C401805F984DAF4F7D
:10BA9000BF4FC816D906EA06FB0608F45ECF60E081
:10BAA00089E998E0DF91CF911F91FF90EF90DF90AF
:10BAB000CF90BF90AF909F908F907F906F905F904E
:10BAC0004F900C945CB3DF91CF911F91FF90EF905A
:10BAD000DF90CF90BF90AF909F908F907F906F90AE
:10BAE0005F904F900895CF92DF92EF92FF92CF93A5
:10BAF0008091390783FD7CC060E08CE898E00E946B
:10BB00005CB383E50E94472DC82F81112DC082E5CB
:10BB10000E94472D811128C0109266050E94CBE734
:10BB20006B017C0128EEC20E23E0D21EE11CF11C49
:10BB3000CAE080916605811135C06091D51270917F
:10BB4000D612882777FD8095982F0E94C9EB209107
:10BB5000B7123091B8124091B9125091BA120E94A6
:10BB60002AED18164CF11EC00E94092D0E9496EB7A
:10BB70007093D6126093D512CC2371F2882777FD8B
:10BB80008095982F0E94C9EB2091B7123091B8127E
:10BB90004091B9125091BA120E942AED18160CF475
:10BBA000BBCF26C060E082E898E0CF91FF90EF9095
:10BBB000DF90CF900C945CB30E94CBE7C616D706FB
:10BBC000E806F90680F46B017C0128EEC20E23E042
:10BBD000D21EE11CF11C0E944E348091C00085FFF2
:10BBE000FCCFC093C6000E94B6510E94242AA1CF68
:10BBF000CF91FF90EF90DF90CF900895CF92DF929A
:10BC0000EF92FF92CF93DF9380E50E94472D882328
:10BC100009F44FC00E94092D6B017C0183E50E944D
:10BC2000472D882331F00E94092D0E9496EBEB01ED
:10BC300002C0CFEFDFEFCE0101960397D0F5C70129
:10BC4000B6010E9496EBF62E262F372FE5E8F3E09B
:10BC5000419151914217530761F183E0EB3BF807A3
:10BC6000B9F737FD26C00E948D9FEF2C60E08F2D25
:10BC70000E9415E9CF3F8FEFD80729F0219771F087
:10BC8000C0E0D0E00DC08F2D0E9484E931E020E0BB
:10BC9000892B09F030E0C32FD22F02C0C1E0D0E0E1
:10BCA0008E2D0E9484E98C179D0719F00E94B651D1
:10BCB000F7CFDF91CF91FF90EF90DF90CF90089575
:10BCC0000F931F93CF93DF93CDB7DEB76E970FB669
:10BCD000F894DEBF0FBECDBF0E94A14F2CE330E031
:10BCE00040E050E00E94FAEE7F936F933F932F93D2
:10BCF00082E49AE09F938F938E010F5F1F4F1F93F3
:10BD00000F930E9424F30FB6F894DEBF0FBECDBF91
:10BD1000EDE3F0E18491882341F09091C00095FF1C
:10BD2000FCCF8093C6003196F5CFF801819188232E
:10BD300039F09091C00095FFFCCF8093C600F6CFFC
:10BD40008091C00085FFFCCF8AE08093C60060E050
:10BD5000C8010E9410B38091C60E882309F1109289
:10BD6000C60E0091670510E0000F111F09521D4E0D
:10BD7000F80160817181882777FD8095982F0E9456
:10BD8000C9EB20914C0130914D0140914E015091F1
:10BD90004F010E942AED18161CF4F801118210823E
:10BDA0006E960FB6F894DEBF0FBECDBFDF91CF9178
:10BDB0001F910F910895CF92DF92EF92FF920F9310
:10BDC0001F93CF93DF93209101073091020740E644
:10BDD000429FC001439F900D112483589A4F909326
:10BDE0000607809305078091390780FF22C0EDE3A5
:10BDF000F0E18491882341F09091C00095FFFCCF41
:10BE00008093C6003196F5CFE0910507F0910607C3
:10BE10008191882339F09091C00095FFFCCF8093E9
:10BE2000C600F6CF8091C00085FFFCCF8AE08093EA
:10BE3000C6008091050790910607FC0120810196BC
:10BE40002032D9F3F0930607E09305072E3461F012
:10BE5000C0910507D09106076AE270E0CE010E940A
:10BE6000ECF20097D1F420C0818190ED980F9A30C8
:10BE700010F08D3269F73296DF0131962C91205304
:10BE80002A30D0F3CD01FC01019620812032D9F374
:10BE9000F0930607E0930507DBCFFC013196829112
:10BEA000803229F08A3219F0FE01619102C01082BD
:10BEB000F6CF2E2F9F2F81918032D9F380538A3075
:10BEC00018F00E949532B3C3E22FF92F20E030E042
:10BED0009AE08191A901949F9001959F300D1124C2
:10BEE00020533109280F311D87FD3A9580818053F9
:10BEF0008A3078F3CF013196DC014C914032D1F396
:10BF0000909304078093030741E050E05093490564
:10BF100040934805643509F469C334F4673451F03B
:10BF20006D3409F450C066C3673621F06D3609F4EC
:10BF30004AC060C32C313105C9F170F42430310599
:10BF400020F42230310500F129C02430310509F0F8
:10BF500066C30E94BF5163C32A35310569F150F4AD
:10BF60002D31310531F12E31310509F058C30E94D0
:10BF7000713955C32B35310511F12C35310509F0D7
:10BF80004EC30E948E334BC380914701882309F42E
:10BF900046C30E942B320E94F24741C381E0223007
:10BFA000310509F080E00E948C4B39C30E9426388D
:10BFB00036C30E94115233C31092650530C381E02D
:10BFC000809365052DC32037310509F49DC108F024
:10BFD00092C02032310509F474C108F049C02731FC
:10BFE000310509F43DC110F52231310509F404C2CF
:10BFF00080F42230310508F426C12131310509F0E1
:10C000000EC360E08FE69AE00E945CB30E94D04BC2
:10C0100006C32531310509F419C108F01CC12431CA
:10C02000310509F0FCC20E94E233F9C22B3131051F
:10C0300009F429C180F42931310509F414C108F04B
:10C0400017C18AE397E00E94C01460E070E0CB0162
:10C050000E947E4EE4C22E31310509F41FC108F062
:10C0600039C12C31310509F0DAC220E040E010C1BD
:10C070002C35310509F4DCC1F8F42235310509F419
:10C08000B4C178F42033310509F427C121353105D5
:10C0900009F495C12A32310509F0C1C20E940F345A
:10C0A000BEC22435310509F4A7C108F4A1C1253564
:10C0B000310509F4A4C1B3C22B36310509F470C1AE
:10C0C00068F42936310509F436C108F043C1283631
:10C0D000310509F0A4C20E94444FA1C22E36310599
:10C0E00009F4FEC008F00DC12D36310509F097C2E4
:10C0F0000E94D35B94C22C3D310509F408C208F0BC
:10C1000047C02139310509F4AEC1F8F427373105AC
:10C1100009F4A6C178F42337310509F491C0253715
:10C12000310509F493C12237310509F078C20E9424
:10C130004A3775C22937310509F48EC108F48AC11E
:10C140002C38310509F4E4C06AC22B3C310509F4EE
:10C15000ACC178F4283C310509F488C1293C31058B
:10C1600009F487C12E3B310509F059C20E94735D65
:10C1700056C22D3C310509F4B2C108F4ADC12E3CC4
:10C18000310509F04CC2CBEBD3E00AE615E0B1C1B2
:10C190002A39B1E03B0709F405C210F52E32F1E06F
:10C1A0003F0709F4E8C170F4223E310509F4DAC111
:10C1B0002D3251E0350709F4D8C12D3D310509F084
:10C1C0002EC2B4C1203381E0380709F4D1C108F48C
:10C1D000E6C12039314009F022C20E948D9F1FC262
:10C1E000263FE1E03E0709F4E6C170F4243F41E058
:10C1F000340709F4DAC108F0DBC12C3A314009F008
:10C200000EC20E94DE430BC22335A3E03A0709F4B5
:10C21000EAC128F4273F314009F4D0C100C2203AD6
:10C22000F3E03F0709F450C0273E334009F0F7C15F
:10C2300081E0809347010E947AB30E940846EFC1D3
:10C24000E8EAF7E0FFC00E94145BE9C18AE397E0E7
:10C250000E949613E4C18AE397E00E946514DFC14F
:10C2600020E041E015C08AE397E00E94C714D7C1DF
:10C2700080913D07882309F4D2C183E50E94472DB0
:10C280008111BAC1CCC18AE397E00E944C16C7C1A4
:10C29000BC018AE397E00E944B18C1C180913D0721
:10C2A000882309F4BCC160E08AE397E00E94DA17B2
:10C2B00060910307709104078AE397E00E942515B7
:10C2C000AEC10E94B74EABC1BC018AE397E00E94A9
:10C2D000551BA5C10E94605EA2C10E94FB399FC18F
:10C2E0008EE40E94472D882309F499C10E942F2DC6
:10C2F00060930B0770930C0780930D0790930E07C4
:10C300008EC10E94FC348BC18BEC98E00E94E04B04
:10C310008091390783FD83C183E50E94472D8823DF
:10C3200009F47DC10E94092D0E9496EB7093D612EC
:10C330006093D51274C10E94BF4D109249051092AE
:10C340004805DF91CF911F910F91FF90EF90DF9003
:10C35000CF90089583E50E94472D882329F00E94FD
:10C360003A2DD82FC92F02C0DFEFC0E080E50E9430
:10C37000472D882319F00E943A2D02C080E090E0FA
:10C380002D2F3C2F2F3F310519F010F02FEF30E00B
:10C39000892B09F044C130936905209368053FC19A
:10C3A00080E50E94472D811105C010926905109209
:10C3B000680535C10E943A2D892BB9F330C10E941E
:10C3C000F0A60E9409A0109269051092680568EE17
:10C3D00073E080E090E00E94FAE760E084E798E094
:10C3E0000E945CB30E943EB91AC110927C0517C12D
:10C3F00081E080937C0514C10E94663610C183E5FC
:10C400000E94472D882309F40AC10E94092D20E0CB
:10C4100030E04AE754E40E94FCED0E949BEB6093FD
:10C420005705709358058093590590935A05F7C0A6
:10C430000E94B036F4C09091C00095FFFCCF80936D
:10C44000C600319684918111F6CFE9C060E00E9468
:10C4500010B3E5C081E001C080E00E948997DFC091
:10C460000E948A40DCC00E94B135D9C00E94284E8B
:10C47000D6C0CBEBD3E007EF1EE089910E94472D99
:10C48000882351F00E94092D0E949BEBD8016D93E7
:10C490007D938D939C9313970C5F1F4FB3E0CF3B1D
:10C4A000DB0759F70E949975BAC0CBEBD3E007E1DF
:10C4B0001FE089910E94472D882339F00E94092DA1
:10C4C000F80160837183828393830C5F1F4FF3E0D5
:10C4D000CF3BDF0771F7A3C00E940D41A0C00E94AF
:10C4E00086419DC00C5F1F4FB3E0CE3BDB0709F4D4
:10C4F00096C089910E94472D8823A1F30E94092D9F
:10C50000D8016D937D938D939C931397EBCF83E527
:10C510000E94472D882309F482C00E94092D0E94A1
:10C5200096EB709342016093410179C083E50E94CC
:10C53000472D882309F473C00E94092D0E9496EBB1
:10C540006B017C018DED90E00E946F4D811167C001
:10C55000E0914E05F0E0EE0FFF1FE15CFE4FD1824F
:10C56000C0825DC00E94FE5D5AC00E94E34157C078
:10C570000E94EE4254C083E50E94472D882319F0A3
:10C580000E94092D03C060E070E0CB0160930A01B6
:10C5900070930B0180930C0190930D0140C00E9499
:10C5A0008C433DC00E940DA03AC00E94841D37C03C
:10C5B0000E94B82534C00E94701F31C083E50E94DC
:10C5C000472D882361F00E94092DC1E020E030E072
:10C5D000A9010E9427EB8111C0E08C2F01C080E0EF
:10C5E0000E9422211CC00E94D94419C0822F0E949F
:10C5F0006E4515C080E014C00E943A2DAC0166273C
:10C6000057FD6095762F4093B8095093B909609310
:10C61000BA097093BB0987E099E00E94338D81E0ED
:10C620001092490510924805882309F44ACCDF91FD
:10C63000CF911F910F91FF90EF90DF90CF900C94CE
:10C64000E845CF93DF938091FD069091FE06049715
:10C6500014F40E943F5160E08AE397E00E940C17B7
:10C660008091FD069091FE06892B09F455C08091BA
:10C670003A078823B1F1809101079091020720E6E3
:10C68000289FE001299FD00D1124C358DA4F69E19A
:10C690007FE0CE010E949EF2892BD1F060E08AE318
:10C6A00097E00E94DA17E7E0FFE08491882341F0E9
:10C6B0009091C00095FFFCCF8093C6003196F5CFD6
:10C6C0008091C00085FFFCCF8AE08093C6000CC03B
:10C6D000BE018AE397E00E949B1680913B07882366
:10C6E00019F00E94DB5E02C00E94E8458091FD06C1
:10C6F0009091FE0601979093FE068093FD0680912F
:10C70000010790910207019664E070E00E94E6EE56
:10C7100090930207809301070E949697DF91CF9133
:10C720000C94B6518F929F92AF92BF92CF92DF92AC
:10C73000EF92FF920F931F93CF93DF938C01875358
:10C740009E4F0E94FB1068018FE6C80ED11CC114D9
:10C75000D10421F178018BE5E81A8EEFF80AE701A0
:10C7600057018FE1A81AB10863ED862E63E0962E7B
:10C77000CC15DD0599F0FE01EE19FF09EA0DFB1D50
:10C7800091828082FE0178978081811102C06F972B
:10C79000EFCFCE014B970E94198EF9CFC801805B75
:10C7A0009F4F0E94FB10C8018F96DF91CF911F9180
:10C7B0000F91FF90EF90DF90CF90BF90AF909F9040
:10C7C0008F900C94FB108AE397E00C9407118AE396
:10C7D00097E00C9492632F923F924F925F926F92E8
:10C7E0007F928F929F92AF92BF92CF92DF92EF9201
:10C7F000FF920F931F93CF93DF93CDB7DEB7689768
:10C800000FB6F894DEBF0FBECDBF1C012A013B015D
:10C8100048015901DC01D8966D917D918D919C91D3
:10C82000DB970E94C7EB6B017C01A30192010E9480
:10C83000FCED0E9414EB0E949BEB69877A878B8743
:10C840009C87A5019401C701B6010E94FCED0E94DE
:10C8500014EB0E949BEB6D877E878F87988B2985D1
:10C860003A854B855C85283731054105510540F4F3
:10C8700088E790E0A0E0B0E089879A87AB87BC8723
:10C880002D853E854F85588928373105410551054D
:10C8900040F488E790E0A0E0B0E08D879E87AF8706
:10C8A000B88B91012C5B3F4FD9018D919D910D90DB
:10C8B000BC91A02D8D839E83AF83B887BC01CD0131
:10C8C0000E94C9EB69837A838B839C8369857A850F
:10C8D0008B859C850E94C7EB698B7A8B8B8B9C8B9D
:10C8E00020E030E0A90169817A818B819C810E94DE
:10C8F00027EB882339F1A7019601C701B6010E94F1
:10C90000FCED4B015C0129893A894B895C89CA019C
:10C91000B9010E94FCED9B01AC01C501B4010E946C
:10C920004DEA4B015C0129813A814B815C81CA014E
:10C93000B9010E944EEA9B01AC01C501B4010E94FD
:10C940002EEB03C060E070E0CB010E9414EB0E946C
:10C9500096EB2B013C016D817E818F8198859095AE
:10C960008095709561957F4F8F4F9F4F0E94C9EBC7
:10C970004B015C016D857E858F8598890E94C7EB90
:10C980006D837E838F83988720E030E0A901C50105
:10C99000B4010E9427EB882349F12D813E814F810C
:10C9A0005885CA01B9010E94FCED6D8B7E8B8F8B7F
:10C9B000988FA7019601C701B6010E94FCED9B016B
:10C9C000AC016D897E898F89988D0E944DEA6B013B
:10C9D0007C01A5019401C501B4010E944EEA9B01AE
:10C9E000AC01C701B6010E942EEB03C060E070E00D
:10C9F000CB010E9404ECF10180889188A288B38861
:10CA000075016401C418D508E608F7080E9496EB82
:10CA1000C61AD70AE80AF90AF7FE6BC020E030E030
:10CA2000A90169817A818B819C810E9427EB8823EF
:10CA300009F447C029813A814B815C81CA01B9015F
:10CA40000E944EEA6B017C01C501B4010E94C7EB54
:10CA50009B01AC01C701B6010E94FCED6B017C019A
:10CA600029893A894B895C89CA01B9010E94FCED88
:10CA70009B01AC01C701B6010E944DEA6B017C012C
:10CA80002D813E814F815885CA01B9010E94FCED7C
:10CA90009B01AC01C701B6010E944EEA6B017C010B
:10CAA00020E030E040E850E469817A818B819C810C
:10CAB0000E94FCED9B01AC01C701B6010E942EEB68
:10CAC00003C060E070E0CB010E9414EB0E9496EB83
:10CAD0002B013C0197FF03C0412C512C320148141B
:10CAE00059046A047B0410F024013501C12CD12CB7
:10CAF00076018FB7F894F101E45BFF4F90819111BB
:10CB000025C0D10154964D925D926D927C925797BB
:10CB1000C40CD51CE61CF71CF101C08ED18EE28E30
:10CB2000F38E29853A854B855C85DC962D933D9364
:10CB30004D935C93DF97A05CBF4F2D853E854F855D
:10CB400058892D933D934D935C9313978FBF6896AF
:10CB50000FB6F894DEBF0FBECDBFDF91CF911F910E
:10CB60000F91FF90EF90DF90CF90BF90AF909F908C
:10CB70008F907F906F905F904F903F902F9008958F
:10CB80004F925F926F927F92AF92BF92CF92DF925D
:10CB9000EF92FF920F931F93CF93DF93EB017A01F4
:10CBA000209709F458C04115510509F454C0AAA4AE
:10CBB000BBA40CA51DA59501A8016EA17FA188A508
:10CBC00099A50E9427EB882309F445C08FA98111FC
:10CBD0003AC0F70146A057A060A471A4A301920136
:10CBE000B501C8010E942AED18166CF5A301920147
:10CBF000C301B2010E94FCED6B017C018AA99BA9D3
:10CC0000ACA9BDA9BC01CD0190589B01AC010E940B
:10CC10004EEA2EA53FA548A959A90E94FCED9B010B
:10CC2000AC01C701B6010E944DEA0E9469EE6B019A
:10CC30007C019B01AC01B501C8010E9427EB87FD77
:10CC400002C056018701A501B8014EA35FA368A7E2
:10CC500079A781E08EABDF91CF911F910F91FF906B
:10CC6000EF90DF90CF90BF90AF907F906F905F90EC
:10CC70004F900895DF92EF92FF920F931F93CF93FF
:10CC8000DF938091F5098FB7F894E090F4098FBF96
:10CC90008091F50990E08E1991098F70992704977A
:10CCA000ECF01091F50913501F7040E050E000E0E7
:10CCB000F12C8DE4D82E1E1589F011501F70D19ED5
:10CCC000E0011124CA50D64F602F7F2DCE010E9463
:10CCD000C065402F5F2D0C2FFD2EEDCFDF91CF9142
:10CCE0001F910F91FF90EF90DF9008954F925F9208
:10CCF0006F927F92AF92BF92CF92DF92EF92FF92AC
:10CD00000F931F93CF93DF938C01EB01009709F4EE
:10CD100053C0FC0187A981114FC046A057A060A451
:10CD200071A4AEA0BFA0C8A4D9A49501A601C30157
:10CD3000B2010E9427EB87FF3FC0A3019201C3010C
:10CD4000B2010E94FCED2B013C01F80182A993A9DC
:10CD5000A4A9B5A9BC01CD0190589B01AC010E94CA
:10CD60004EEAF80126A537A540A951A90E94FCED7D
:10CD70009B01AC01C301B2010E944DEA0E9469EE21
:10CD80007B018C019B01AC01B501C6010E9427EB20
:10CD900087FF02C0750186019701A801B501C60190
:10CDA0000E9427EB882341F0A701B8014EA35FA39F
:10CDB00068A779A781E08EABDF91CF911F910F918A
:10CDC000FF90EF90DF90CF90BF90AF907F906F90EB
:10CDD0005F904F900895EF92FF920F931F93CF9320
:10CDE000DF931091F409F12C00E080E090E02DE455
:10CDF000E22E2091F509121789F0E19EE00111243D
:10CE0000CA50D64FAE016F2D702F0E9476661F5FFD
:10CE10001F708F2D902FFC2E0D2FEBCF40E050E098
:10CE20006F2D702FDF91CF911F910F91FF90EF9099
:10CE30000C9476664F925F926F927F928F929F9240
:10CE4000AF92BF92CF92DF92EF92FF920F931F9318
:10CE5000CF93DF939090F409C0E0D0E03DE4832EBF
:10CE6000892D992787FD90952091F50930E082174B
:10CE70009307B9F1889E5001899EB00C1124C50119
:10CE80008A50964F5C01209731F18EA9811104C020
:10CE9000F50186A98823F9F0CAA0DBA0ECA0FDA0CB
:10CEA000A7019601F50166A177A180A591A50E9431
:10CEB0002EEB2B013C01A70196016EA17FA188A555
:10CEC00099A50E942EEBAB01BC0193018201CE011A
:10CED0000E94EB631EAA9394F92DFF709F2EE5012B
:10CEE000BFCF2097F1F0CAA0DBA0ECA0FDA0A70166
:10CEF00096016DEC7CEC8CE49DE30E942EEB4B01E3
:10CF00005C01A70196016EA17FA188A599A50E9449
:10CF10002EEBAB01BC0195018401CE010E94EB63B5
:10CF20001EAADF91CF911F910F91FF90EF90DF909C
:10CF3000CF90BF90AF909F908F907F906F905F90B9
:10CF40004F9008950E943A660E94EB660C941A670F
:10CF50001092F4091092F50980E1E4EEF9E0DF01A6
:10CF60001D928A95E9F71092D4091092D509109272
:10CF7000D6091092D7091092D8091092D9091092A7
:10CF8000DA091092DB091092DC091092DD09109287
:10CF9000DE091092DF091092E0091092E109109267
:10CFA000E2091092E3091092D0091092D10910926F
:10CFB000D2091092D30908954F925F926F927F9297
:10CFC0008F929F92AF92BF92CF92DF92EF92FF9299
:10CFD0000F931F93CF93DF938091C60E882309F49C
:10CFE000EBC000914C0110914D01D0914E01C091C8
:10CFF0004F016091D7127091D812882777FD8095E4
:10D00000982F0E94C9EB20E030E040E050E40E94FD
:10D010004EEA98014D2F5C2F0E9427EB87FDCCC074
:10D020005090F409612C712C812C912C4DE4442EEC
:10D030008091F509581609F44EC0459C5001112401
:10D04000C5018A50964F5C01FC0180819181A281CB
:10D05000B381892B8A2B8B2B81F484819581A681C6
:10D06000B781892B8A2B8B2B41F480859185A285F2
:10D07000B385892B8A2B8B2B49F1F5016485758546
:10D08000868597850E94C9EB6B017C01F50160895B
:10D090007189828993890E94C7EB9B01AC01C7010A
:10D0A000B6010E942EEBF50122A133A144A155A1A6
:10D0B0000E94FCED6B017C019B01AC01B301C4013A
:10D0C0000E9427EB87FF02C0360147015394F52DDC
:10D0D000FF705F2EADCF2091480130914901409102
:10D0E0004A0150914B01B301C4010E94FCED9B0128
:10D0F000AC01B8018D2F9C2F0E944EEA6B017C0180
:10D1000098014D2F5C2F0E9427EB87FD14C00091E2
:10D11000500110915101D0915201C09153019801D9
:10D120004D2F5C2FB601C7010E942AED18161CF086
:10D130008601DE2DCF2D8090CB099090CC09A09058
:10D14000CD09B090CE0998014D2F5C2FC501B401D7
:10D150000E942AED1816E4F420E037ED43EA5CE380
:10D16000B8018D2F9C2F0E94FCED6B017C0128E4FF
:10D1700031EE4AE75FE3C501B4010E94FCED9B017B
:10D18000AC01C701B6010E944EEA8B01D82FC92F0E
:10D19000C801AD2FBC2F8093CB099093CC09A093ED
:10D1A000CD09B093CE09B8018D2F9C2F0E9496EB2C
:10D1B0007093D8126093D712DF91CF911F910F9186
:10D1C000FF90EF90DF90CF90BF90AF909F908F90A7
:10D1D0007F906F905F904F9008950F931F93CF9320
:10D1E000C09168059091F5098091F409981781F034
:10D1F0008091F4099DE4899FF0011124E25CF54FD0
:10D20000C0819091F509891719F08F5F8F70F9CF60
:10D21000CC2321F10E94CBE70091C7091091C809E6
:10D220002091C9093091CA0901151105210531055F
:10D2300079F4DC01CB018A569F4FAF4FBF4F8093EB
:10D24000C7099093C809A093C909B093CA090FC030
:10D25000601771078207930750F00AC01092C70940
:10D260001092C8091092C9091092CA0901C0CFEFE3
:10D27000C093B612CF911F910F910C94DC672F923F
:10D280003F924F925F926F927F928F929F92AF9256
:10D29000BF92CF92DF92EF92FF920F931F93CF93A3
:10D2A000DF93CDB7DEB7C458D1090FB6F894DEBF0F
:10D2B0000FBECDBF69AB7AAB8BAB9CAB2DAB3EAB9E
:10D2C0004FAB58AFE9AEFAAE0BAF1CAF60968FAE66
:10D2D000609764969FAE6497A896AFAEA897A09605
:10D2E000BFAEA097C756DF4F1881C959D0402091D3
:10D2F000F5092F5F2F70AC962FAFAC97E22EFF246D
:10D30000E7FCF0948091F40990E08E159F0519F4E4
:10D310000E94B651F7CFCE01C9969F938F93049781
:10D320009F938F9304979F938F934DB75EB744520B
:10D3300051090FB6F8945EBF0FBE4DBFADB7BEB773
:10D34000119684E2E4E5F1E001900D928A95E1F70F
:10D350000E94CAE00FB6F894DEBF0FBECDBF209189
:10D36000070F3091080F4091090F50910A0F69A9DA
:10D370007AA98BA99CA90E94FCED0E94CCED2B01FF
:10D380003C0169A37AA38BA39CA320910B0F30913E
:10D390000C0F40910D0F50910E0F6DA97EA98FA912
:10D3A00098AD0E94FCED0E94CCED4B015C016DA399
:10D3B0007EA38FA398A720910F0F3091100F40915B
:10D3C000110F5091120F69AD7AAD8BAD9CAD0E94DB
:10D3D000FCED0E94CCED2B966CAF7DAF8EAF9FAF76
:10D3E0002B9769A77AA78BA79CA72091130F309141
:10D3F000140F4091150F5091160FD6016D917D912C
:10D400008D919C910E94FCED0E94CCED6B017C0102
:10D410006DA77EA78FA798AB8091E4099091E5094D
:10D42000A091E609B091E709A3019201281B390BED
:10D430004A0B5B0B2F962CAF3DAF4EAF5FAF2F97D4
:10D440008091E8099091E909A091EA09B091EB096E
:10D45000881A990AAA0ABB0A8091EC099091ED09F1
:10D46000A091EE09B091EF092B962CAD3DAD4EADDC
:10D470005FAD2B97281B390B4A0B5B0B2B962CAF00
:10D480003DAF4EAF5FAF2B978091390783FF08C048
:10D49000C092F009D092F109E092F209F092F309FA
:10D4A0008091F0099091F109A091F209B091F309EE
:10D4B00026013701481A590A6A0A7B0A09F497C0FB
:10D4C00034E0139FF0011124E354FD4E20910A0132
:10D4D00030910B0140910C0150910D0160817181DF
:10D4E000828193810E9427EB87FF2CC0C092F009B4
:10D4F000D092F109E092F209F092F309EDE3F0E144
:10D500008491882341F09091C00095FFFCCF8093D7
:10D51000C6003196F5CFE8E6F0E18491882341F02A
:10D520009091C00095FFFCCF8093C6003196F5CF57
:10D530008091C00085FFFCCF8AE08093C600412C1B
:10D54000512C3201C301B20177FE07C0662777274D
:10D55000CB0164197509860997090E94C9EB6B0113
:10D560007C0120E030E046EE53E46091130F7091AF
:10D57000140F8091150F9091160F0E94FCED9B01E6
:10D58000AC01C701B6010E942AED181684F58DA5DD
:10D590009EA5AFA5B8A98093F0099093F109A09337
:10D5A000F209B093F309EDE3F0E18491882341F0AF
:10D5B0009091C00095FFFCCF8093C6003196F5CFC7
:10D5C000EAE4F0E18491882341F09091C00095FF56
:10D5D000FCCF8093C6003196F5CF8091C00085FFC7
:10D5E000FCCF8AE08093C600412C512C32018091FF
:10D5F000F5094DE4849F10011124C1018A50964F12
:10D600001C01FC01E45BFF4F10822F962CAD3DAD59
:10D610004EAD5FAD2F9723962CAF3DAF4EAF5FAFB2
:10D62000239757FF0DC050954095309521953F4F5A
:10D630004F4F5F4F23962CAF3DAF4EAF5FAF239759
:10D6400023968CAD9DADAEADBFAD2397F101808328
:10D650009183A283B38327968CAE9DAEAEAEBFAE50
:10D660002797B7FE0DC022273327A90128193909AA
:10D670004A095B0927962CAF3DAF4EAF5FAF2797A6
:10D6800027968CAD9DADAEADBFAD2797F1018483DC
:10D690009583A683B7832B96CCACDDACEEACFFAC08
:10D6A0002B97F7FE08C0F094E094D094C094C11C6E
:10D6B000D11CE11CF11CD1011896CD92DD92ED92A6
:10D6C000FC921B97E12FF0E06996FFAFEEAF6997F0
:10D6D000C301B20177FE07C066277727CB01641923
:10D6E0007509860997090E94C9EB69962EAD3FAD71
:10D6F0006997220F331F220F331FA5963FAF2EAF1E
:10D70000A597F901E95CFE4F208131814281538167
:10D710000E94FCED0E9496EB9B01AC016996EEAD78
:10D72000FFAD6997EE0FFF1FE15CFE4FA081B18155
:10D730000E944CEF24E630E040E050E00E941CEFF5
:10D74000D1011C962D933D934D935C931F97279683
:10D750008CAD9DADAEADBFAD2797C816D906EA0614
:10D76000FB0614F46C017D01C216D306E406F5062F
:10D7700014F469017A0123968CAD9DADAEADBFADB9
:10D7800023978C159D05AE05BF0514F4D701C6017E
:10D79000F101808B918BA28BB38B0697A105B1050C
:10D7A00010F40C94F473E85BFF4F8091680590913E
:10D7B0006905AA2797FDA095BA2F80839183A2833C
:10D7C000B3832F968CAD9DADAEADBFAD2F9788279F
:10D7D000B7FD83959927AA27BB27282FB7FC22607E
:10D7E0002B968CAD9DADAEADBFAD2B97B7FD246034
:10D7F00077FC2860D10190962C93909791961C937A
:10D8000023962CAD3DAD4EAD5FAD2397232B242B3E
:10D81000252B09F05E98F10184819581A681B7815D
:10D82000892B8A2B8B2B09F05E98F10180859185DD
:10D83000A285B385892B8A2B8B2B09F01598F101D2
:10D8400084859585A685B785892B8A2B8B2B69F0D6
:10D850008091CF09882319F081508093CF0911114D
:10D8600004C05E9880E28093CF09D1011C962D916F
:10D870003D914D915C911F976F962CAF3DAF4EAF90
:10D880005FAF6F97232B242B252B81F1B091F30EE3
:10D89000BFAFE091F40E2496EFAF24970091F50E00
:10D8A0001091F60E2B2F3E2FA80160966FAD60975A
:10D8B00064967FAD6497A8968FADA897A0969FAD0C
:10D8C000A0970E9427EB87FD20C06096FFAD609770
:10D8D000FFAF64962FAD649724962FAF2497A89638
:10D8E0000FADA897A0961FADA0970FC03091D70E8F
:10D8F0003FAF4091D80E24964FAF24970091D90E98
:10D900001091DA0E232F342FCFCF2F966CAD7DAD33
:10D910008EAD9FAD2F970E94C9EB2091070F3091DC
:10D92000080F4091090F50910A0F0E942EEB2F967D
:10D930006CAF7DAF8EAF9FAF2F97698B7A8B8B8B40
:10D940009C8BC501B4010E94C9EB20910B0F309153
:10D950000C0F40910D0F50910E0F0E942EEB4B01BA
:10D960005C016D8B7E8B8F8B988F2B966CAD7DAD14
:10D970008EAD9FAD2B970E94C9EB20910F0F309178
:10D98000100F4091110F5091120F0E942EEB6B015E
:10D990007C01698F7A8F8B8F9C8FC301B2010E94AB
:10D9A000C9EB2091130F3091140F4091150F509136
:10D9B000160F0E942EEBA596EEADFFADA597E95C84
:10D9C000FE4F20813181428153810E94FCED2B0169
:10D9D0003C016996EEADFFAD6997EE0FFF1FE15C6C
:10D9E000FE4F60817181882777FD8095982F0E9476
:10D9F000C9EB9B01AC01C301B2010E94FCED20E028
:10DA000030E048EC52E40E942EEB6D8F7E8F8F8FBA
:10DA100098A3D1012D913D914D915C9113976B96F7
:10DA20002CAF3DAF4EAF5FAF6B9726303105410550
:10DA3000510504F514964D905D906D907C9017976C
:10DA4000B6E04B16510461047104A4F4F101408462
:10DA5000518462847384F6E04F16510461047104AA
:10DA60004CF4DC01CB01BF77F10186A797A7A0ABEF
:10DA7000B1AB29C02F966CAD7DAD8EAD9FAD2F970C
:10DA80000E94A7EE2B013C01C501B4010E94A7EE44
:10DA90009B01AC01C301B2010E944EEA4B015C0143
:10DAA000C701B6010E94A7EE9B01AC01C501B401FC
:10DAB0000E944EEA0E9469EED1019E966D937D937D
:10DAC0008D939C93D197D1019E962D913D914D912F
:10DAD0005C91D197AB962CAF3DAF4EAF5FAFAB979C
:10DAE00060E070E080E89FE30E942EEB9B01AC01B8
:10DAF0006FAD24967FAD2497C8010E94FCED6B01A9
:10DB00007C011091F5098091F409181B1F70E12F19
:10DB1000F0E0EA96FFAFEEAFEA97A701960160E06A
:10DB200074E284E799E40E942EEB0E94CCED4B0155
:10DB30005C01EA968EAD9FADEA970297069798F53D
:10DB40008091270F9091280FA091290FB0912A0F53
:10DB500088169906AA06BB0630F5BC01CD016819E6
:10DB600079098A099B09660F771F881F991F212F42
:10DB700030E040E050E00E94FAEECA01B9010E9494
:10DB8000C7EB0E94CCED680D791D8A1D9B1D0E947C
:10DB9000C7EB9B01AC0160E074E284E799E40E946A
:10DBA0002EEB6B017C01A7019601AB966CAD7DADB0
:10DBB0008EAD9FADAB970E94FCED67966CAF7DAFCD
:10DBC0008EAF9FAF6797D10192966D937D938D93A2
:10DBD0009C93959750964D905D906D907C90539747
:10DBE000C301B2010E94C7EBA3966CAF7DAF8EAFAD
:10DBF0009FAFA397A70196010E94FCED0E9414EB32
:10DC00000E949BEBA7966CAF7DAF8EAF9FAFA7979F
:10DC1000F10160AF71AF82AF93AF9E012F5E3F4FB6
:10DC200061963FAF2EAF619747E15FE0E6965FAF49
:10DC30004EAFE697CE0181969EAF8DAFDE01119675
:10DC4000E296BFAFAEAFE29728961FAE28972C960C
:10DC50001FAE2C97B0E8BFAFEFE32496EFAF249749
:10DC60006196AEADBFAD61976D917D918D919D91A6
:10DC70006196BFAFAEAF6197A70196010E94FCED20
:10DC8000E296EEADFFADE29761937193819391932C
:10DC9000E296FFAFEEAFE2979B01AC015F77E096B3
:10DCA0002CAF3DAF4EAF5FAFE097E696AEADBFADE8
:10DCB000E6978D909D90AD90BD90E696BFAFAEAFCC
:10DCC000E697A5019401E0966CAD7DAD8EAD9FAD5C
:10DCD000E0970E942AED181654F5E0962CAD3DAD64
:10DCE0004EAD5FADE097C501B4010E942EEB162F3B
:10DCF000072FB82EA92E262F372F482F592F2896B9
:10DD00006FAD28972C967FAD2C978FAD24969FAD45
:10DD100024970E9427EB87FD0AC028961FAF2897FB
:10DD20002C960FAF2C97BFAE2496AFAE249761967A
:10DD3000EEADFFAD61972DAD3EADE217F30709F0F3
:10DD40008FCF20E030E040E85FE328966FAD289762
:10DD50002C967FAD2C978FAD24969FAD24970E9473
:10DD600027EB87FF55C07E0131E1E30EF11C8E01E8
:10DD70000F5F1F4F28962FAD28972C963FAD2C97FD
:10DD80004FAD24965FAD2497D8016D917D918D9113
:10DD90009C910E94FCEDF8016193719381939193A2
:10DDA0008F01EE15FF0531F728962FAD28972C9699
:10DDB0003FAD2C974FAD24965FAD249767966CAD21
:10DDC0007DAD8EAD9FAD67970E94FCEDD10192961F
:10DDD0006D937D938D939C939597A7966CAD7DAD38
:10DDE0008EAD9FADA7970E94C7EB28962FAD2897C1
:10DDF0002C963FAD2C974FAD24965FAD24970E9493
:10DE0000FCED0E949BEBF10160AF71AF82AF93AF6D
:10DE1000AB962CAD3DAD4EAD5FADAB97A3966CAD63
:10DE20007DAD8EAD9FADA3970E942EEB4B015C01A3
:10DE3000D10114962D913D914D915C9117972B96A0
:10DE40002CAF3DAF4EAF5FAF2B9718962D913D9104
:10DE50004D915C911B972F962CAF3DAF4EAF5FAFAE
:10DE60002F976B962CAD3DAD4EAD5FAD6B97232BD1
:10DE7000242B252B31F52B968CAD9DADAEADBFADD2
:10DE80002B97892B8A2B8B2BE1F42F962CAD3DAD54
:10DE90004EAD5FAD2F97232B242B252B91F4209192
:10DEA000EB0E3091EC0E4091ED0E5091EE0EC5014F
:10DEB000B4010E94FCED0E9414EB81010C5B1F4F2A
:10DEC0001BC081010C5B1F4F6F962CAD3DAD4EAD5D
:10DED0005FAD6F97232B242B252BB9F42091E70EF0
:10DEE0003091E80E4091E90E5091EA0EC501B4015F
:10DEF0000E94FCED0E9414EB0E949BEBD8016D93F5
:10DF00007D938D939C93139715C02091EF0E3091C4
:10DF1000F00E4091F10E5091F20EC501B4010E9435
:10DF2000FCED0E9414EB0E949BEBF801608371836F
:10DF300082839383F101EC5BFF4FC080D180E2804C
:10DF4000F3802091C70E3091C80E4091C90E5091B8
:10DF5000CA0E23962CAF3DAF4EAF5FAF2397809193
:10DF6000CB0E9091CC0EA091CD0EB091CE0E2796F7
:10DF70008CAF9DAFAEAFBFAF27972091CF0E309142
:10DF8000D00E4091D10E5091D20E63962CAF3DAF82
:10DF90004EAF5FAF63978091D30E9091D40EA09156
:10DFA000D50EB091D60E67968CAF9DAFAEAFBFAF1A
:10DFB00067976B962CAD3DAD4EAD5FAD6B97C701CE
:10DFC000B6010E94C2EEA30192010E94FAEE2396CE
:10DFD0008CAD9DADAEADBFAD239782179307A4075F
:10DFE000B50780F49C01AD01C301B2010E94C2EEED
:10DFF0006B962CAD3DAD4EAD5FAD6B970E94FAEECA
:10E0000069017A01A70196012B966CAD7DAD8EADAD
:10E010009FAD2B970E94C2EEA30192010E94FAEEDF
:10E0200027968CAD9DADAEADBFAD279782179307F8
:10E03000A407B50780F49C01AD01C301B2010E94A1
:10E04000C2EE2B962CAD3DAD4EAD5FAD2B970E9431
:10E05000FAEE69017A01A70196012F966CAD7DADAC
:10E060008EAD9FAD2F970E94C2EEA30192010E9438
:10E07000FAEE63968CAD9DADAEADBFAD63978217E2
:10E080009307A407B50780F49C01AD01C301B20159
:10E090000E94C2EE2F962CAD3DAD4EAD5FAD2F97D9
:10E0A0000E94FAEE69017A01A70196016F966CADA4
:10E0B0007DAD8EAD9FAD6F970E94C2EEA301920120
:10E0C0000E94FAEE67968CAD9DADAEADBFAD679781
:10E0D00082179307A407B50780F49C01AD01C30123
:10E0E000B2010E94C2EE6F962CAD3DAD4EAD5FAD5C
:10E0F0006F970E94FAEE69017A01F101EC5BFF4F24
:10E10000C082D182E282F382C701B6010E94C7EBCE
:10E110006B017C01A50194010E942EEBC358DF4FD7
:10E12000688379838A839B83CD57D040D101D2966F
:10E130006D937D938D939C93D59720E030E040E8DC
:10E140005BE4C701B6010E94FCED20E034E244EF3D
:10E1500059E40E942EEB0E9496EBF101648F758FBB
:10E16000868F978F2091E30E3091E40E4091E50E5B
:10E170005091E60EA3962CAF3DAF4EAF5FAFA39785
:10E1800020E030E040E05FE3A3966CAD7DAD8EAD66
:10E190009FADA3970E94FCED28966FAF28972C9611
:10E1A0007FAF2C978FAF24969FAF24978091DF0E7F
:10E1B0009091E00EA091E10EB091E20EA7968CAF87
:10E1C0009DAFAEAFBFAFA79720E030E040E05FE388
:10E1D000BC01CD010E94FCED162F072FF82EE92E71
:10E1E0002091DB0E3091DC0E4091DD0E5091DE0E61
:10E1F000E0962CAF3DAF4EAF5FAFE09720E030E050
:10E2000040E05FE3E0966CAD7DAD8EAD9FADE097F5
:10E210000E94FCEDD62EC72EB82EA92E89859A8590
:10E22000AB85BC85E4968CAF9DAFAEAFBFAFE49736
:10E230002D853E854F855889E8962CAF3DAF4EAF72
:10E240005FAFE897BC01CD019F77212F302F4F2D75
:10E250005E2D0E942AED1816E4F4212F302F4F2D49
:10E260005E2D28966FAD28972C967FAD2C978FAD9D
:10E2700024969FAD24970E9427EB87FD0AC028961D
:10E280001FAF28972C960FAF2C97FFAE2496EFAEBA
:10E2900024972D2D3C2D4B2D5A2DE8966CAD7DAD40
:10E2A0008EAD9FADE8979F770E942AED1816E4F493
:10E2B0002D2D3C2D4B2D5A2D28966FAD28972C9641
:10E2C0007FAD2C978FAD24969FAD24970E9427EBAE
:10E2D00087FD0AC02896DFAE28972C96CFAE2C97E4
:10E2E000BFAE2496AFAE2497D1019296BC916C96A6
:10E2F000BFAF6C97F101F3A16896FFAF6897D101AA
:10E300009496BC916096BFAF6097F101F5A16496B9
:10E31000FFAF64976C962FAD6C9768963FAD68978A
:10E320004B2F5F2F28966FAD28972C967FAD2C979B
:10E330008FAD24969FAD24970E9427EB87FD16C0D2
:10E340006C962FAD6C9728962FAF289768963FADA7
:10E3500068972C963FAF2C9760964FAD60974FAF64
:10E3600064965FAD649724965FAF2497EA968EAD6E
:10E370009FADEA9702970CF42CC19091D009E996D1
:10E380009FAFE997A091D109EB96AFAFEB97B09112
:10E39000D209EC96BFAFEC97E091D309ED96EFAFC1
:10E3A000ED9727E137EB41ED58E3692F7A2F8B2F5B
:10E3B0009E2F0E942AED18160CF00BC12091D40953
:10E3C0003091D5094091D6095091D70969817A8158
:10E3D0008B819C810E944DEA2B013C012091D80940
:10E3E0003091D9094091DA095091DB096D817E8124
:10E3F0008F8198850E944DEA4B015C012091DC09D8
:10E400003091DD094091DE095091DF09E4966CAD51
:10E410007DAD8EAD9FADE4970E944DEA6B017C010E
:10E42000E894F7F82091E0093091E1094091E20980
:10E430005091E309E8966CAD7DAD8EAD9FADE89748
:10E440000E944DEA9B01AC015F77CF57DF4F2883D5
:10E4500039834A835B83C158D040A3019201C30131
:10E46000B2010E94FCED2B013C01A5019401C50104
:10E47000B4010E94FCED9B01AC01C301B2010E94FA
:10E480004EEA0E9469EE4B015C01A3962CAD3DADB6
:10E490004EAD5FADA3970E942AED18166CF4A5014E
:10E4A0009401A3966CAD7DAD8EAD9FADA3970E94F8
:10E4B0002EEB4B015C0106C0812C912C50E8A52E5F
:10E4C0006FE3B62EA7962CAD3DAD4EAD5FADA797D1
:10E4D000C701B6010E942AED1816E4F4A7019601BF
:10E4E000A7966CAD7DAD8EAD9FADA7970E942EEB2C
:10E4F000162F072FF82EE92E262F372F482F592FAA
:10E50000B401C5010E9427EB87FD04C0812E902E27
:10E51000AF2CBE2CE0962CAD3DAD4EAD5FADE0977F
:10E52000CF57DF4F688179818A819B81C158D04064
:10E530000E942AED1816E4F4CF57DF4F2881398165
:10E540004A815B81C158D040E0966CAD7DAD8EAD07
:10E550009FADE0970E942EEB7B018C019B01AC01EB
:10E56000B401C5010E9427EB87FD02C04701580195
:10E570009401A5016C966FAD6C9768967FAD689716
:10E5800060968FAD609764969FAD64970E94FCED96
:10E590007B018C019B01AC01E9966FADE997EB968D
:10E5A0007FADEB97EC968FADEC97ED969FADED9729
:10E5B0000E9427EB87FF17C0E996EFACE997EB962F
:10E5C000FFACEB97EC960FADEC97ED961FADED978A
:10E5D0000AC02896EFAC28972C96FFAC2C970FAD6D
:10E5E00024961FAD2497C701D801F10182A793A7F4
:10E5F000A4A7B5A7C358DF4F688179818A819B8121
:10E60000CD57D04090589B01AC010E944EEAAB968A
:10E610002CAD3DAD4EAD5FADAB970E94FCED9B01C7
:10E62000AC016BE077ED83E29BE30E944DEA0E9430
:10E6300069EE5B016C019B01AC01B701C8010E944E
:10E6400027EB87FF02C0902E03C075019C2C1D2D67
:10E65000C701A92DB12FF10186A397A3A0A7B1A748
:10E6600001E09501A6016C966FAD6C9768967FAD41
:10E67000689760968FAD609764969FAD64970E948F
:10E6800027EB18160CF400E0D101D7960C93D7971E
:10E6900081E0D6968C9389819A81AB81BC818093ED
:10E6A000D4099093D509A093D609B093D7098D8149
:10E6B0009E81AF81B8858093D8099093D909A093A2
:10E6C000DA09B093DB09E4962CAD3DAD4EAD5FADFC
:10E6D000E4972093DC093093DD094093DE095093E1
:10E6E000DF09E8968CAD9DADAEADBFADE8978093E8
:10E6F000E0099093E109A093E209B093E3096C96D5
:10E700008FAD6C9768969FAD68976096AFAD609738
:10E710006496BFAD64978093D0099093D109A0937C
:10E72000D209B093D3099C01AD0128966FAD28970B
:10E730002C967FAD2C978FAD24969FAD24970E9489
:10E740002EEB2B013C016C962FAD6C9768963FAD7C
:10E75000689760964FAD609764965FAD6497B70118
:10E76000892D912F0E942EEBAB01BC0193018201F8
:10E77000C1010E94EB63AC969FADAC979093F509F5
:10E7800089A19AA1ABA1BCA18093E4099093E5096A
:10E79000A093E609B093E7098DA19EA1AFA1B8A50A
:10E7A0008093E8099093E909A093EA09B093EB09F3
:10E7B00089A59AA5ABA5BCA58093EC099093ED091A
:10E7C000A093EE09B093EF098DA59EA5AFA5B8A9BA
:10E7D0008093F0099093F109A093F209B093F309A3
:10E7E0000E94A2670E940499CC57DF4F0FB6F8949D
:10E7F000DEBF0FBECDBFDF91CF911F910F91FF9074
:10E80000EF90DF90CF90BF90AF909F908F907F90D0
:10E810006F905F904F903F902F9008956F927F92EE
:10E820008F929F92AF92BF92CF92DF92EF92FF9220
:10E830000F931F93CF93DF93CDB7DEB7A4970FB697
:10E84000F894DEBF0FBECDBF3C0182E090E00E9495
:10E85000F29F6B017C0181E090E00E94F29F4B01EE
:10E860005C0180E090E00E94F29FAB01BC01950149
:10E870008401C3010E94EEDE8DB79EB784970FB668
:10E88000F8949EBF0FBE8DBFADB7BEB7119684E2A0
:10E89000E4E5F1E001900D928A95E1F7CE01019651
:10E8A0000E94D7E28DB79EB784960FB6F894DEBF6C
:10E8B0000FBECDBF84970FB6F8949EBF0FBE8DBF1D
:10E8C000ADB7BEB7119684E2FE01319601900D926C
:10E8D0008A95E1F7C3010E9485DF0FB6F894DEBF89
:10E8E0000FBECDBFC301A4960FB6F894DEBF0FBE16
:10E8F000CDBFDF91CF911F910F91FF90EF90DF90EF
:10E90000CF90BF90AF909F908F907F906F90089521
:10E91000CF92DF92EF92FF920F931F93CF93DF93EB
:10E92000CDB7DEB76C970FB6F894DEBF0FBECDBF84
:10E93000698B7A8B8B8B9C8B2D8B3E8B4F8B588F5F
:10E94000E98EFA8E0B8F1C8FCE0149969F938F9381
:10E9500004979F938F9304979F938F938DB79EB740
:10E9600084970FB6F8949EBF0FBE8DBFADB7BEB7EC
:10E97000119684E2E4E5F1E001900D928A95E1F7C9
:10E980000E94CAE00FB6F894DEBF0FBECDBF209143
:10E99000070F3091080F4091090F50910A0F6989B4
:10E9A0007A898B899C890E94FCED0E94CCED609352
:10E9B000E4097093E5098093E6099093E7096D8770
:10E9C0007E878F87988B20910B0F30910C0F409191
:10E9D0000D0F50910E0F6D897E898F89988D0E9441
:10E9E000FCED0E94CCED6093E8097093E9098093F7
:10E9F000EA099093EB0969877A878B879C87209136
:10EA00000F0F3091100F4091110F5091120F698D1F
:10EA10007A8D8B8D9C8D0E94FCED0E94CCED6093D5
:10EA2000EC097093ED098093EE099093EF096D83E3
:10EA30007E838F8398872091130F3091140F40911C
:10EA4000150F5091160FF6016081718182819381BB
:10EA50000E94FCED0E94CCED6093F0097093F109E7
:10EA60008093F2099093F30969837A838B839C8363
:10EA70009E012F5F3F4FAE014B5F5F4FBE01675F4F
:10EA80007F4FCE010D960E94979F1092D009109251
:10EA9000D1091092D2091092D3091092D409109280
:10EAA000D5091092D6091092D7091092D809109260
:10EAB000D9091092DA091092DB091092DC09109240
:10EAC000DD091092DE091092DF091092E009109220
:10EAD000E1091092E2091092E3096C960FB6F894DE
:10EAE000DEBF0FBECDBFDF91CF911F910F91FF9081
:10EAF000EF90DF90CF9008952091130F3091140F75
:10EB00004091150F5091160FFC0160817181828137
:10EB100093810E94FCED0E94CCED6093F00970930C
:10EB2000F1098093F2099093F30980EF99E00C9436
:10EB3000D39FCF92DF92EF92FF920F931F93CF93C9
:10EB4000DF9300D000D0CDB7DEB777EFC72E7EE0E1
:10EB5000D72EE7E0EE2EEFE0FE2E07EC1EE0F601EA
:10EB600061917191819191916F01F70121913191A1
:10EB7000419151917F0129833A834B835C830E94A9
:10EB8000C7EB29813A814B815C810E94FCED0E9498
:10EB90009BEBF80161937193819391938F01F7E05F
:10EBA000CF16FFE0DF06D9F60F900F900F900F9071
:10EBB000DF91CF911F910F91FF90EF90DF90CF9059
:10EBC00008954F925F926F927F92AF92BF92CF92D1
:10EBD000DF92EF92FF920F931F93CF93DF93EC019D
:10EBE0008B017A0163E070E00E94E6EE5C01F801BF
:10EBF000D70120E030E028173907A4F44081518183
:10EC0000628173814D905D906D907C9013974192DD
:10EC10005192619271924D935D936D937D932F5FAD
:10EC20003F4FE9CFDC01AA0FBB1FAA0FBB1FF801A2
:10EC3000EA0FFB1FAE0DBF1DAC16BD060CF040C0A9
:10EC400040815181628173810D911D912D913C9183
:10EC5000139700831183228333834D935D936D93C8
:10EC60007C931397448155816681778114960D9129
:10EC70001D912D913C91179704831583268337832B
:10EC800014964D935D936D937C9317970085118532
:10EC9000228533851896CD90DD90ED90FC901B97E2
:10ECA000C086D186E286F38618960D931D932D9328
:10ECB0003C931B9783E0A80EB11C3C961C96BCCFDE
:10ECC000DF91CF911F910F91FF90EF90DF90CF9048
:10ECD000BF90AF907F906F905F904F9008952F926C
:10ECE0003F924F925F926F927F928F929F92AF92DC
:10ECF000BF92CF92DF92EF92FF920F931F93CF9329
:10ED0000DF9300D000D000D0CDB7DEB75C017C83AC
:10ED10006B838A01FA01C080D180E280F38020E019
:10ED200030E0A901C701B6010E9427EB87FF04C0AC
:10ED3000F7FAF094F7F8F0949501220F331F220FA1
:10ED4000331F3A8329831E821D828D819E81EB8130
:10ED5000FC818E179F07B4F5812C912C212C312C2E
:10ED60002A143B042CF5F801E80DF91D4080518070
:10ED70006280738020E030E0A901C301B2010E94EB
:10ED800027EB87FF04C077FA709477F87094A3019B
:10ED90009201C701B6010E9427EB87FF02C07301F1
:10EDA00062013FEF231A330A84E0880E911CD8CF0A
:10EDB000ED81FE813196FE83ED8329813A81020F38
:10EDC000131FC3CFC701B60126960FB6F894DEBF56
:10EDD0000FBECDBFDF91CF911F910F91FF90EF90AC
:10EDE000DF90CF90BF90AF909F908F907F906F906B
:10EDF0005F904F903F902F9008952F923F924F92A7
:10EE00005F926F927F928F929F92AF92BF92CF92BA
:10EE1000DF92EF92FF920F931F93CF93DF937B01CB
:10EE2000EE0CFF1CEE0CFF1CE0E0F0E000E010E058
:10EE3000041715073CF5A0E0B0E0212C312C590156
:10EE4000AE0EBF1E4C018E0E9F1E26163706ACF46A
:10EE50006501CA0EDB1EE601488059806A807B800E
:10EE60006401CA0EDB1EE601488259826A827B82F7
:10EE7000DFEF2D1A3D0A1496E8CF0F5F1F4FEE0DFE
:10EE8000FF1DD6CFDF91CF911F910F91FF90EF9093
:10EE9000DF90CF90BF90AF909F908F907F906F90BA
:10EEA0005F904F903F902F9008952F923F924F92F6
:10EEB0005F926F927F928F929F92AF92BF92CF920A
:10EEC000DF92EF92FF920F931F93CF93DF9300D0C7
:10EED00000D000D0CDB7DEB79E838D834A015B01A1
:10EEE0003901181619060CF028C120E030E0A901FC
:10EEF000C501B4010E9427EB882309F41EC101302B
:10EF0000110529F421E0C216D10489F473C017FF5A
:10EF10000EC021E030E04D815E81241B350B209F27
:10EF2000C001219F900D309F900D112402C080E000
:10EF300090E0D7FE0EC021E030E0ED81FE812E1B77
:10EF40003F0B2C9DA0012D9D500D3C9D500D11247B
:10EF500002C040E050E09601220F331F220F331F02
:10EF60003C832B83F801EE0FFF1FEE0FFF1FFA8388
:10EF7000E9838A01000F111F000F111F0E0D1F1DC5
:10EF80007C01EE0CFF1CEE0CFF1CE60CF71C612C48
:10EF9000712CC12CD12C412C512C18012C0C3D1C56
:10EFA000F701E60DF71D2081318142815381C501B2
:10EFB000B4010E94FCED9B01AC01F1016081718103
:10EFC000828193810E944EEAF10160837183828382
:10EFD0009383FFEF4F1A5F0A2B813C81C20ED31E31
:10EFE00049815A81640E751E8D819E81481659068D
:10EFF000A1F6A3C0CD80DE8093E0C922DD241301F9
:10F000008701412C512C4C145D04ECF4F101219149
:10F010003191419151911F01C501B4010E94FCED54
:10F020009B01AC01F80160817181828193810E9412
:10F030004EEAF80161937193819391938F01FFEFF1
:10F040004F1A5F0AE0CFC601880F991F880F991FDA
:10F050008701080F191F7C0124E0E20EF11CE60C69
:10F06000F71C4D815E81C416D5060CF066C0F70111
:10F0700034972081318142815381C501B4010E94BE
:10F08000FCED9B01AC01F80160817181828193816B
:10F090000E944EEAF8016083718382839383F701B3
:10F0A0002081318142815381C501B4010E94FCED70
:10F0B0009B01AC01F80164817581868197810E9472
:10F0C0004EEAF8016483758386839783F701248170
:10F0D000358146815781C501B4010E94FCED9B0139
:10F0E000AC01F80160857185828593850E944EEAA6
:10F0F000F8016087718782879387F70120853185C2
:10F1000042855385C501B4010E94FCED9B01AC0111
:10F11000F80164857585868597850E944EEAF80119
:10F120006487758786879787F4E0CF0ED11C005FD0
:10F130001F4F20E1E20EF11C94CF26960FB6F894F3
:10F14000DEBF0FBECDBFDF91CF911F910F91FF901A
:10F15000EF90DF90CF90BF90AF909F908F907F9077
:10F160006F905F904F903F902F9008952F923F9215
:10F170004F925F926F927F928F929F92AF92BF92C7
:10F18000CF92DF92EF92FF920F931F93CF93DF9373
:10F1900000D000D0CDB7DEB77C015B016901181645
:10F1A00019060CF01DC14130510521F40130110543
:10F1B00079F46AC057FF0CC081E090E08E199F0976
:10F1C000849F2001859F500C949F500C112402C0F5
:10F1D000412C512C17FF0CC021E030E02E193F09C3
:10F1E000209FC001219F900D309F900D112402C0DF
:10F1F00080E090E01A01220C331C220C331C980191
:10F20000220F331F220F331F3A832983440C551CCE
:10F21000440C551C4A0C5B1C5C01AA0CBB1CAA0CC0
:10F22000BB1CAC0CBD1C00E010E0C12CD12C612C2F
:10F23000712C812C912C1C821B82F201EC0DFD1D86
:10F24000D501A00FB11F2D913D914D915C91608131
:10F250007181828193810E94FCED9B01AC01B3011D
:10F26000C4010E944EEA3B014C018B819C810196B6
:10F270009C838B83C20CD31CE981FA810E0F1F1F64
:10F280008E159F05D1F6B0C065E070E00E94E6EEF5
:10F290009C838B832C01BA82A9821901612C712C69
:10F2A000812C912C00E010E02B813C810217130788
:10F2B000DCF4E981FA816191719181919191FA83F4
:10F2C000E983F10121913191419151911F010E94F6
:10F2D000FCED9B01AC01B301C4010E944EEA3B016D
:10F2E0004C010F5F1F4FE0CFC901880F991F880F96
:10F2F000991F8501080F191F1C012C0C3D1C4E1471
:10F300005F040CF071C0F101208131814281538191
:10F31000F80160817181828193810E94FCED5B0123
:10F320006C01F1012481358146815781F8016481A6
:10F330007581868197810E94FCED9B01AC01C6011D
:10F34000B5010E944EEA5B016C01F1012085318517
:10F3500042855385F80160857185828593850E9479
:10F36000FCED9B01AC01C601B5010E944EEA5B01B8
:10F370006C01F1012485358546855785F801648542
:10F380007585868597850E94FCED9B01AC01C601C1
:10F39000B5010E944EEA5B016C01F10120893189BF
:10F3A00042895389F80160897189828993890E9411
:10F3B000FCED9B01AC01C601B5010E944EEA9B0128
:10F3C000AC01B301C4010E944EEA3B014C01F5E0DF
:10F3D0004F0E511C0C5E1F4F24E1220E311C8FCFAB
:10F3E000612C712C812C912CB301C4010F900F90D2
:10F3F0000F900F90DF91CF911F910F91FF90EF90A1
:10F40000DF90CF90BF90AF909F908F907F906F9044
:10F410005F904F903F902F9008952F923F924F9280
:10F420005F926F927F928F929F92AF92BF92CF9294
:10F43000DF92EF92FF920F931F93CF93DF9300D051
:10F4400000D0CDB7DEB79C838B83181619060CF05D
:10F450009AC0141615060CF096C0019799F4FB019A
:10F46000C080D180E280F38020E030E0A901C701B4
:10F47000B6010E9427EB87FF89C0F7FAF094F7F8EE
:10F48000F09484C0CA01880F991F880F991F9A832E
:10F4900089838B01212C312C812C912CA0E8AA2E60
:10F4A000AFE3BA2E412C512C612C712CF801C08095
:10F4B000D180E280F38020E030E0A901C701B601ED
:10F4C0000E9427EB882309F444C020E030E0A90122
:10F4D000C701B6010E9427EB87FF04C0F7FAF0943A
:10F4E000F7F8F094A7019601B201C3010E9427EB3F
:10F4F00087FF1DC0A7019601B201C3010E942EEB38
:10F500002B013C019B01AC01C501B4010E94FCED43
:10F51000A30192010E94FCED20E030E040E85FE3AF
:10F520000E944EEA4B015C012601370112C0920194
:10F53000A301C701B6010E942EEB9B01AC010E9402
:10F54000FCED9B01AC01C501B4010E944EEA4B01E8
:10F550005C01FFEF2F1A3F0A89819A81080F191F5A
:10F56000EB81FC812E163F0609F0A0CFC501B40146
:10F570000E9469EE9B01AC01B201C3010E94FCED47
:10F580006B017C0103C0C12CD12C7601C701B601EF
:10F590000F900F900F900F90DF91CF911F910F91CF
:10F5A000FF90EF90DF90CF90BF90AF909F908F90A3
:10F5B0007F906F905F904F903F902F9008952F9283
:10F5C0003F924F925F926F927F928F929F92AF92F3
:10F5D000BF92CF92DF92EF92FF920F931F93CF9340
:10F5E000DF93CDB7DEB7E4970FB6F894DEBF0FBE5A
:10F5F000CDBF9C878B877A876987588B4F87290176
:10F600001CA30BA315019C8E8B8E2F96EEADFFAD28
:10F610002F97CF01815F984D21E030E08F319E44DC
:10F6200010F420E030E0CF0160E177E20E94E6EEE6
:10F6300061E070E07E8B6D8B892B11F41E8A1D8A30
:10F64000CF0168EE73E00E94E6EE8D599F4FA1E076
:10F65000B0E0BAA3A9A3873C910510F41AA219A29D
:10F66000CF0164E670E00E94E6EE099641E050E0CA
:10F670005E8F4D8F439710F41E8E1D8ECF016AE072
:10F6800070E00E94E6EE61E070E078A36F8F892B56
:10F6900011F418A21F8E6F84788871E0671A7108C0
:10F6A000461457040CF432016114710409F062C06D
:10F6B000232B51F0F70180819181A281B381F60162
:10F6C00080839183A283B3832D893E89232B51F0BC
:10F6D000F70180819181A281B381F10180839183BF
:10F6E000A283B3832F8D38A1232B69F0F70180818A
:10F6F0009181A281B3812D96EEADFFAD2D978083D0
:10F700009183A283B38329A13AA1232BF9F0AB857E
:10F71000BC858D909D90AD90BC9020E030E0A9011B
:10F72000C501B4010E9427EB882391F0A501940143
:10F73000F70160817181828193810E942EEBAB8DF4
:10F74000BC8D6D937D938D939C9313971D8202C006
:10F75000B1E0BD831D86ED8DFE8DEF2B09F413C442
:10F760002B96AEADBFAD2B971D921D921D921C9294
:10F77000139709C42115310529F4ED89FE89EF2B72
:10F78000B9F413C0F701D60181E090E04F855889A4
:10F790004817590794F341915191619171914D939B
:10F7A0005D936D937D930196F1CF232BA1F46DC0F2
:10F7B000F701D10181E090E06F85788968177907BA
:10F7C000A4F341915191619171914D935D936D932A
:10F7D0007D930196F1CFA985BA85A095B095AA0F22
:10F7E000BB1FAA0FBB1FBE83AD839301220F331F24
:10F7F000220F331FEBA1FCA1E20FF31FFAABE9AB21
:10F8000049855A854F5F5F4FC3010197849F50011F
:10F81000859FB00C949FB00C1124AA0CBB1CAA0CA1
:10F82000BB1C4B855C85A40EB51EB601620F731F11
:10F83000A985BA858A9F40018B9F900C9A9F900C56
:10F840001124860C971C880C991C880C991C840E1A
:10F85000951E18A61FA21EA21DA21E861D86E1E0EF
:10F86000F0E0FA83E983645071097CA76BA7F4E0A8
:10F870008F1A91082F853889261937093CAB2BAB95
:10F88000A981BA816A167B0634F48D899E89892BF9
:10F8900009F07EC09EC0E9A9FAA94D855E85E40FF6
:10F8A000F51F3497C080D180E280F38020E030E003
:10F8B000A901C701B6010E9427EB882309F44EC0B5
:10F8C0006DA17EA16A0D7B1D7AA769A7DB018D91D1
:10F8D0009D910D90BC91A02D8DA79EA7AFA7B8AB11
:10F8E000FB01C082D182E282F38201E010E02BA50D
:10F8F0003CA54D855E85240F351F3A8B298B41E051
:10F9000050E06FA178A5680D791D78876F838BA96A
:10F910009CA9A981BA818A0F9B1F9C838B830E941B
:10F92000B6789058A70196010E942EEBAB01BC015E
:10F93000CC24C394D12CE988FA882F8138858B8117
:10F940009C810E9455772DA53EA54FA558A9A9A534
:10F95000BAA52D933D934D935C931397E981FA815A
:10F960003196FA83E9832D853E85245031093E87FF
:10F970002D874DA15EA16D817E81460F571F5EA32D
:10F980004DA38FA198A5860F971F98A78FA378CF17
:10F990002BA13CA138872F83A984BA843FEFA31AF7
:10F9A000B30AAA0CBB1CAA0CBB1C4B855C855A83F2
:10F9B00049836F8578897E836D833E862D864A01D3
:10F9C00081E090E09C838B838B819C816816790613
:10F9D00034F4E9A1FAA1EF2B09F06FC062C0AF8146
:10F9E000B885CD90DD90ED90FD90B887AF8320E095
:10F9F00030E0A901C701B6010E9427EB8823B9F1C5
:10FA0000A981BA812D913D914D915C911397298BDC
:10FA10003A8B4B8B5C8BFD01C082D182E282F382F8
:10FA200001E010E02D853E8541E050E0B4018D817C
:10FA30009E810E94B6789058A70196010E942EEBF5
:10FA4000AB01BC01CC24C394D12CED84FE84940181
:10FA50008D819E810E94557729893A894B895C89DD
:10FA6000A981BA812D933D934D935C931397EB81BC
:10FA7000FC813196FC83EB8329813A812A0D3B1D61
:10FA80003A8329834D815E81415051095E834D83C4
:10FA90008A0C9B1C6D857E856C5F7F4F7E876D8792
:10FAA00093CFAF8DB8A1AB2B91F1B1012D964EAD97
:10FAB0005FAD2D9721E030E017C0B1014B8D5C8D1B
:10FAC00021E030E04216530664F3FB0181919191ED
:10FAD000A191B191BF01FA0181939193A193B19347
:10FAE000AF012F5F3F4FEECF421653060CF441C0DB
:10FAF000FB0181919191A191B191BF01FA01819393
:10FB00009193A193B193AF012F5F3F4FEDCFED8D57
:10FB1000FE8DEF2BC1F12F85388942165306E4F58F
:10FB20009201B201660F771F660F771FA101460F82
:10FB3000571F2B968EAD9FAD2B97680F791F80E0D6
:10FB400090E02F5F3F4FAF85B889A217B3070CF441
:10FB5000F6C1FA01E80FF91FC080D180E280F3807E
:10FB6000FB01E80FF91FC082D182E282F382049682
:10FB7000E8CF2D8D3E8D232B71F6EF85F8894E163B
:10FB80005F060CF4E1C1A9A1BAA1AB2BA1F462C03C
:10FB90008D8D9E8D892BB9F32B96EEADFFAD2B97F6
:10FBA00081E090E04816590674F311921192119277
:10FBB00011920196F7CFF201EE0FFF1FEE0FFF1F1C
:10FBC0002B8D3C8D2E0F3F1F3A8329832CEF4985C7
:10FBD0005A852403B001259F700D11247AA369A3CF
:10FBE00040955095440F551F440F551F5E8B4D8B0C
:10FBF00029853A852F5F3F4FC2010197829F4001BF
:10FC0000839F900C929F900C1124880C991C880C57
:10FC1000991CAB85BC858A0E9B1EE985FA858E9F53
:10FC200050018F9FB00C9E9FB00C1124AA0CBB1CDE
:10FC3000AA0CBB1CAA0EBB1E12011A8A198A1886AE
:10FC40001F8221E030E03C832B83EB81FC814E1648
:10FC50005F061CF41D821D865DC0A2016B817C8144
:10FC6000461B570B5EA34DA32D823D86E989FA8979
:10FC7000E80DF91DC080D180E280F38020E030E003
:10FC8000A901C701B6010E9427EB882309F442C0ED
:10FC9000A7019601A981BA819E918E917E916E9164
:10FCA000BA83A9830E942EEBE981FA816083718374
:10FCB00082839383F1E02F16310491F0AB01BC01F4
:10FCC0007058CC24C394D12CEB8CFC8C01E010E058
:10FCD0002F8138852A0D3B1D8DA19EA10E9455774D
:10FCE0002B813C812F5F3F4F3C832B8331E0231AD4
:10FCF00031084F81588569A17AA1460F571F58874F
:10FD00004F8389899A89AD89BE898A0F9B1F9A8BF7
:10FD1000898B9BCF2D8D3E8D232B29F44F8D58A1A0
:10FD2000452B09F430C169857A8560957095660F19
:10FD3000771F660F771F7A83698389859A85019675
:10FD4000930121503109289F1001299F300C389FC1
:10FD5000300C1124220C331C220C331C8B859C8507
:10FD6000280E391EC301880F991F880F991FABA158
:10FD7000BCA1A80FB91FBCA3ABA32B96EEADFFADE2
:10FD80002B97E80FF91FF88FEF8B49855A85249F31
:10FD90002001259F500C349F500C1124460C571CF9
:10FDA000440C551C440C551C6B857C85460E571E17
:10FDB0002D96AEADBFAD2D97A80FB91F1C821B822B
:10FDC0001C861B86E1E0F0E0FA87E9871497BA8F7A
:10FDD000A98FF4E04F1A51082F8538892619370961
:10FDE000388B2F874F89588D44505109588F4F8B2E
:10FDF00089859A85681679060CF4C5C0EBA1FCA12B
:10FE00006B857C85E60FF71F3497C080D180E28038
:10FE1000F38020E030E0A901C701B6010E9427EB82
:10FE2000882309F476C0D1018D919D910D90BC91EC
:10FE3000A02D898B9A8BAB8BBC8BF101C082D182B8
:10FE4000E282F3822D8D3E8D232B59F101E010E0EB
:10FE50004F89588D6B857C85460F571F58874F8378
:10FE60009A0141E050E08B809C80840C951CB40189
:10FE7000AF84B88889859A85A80EB91EC5010E94ED
:10FE8000B6789058A70196010E942EEBAB01BC01F9
:10FE9000CC24C394D12CEF80F8849401C5010E9436
:10FEA0005577AF8DB8A1AB2B51F101E010E0E98C93
:10FEB000FA8CEB85FC85EE0EFF1E970141E050E0C9
:10FEC0008B809C80840C951CB401AF84B888898594
:10FED0009A85A80EB91EC5010E94B6789058D10126
:10FEE0002D913D914D915C910E942EEBAB01BC0197
:10FEF000CC24C394D12C9401C5010E945577298943
:10FF00003A894B895C89D1012D933D934D935C9344
:10FF10001397E985FA853196FA87E9872B853C8521
:10FF2000245031093C872B8749815A81240E351E84
:10FF30006B817C81640F751F7C836B8359CFAF8D80
:10FF4000B8A1AB2B09F428CEC201A201440F551F62
:10FF5000440F551F2D962EAD3FAD2D97420F531FC9
:10FF600020E030E001966F857889681779070CF4F6
:10FF70000FCEFA01E20FF31F108211821282138258
:10FF80002C5F3F4FEFCF8D819D85E4960FB6F8949F
:10FF9000DEBF0FBECDBFDF91CF911F910F91FF90BC
:10FFA000EF90DF90CF90BF90AF909F908F907F9019
:10FFB0006F905F904F903F902F9008952F923F92B7
:10FFC0004F925F926F927F928F929F92AF92BF9269
:10FFD000CF92DF92EF92FF920F931F93CF93DF9315
:10FFE00000D0CDB7DEB73A832983380126016501F9
:10FFF00014010115110599F01F922EE62F93DF923F
:020000021000EC
:10000000AF92DF92AF9242010F89188D93010E9447
:10001000DF7A0F900F900F900F900F900F90F101DB
:1000200080E090E029813A81821793074CF4208187
:100030003181319521953109219331930196F2CF88
:100040009301220F331F220F331F240D351D80E033
:1000500090E0A981BA816A167B0664F4F901E80F81
:10006000F91F10821182128213824FEF641A740AF0
:100070000496EFCF3201B10141E050E0E981FA810D
:10008000E417F507E4F1FB01208131811216130614
:1000900074F1319521953109318320832417350777
:1000A00031F1D3018D909D90AD90BC901397F901E3
:1000B000E150F04CEE0FFF1FEE0FFF1FE40DF51D9A
:1000C000C080D180E280F380CD92DD92ED92FC92EF
:1000D000139780829182A282B382F901E150F048A5
:1000E000EE0FFF1FE20DF31D20813181D2CF4F5F54
:1000F0005F4F6E5F7F4FB4E06B0E711CBFCF0F90F0
:100100000F90DF91CF911F910F91FF90EF90DF90B3
:10011000CF90BF90AF909F908F907F906F905F90A7
:100120004F903F902F9008952F923F924F925F9261
:100130006F927F928F929F92AF92BF92CF92DF92F7
:10014000EF92FF920F931F93CF93DF934C016A01BD
:100150007B013901181619060CF0A3C001301105F6
:1001600009F069C065E070E00E94E6EEEC012C0148
:10017000590100E010E00C171D0794F4A701960147
:10018000F50160817181828193810E94FCEDF5010E
:1001900061937193819391935F010F5F1F4FEBCF39
:1001A000CC0FDD1FCC0FDD1FC60DD71D4814590421
:1001B0000CF077C0A7019601688179818A819B81C3
:1001C0000E94FCED688379838A839B83A701960153
:1001D0006C817D818E819F810E94FCED6C837D838B
:1001E0008E839F83A7019601688579858A859B8583
:1001F0000E94FCED688779878A879B87A701960113
:100200006C857D858E859F850E94FCED6C877D8742
:100210008E879F87A7019601688979898A899B893A
:100220000E94FCED688B798B8A8B9B8BF5E04F0EDF
:10023000511C6496BBCF17FF0CC081E090E0881979
:100240009909809F2001819F500C909F500C112490
:1002500002C0412C512C1801220C331C220C331CDF
:10026000440C551C440C551C460C571C00E010E077
:10027000C0E0D0E05201A00EB11EA7019601F50129
:1002800060817181828193810E94FCEDF501608320
:100290007183828393832196020D131DC815D9059E
:1002A00049F7DF91CF911F910F91FF90EF90DF9071
:1002B000CF90BF90AF909F908F907F906F905F9006
:1002C0004F903F902F9008952F923F924F925F92C0
:1002D0006F927F928F929F92AF92BF92CF92DF9256
:1002E000EF92FF920F931F93CF93DF93CDB7DEB7BB
:1002F000E6970FB6F894DEBF0FBECDBF9E838D8309
:100300007E8B6D8B1A013A8B298B18A70FA3FC8E5D
:10031000EB8EDAA6C9A6AB2809F4C8C087017C0118
:1003200066246394712CCC24C394D12C29893A89F6
:100330002C153D050CF44AC0D8018D919C9197FF76
:1003400005C0222733272C193D0901C09601F80169
:10035000318320831816190684F5C614D704D1F00A
:10036000C30101972D893E89829FB001839F700D43
:10037000929F700D1124660F771F660F771F4D81B6
:100380005E81640F751F1214130424F4A701C101C8
:100390000E94E175F301E150F048EE0FFF1F8B8DD5
:1003A0009C8DE80FF91F80819181D8018D939C93DA
:1003B000D182C082BFEF6B1A7B0AEFEFCE1ADE0A42
:1003C0000E5F1F4FF4E0EF0EF11CB0CF4901880C17
:1003D000991C4B8D5C8D840E951E2CEF4D895E898A
:1003E00024036001259FD00C112489899A890197E3
:1003F000849F8001859F100D949F100D1124000F84
:10040000111F000F111F8D819E81080F191F498830
:100410005A887201A12CB12C1E141F040CF04BC081
:10042000D4019E918E914D0197FF3AC0919581958F
:1004300091098D939C93E414F50479F1A501400F83
:10044000511FC2010197ED89FE898E9FB0018F9FD8
:10045000700D9E9F700D1124660F771F660F771F1A
:100460002D813E81620F731F121413041CF4C1010D
:100470000E94E175F201E150F048EE0FFF1F4B8D35
:100480005C8DE40FF51F80819181D4012D913C9109
:100490001197318320838D939C93B1E04B1A5108BF
:1004A000E1E0EE1AF108AC0CBD1CB6CF412C512C8A
:1004B00066246394712C2D893E89220F331F220FED
:1004C000331F388F2F8BCD80DE80C21AD30A930161
:1004D000215031094D895E89249FC001259F900DCF
:1004E000349F900D1124880F991F880F991FC80EF3
:1004F000D91E4301880C991C880C991CAFA0B8A484
:10050000A80CB91C930100E010E0E12CF12C8F89BC
:10051000988DE80EF91E0C5F1F4F42165306BCF073
:1005200041E050E0B6016E0D7F1DC1012CAB3DAB2B
:100530000E940D7AF501E00FF11F389760837183F7
:10054000828393832CA93DA92F5F3F4FE0CFA9A5BC
:10055000BAA58A0E9B1E930180E090E00496421695
:1005600053069CF0F501E80FF91F3897408151813F
:1005700062817381F401E80FF91F3897408351833A
:10058000628373832F5F3F4FE9CFE989FA89F8AB24
:10059000EFA72E163F0614F438AA2FA62F89388D00
:1005A0002C5F3F4F3AAB29AB4FA158A55A8F498FCB
:1005B00089A59AA59AA389A3D1011197B8A3AF8F52
:1005C000ED81FE81FEA3EDA3F88BEF87FC8BEB8B17
:1005D00021E030E03A832983A981BA81EFA5F8A907
:1005E000EA17FB070CF462C249815A814615570588
:1005F0000CF49EC0441555050CF09AC05E8F4D8FCB
:100600008A01E12CF12C1D86812CA12CB12CC98CE6
:10061000DA8C54E0C50ED11CF601EE0DFF1D3497A7
:1006200080818B8391819F839280A381A9879C0184
:10063000492D5A2F6D85782DC5010E9427EB87FD26
:1006400006C0BD85BB838F829A2CB98602C01E8FDF
:100650000D8F0F5F1F4FE4E0EE0EF11C40165106A8
:1006600034F0FB81FD878F80A92CB984D5CF2D8DE7
:100670003E8D49815A812417350709F459C0C901B3
:100680000197AD89BE898A9FA0018B9F500D9A9FCB
:10069000500D1124440F551F440F551FED81FE814D
:1006A0004E0F5F1F121413042CF46DA17EA1C10123
:1006B0000E94E1758D8D9E8D8150904C880F991F01
:1006C000880F991FA98DBA8D4D915D916D917C9187
:1006D000EFA1F8A5E80FF91F40835183628373836C
:1006E000E9A1FAA14081518162817381E9A5FAA54E
:1006F000E80FF91F40835183628373834D8D5E8DB4
:1007000041505048440F551F2B8D3C8D420F531FB5
:10071000DA018D919C911197E981FA81EE0FFF1F0B
:10072000E20FF31F329122912D933C9391838083AA
:10073000E98DFA8D1192119211921192FA8FE98F2F
:1007400029813A812215330509F489C14F8D58A1B9
:100750004F5F5F4F5CA34BA341E050E06B897C8906
:100760008BA19CA10E940D7A69877A878B879C87D1
:1007700020E030E0A9010E9427EB882309F46FC133
:10078000AF85B889CD90DD90ED90FC9020E030E011
:10079000A901C701B6010E9427EB8823E1F020E000
:1007A00030E0A901C701B6010E9427EB87FF05C011
:1007B00020E030E040E85FEB04C020E030E040E8BB
:1007C0005FE369857A858B859C850E94FCED69874E
:1007D0007A878B879C8729853A854B855C8560E085
:1007E00070E080E89FE30E942EEBAB01BC0101E0CA
:1007F00010E02B893C898BA19CA10E94948020E071
:1008000030E040E85FE3EF85F889608171818281A3
:1008100093810E944EEAAF85B8896D937D938D9345
:100820009C931397E981FA813196F887EF832B899E
:100830003C894F89588D240F351F3C832B8389A118
:100840009AA104969E8F8D8FA98DBA8DBE87AD8794
:100850002F81388549895A89421753070CF4E5C01E
:1008600001E010E02B813C8141E050E06B897C8904
:100870008BA19CA10E94B6789058EF85F8892081C1
:100880003181428153810E942EEBAB01BC01CC240B
:10089000C394D12CEB80FC802B893C898BA19CA13B
:1008A0000E9455772F813885261537050CF4A3C093
:1008B000421653060CF49FC0AD85BE85CD90DD90E9
:1008C000ED90FC9020E030E0A901C701B6010E9444
:1008D00027EB882309F48FC0EB81FC818080918015
:1008E000A280B38020E030E0A901C501B4010E94DC
:1008F00027EB87FF04C0C501B401905802C0C501B1
:10090000B401A70196010E942EEB9B01AC010E944D
:10091000FCED9B01AC0160E070E080E89FE30E9489
:100920004DEA8B015C0120E030E0A9010E942AED34
:1009300018161CF4AEAABBAA04C000E010E01EAA60
:100940001BAAAD8DBE8D2D913D914D915C91C7013E
:10095000B6010E942EEB4B015C012DEC3CEC4CE40B
:100960005DE3B8018EA99BA90E94FCED6BA77CA753
:100970008DA79EA7A5019401C501B4010E94FCEDBD
:100980009B01AC016BA57CA58DA59EA50E94FCEDED
:1009900020E030E040E85FE30E944EEA20E030E0F3
:1009A00040E85FE30E9427EB882371F0B8018EA92D
:1009B0009BA90E9469EE9B01AC01C701B6010E9490
:1009C000FCEDED85FE8513C041E050E06B817C813C
:1009D0006C5F7F4F8F8D98A10E940D7AAD85BE858B
:1009E0006D937D938D939C931397ED8DFE8D608316
:1009F0007183828393832F8138852F5F3F4F3887A0
:100A00002F834D855E854C5F5F4F5E874D878D8D53
:100A10009E8D04969E8F8D8FAB81BC81EF89F88D62
:100A2000AE0FBF1FBC83AB8313CFEF85F8898081E6
:100A30009181A281B381298D3A8D24503109F90128
:100A400080839183A283B38389859A85AB85BC8596
:100A5000B058EF85F88980839183A283B38329817D
:100A60003A812F5F3F4F3A8329834B895C8989A95B
:100A70009AA9480F591F5C8B4B8BAF85B889A80F7B
:100A8000B91FB88BAF87E9A1FAA13496FAA3E9A3FD
:100A90002DA13EA14F89588D240F351F3EA32DA3B4
:100AA0008F8D98A1019798A38F8F96CDE6960FB65C
:100AB000F894DEBF0FBECDBFDF91CF911F910F9194
:100AC000FF90EF90DF90CF90BF90AF909F908F906E
:100AD0007F906F905F904F903F902F9008952F924E
:100AE0003F924F925F926F927F928F929F92AF92BE
:100AF000BF92CF92DF92EF92FF920F931F93CF930B
:100B0000DF93CDB7DEB72C970FB6F894DEBF0FBEDC
:100B1000CDBF9C838B837E836D835A834983390148
:100B2000E986FA860B871C87D886CF8275018401F7
:100B30004DB65EB6C901880F991F880F991F2DB752
:100B40003EB7281B390B0FB6F8943EBF0FBE2DBF22
:100B50008DB79EB701966C01F50180E090E0861597
:100B6000970524F4119211920196F9CFAA24A39427
:100B7000B12C930149815A816D817E818B819C8149
:100B80000E946481EF81F88511821082130129810E
:100B90003A81261537050CF419010D811E810F5F6E
:100BA0001F4F000F111F000F111F8B819C819A8313
:100BB0008983612C712C621473040CF040C0E981AC
:100BC000FA8180809180A280B38020E030E0A9018A
:100BD000C501B4010E9427EB87FF04C0B7FAB094A7
:100BE000B7F8B094EB81FC81C080D180E280F380C3
:100BF00020E030E0A901C701B6010E9427EBA70160
:100C0000960187FD505889819A81800F911F9A83A0
:100C1000898369857A858B859C850E94FCED9B0183
:100C2000AC01C501B4010E9427EB181644F49FEFF4
:100C3000691A790AEF81F88571826082BCCF0FB69C
:100C4000F8945EBE0FBE4DBE0FB6F8945EBE0FBEEA
:100C50004DBE2C960FB6F894DEBF0FBECDBFDF9110
:100C6000CF911F910F91FF90EF90DF90CF90BF90A9
:100C7000AF909F908F907F906F905F904F903F903C
:100C80002F9008952F923F924F925F926F927F9292
:100C90008F929F92AF92BF92CF92DF92EF92FF928C
:100CA0000F931F93CF93DF93CDB7DEB72A970FB67D
:100CB000F894DEBF0FBECDBF9A8389832B011A0142
:100CC0003901DC82CB82B886AF829A8689868BA175
:100CD0008D839CA19E838DA19EA16417750764F1ED
:100CE0001216130664F51816190664F5019741F4F7
:100CF0008D809E80A9A0BAA089819A810E946F856B
:100D0000EB81FC8100811181FE81FF938D818F93A6
:100D100089A09AA0AF8CB8A0C984DA84EF80F88447
:100D20009301A101B20189819A810E94DE7F0F9017
:100D30000F9080E090E008C08FEF9FEF05C08EEF2E
:100D40009FEF02C08DEF9FEF2A960FB6F894DEBF9B
:100D50000FBECDBFDF91CF911F910F91FF90EF900C
:100D6000DF90CF90BF90AF909F908F907F906F90CB
:100D70005F904F903F902F9008952F923F924F9207
:100D80005F926F927F928F929F92AF92BF92CF921B
:100D9000DF92EF92FF920F931F93CF93DF9300D0D8
:100DA00000D0CDB7DEB74C013B012A014DB75EB78D
:100DB0005C834B83469EC001479E900D569E900DCE
:100DC0001124880F991F880F991F481B590B0FB6C4
:100DD000F8945EBF0FBE4DBF8DB79EB701961C0144
:100DE000C201880F991F880F991F481B590B0FB616
:100DF000F8945EBF0FBE4DBF8DB79EB701966C01D4
:100E0000C301880F991F880F991F481B590B0FB6F4
:100E1000F8945EBF0FBE4DBF8DB79EB701967C01A3
:100E2000C201880F991F481B590B0FB6F8945EBF7B
:100E30000FBE4DBF8DB79EB701965C01A201B301F5
:100E4000C1010E94FD76A101B201C3010E946F762B
:100E50009B01AC0160E070E080E895E20E942EEB1F
:100E60001F9221E02F93DF92CF92BF92AF92FF9219
:100E7000EF9258019E012F5F3F4F69017B018C016A
:100E80009201A301B301C1010E9442864DB75EB732
:100E9000485F5F4F0FB6F8945EBF0FBE4DBF8B81AA
:100EA0009C810FB6F8949EBF0FBE8DBF0F900F9020
:100EB0000F900F90DF91CF911F910F91FF90EF90C6
:100EC000DF90CF90BF90AF909F908F907F906F906A
:100ED0005F904F903F902F9008958FEF8EBD0DB48F
:100EE00007FEFDCF8EB508958EBD0DB407FEFDCF74
:100EF000089561E0FC0180810C944EE9FC0122819F
:100F0000322F306A36953CBD20FD06C031E02630D8
:100F100009F430E0232F01C020E02DBD60E0FC018A
:100F200080810C944EE9CF92DF92EF92FF920F9363
:100F30001F93CF93DF93EC018B017A010E94CBE7E3
:100F40006B010E946D878B838F3F49F40E94CBE732
:100F50006C197D096D327140A0F381E103C08E3FB1
:100F600051F08FE08983CE010E9479878FEF0E9434
:100F7000748780E02AC0E114F104E1F081E0E81A0E
:100F8000F1088FEF8EBDF8012FEFCF01801B910B81
:100F90008E159F0538F40DB407FEFDCF8EB58193F5
:100FA0002EBDF3CF0DB407FEFDCF8EB5F801EE0DCB
:100FB000FF1D80830E946D870E946D87CE010E9475
:100FC00079878FEF0E94748781E0DF91CF911F9125
:100FD0000F91FF90EF90DF90CF9008950F931F93A4
:100FE000CF93DF93EB010E94CBE78B010E946D87CB
:100FF0008F3F49F00E94CBE7601B710B6C177D0798
:10100000A8F380E001C081E0DF91CF911F910F91A3
:101010000895CF92DF92FF920F931F93CF93DF93A8
:1010200000D000D0CDB7DEB76C01F62E29833A830D
:101030004B835C830E947E876CE271E0C6010E9454
:10104000EE878F2D80640E94748708E110E05C8138
:101050004B813A812981DA01C901002E04C0B6957D
:10106000A795979587950A94D2F729833A834B835E
:101070005C830E9474870850110929813A814B8151
:101080005C81083F8FEF180731F7FF2029F0E8E077
:10109000FE1621F08FEF03C085E901C087E80E94AA
:1010A0007487FCE0FF1202C00E946D8710E00E946E
:1010B0006D87F601838387FF04C01F3F11F01F5F18
:1010C000F6CF0F900F900F900F90DF91CF911F915F
:1010D0000F91FF90DF90CF900895BF92CF92DF9253
:1010E000EF92FF920F931F93CF93DF93EC01B62EF5
:1010F0001C82198248830E94CBE78B0161E08881C2
:101100000E9415E9CE010E94798760E086E00E9486
:1011100015E961E085E00E9415E961E087E00E9441
:1011200015E961E084E00E9415E961E084E00E9435
:101130004EE986E08A8383E58CBD1DBC2AE0F22E51
:101140008FEF0E947487FA94D9F720E030E0A9016C
:1011500060E0CE010E940988F82E8B8381E0F816AA
:1011600049F00E94CBE7601B710B613D774068F34B
:1011700081E04BC02AEA31E040E050E068E0CE0177
:101180000E94098882FF02C0FC820DC094E0F92E03
:101190000E946D878B83FA94D9F78A3A11F082E026
:1011A00034C082E08C838C81823031F4C12CD12C0C
:1011B000E12C80E4F82E03C0C12CD12C760120E074
:1011C00030E0A90167E3CE010E940988A7019601DA
:1011D00069E2CE010E9409888B83882349F00E942E
:1011E000CBE7601B710B613D774048F38AE00DC08F
:1011F0008C818230E1F420E030E0A9016AE3CE0185
:101200000E940988882331F088E08983CE010E94FA
:10121000798719C00E946D87807C803C11F483E03F
:101220008C830E946D870E946D870E946D87CE011E
:101230000E94798786E08B1518F488E1898303C0C2
:10124000BA8281E001C080E0DF91CF911F910F91C0
:10125000FF90EF90DF90CF90BF9008950F931F9372
:10126000CF93DF93EC0189018C81833039F039E031
:10127000440F551F661F771F3A95D1F79A01AB01AE
:1012800061E1CE010E94098881110AC040E052E06C
:10129000B801CE01DF91CF911F910F910C949387EC
:1012A00084E08983CE010E94798780E0DF91CF912D
:1012B0001F910F910895CF93DF93EC016EBD20E055
:1012C00030E00DB407FEFDCFFA01E20FF31F80817D
:1012D0008EBD0DB407FEFDCF81818EBD2E5F3F4FC9
:1012E000211582E0380769F70DB407FEFDCF8FEFB7
:1012F0000E9474878FEF0E9474870E946D878B8392
:101300008F71853039F083E18983CE010E9479871E
:1013100080E001C081E0DF91CF9108950F931F938A
:10132000CF93DF93EC0189018C81833039F089E020
:10133000440F551F661F771F8A95D1F79A01AB019D
:1013400068E1CE010E940988882311F086E023C05D
:10135000A8016EEFCE010E945B898823E9F068E561
:1013600072E0CE010E94EE87182F811102C087E142
:1013700012C020E030E0A9016DE0CE010E94098892
:10138000811108C00E946D87811104C0CE010E94A6
:10139000798706C086E18983CE010E94798710E0B3
:1013A000812FDF91CF911F910F910895CF93DF93FC
:1013B000EC019C012C5F3F4F41E050E060E070E0A9
:1013C000898D9A8D0E94E494882399F04D895E89D5
:1013D0006F89788D452B462B472B59F44C815D81C5
:1013E0006E817F814D8B5E8B6F8B788F998190683A
:1013F0009983DF91CF910895CF92DF92EF92FF9280
:101400000F931F93CF93DF93EC0189899A89AB895E
:10141000BC89803E9F4FAF41B10510F080E06CC0A9
:10142000CE010E94D6898823C9F30E94F492182F16
:101430008823A1F3E98DFA8DCC80DD80EE80FF80DA
:1014400032E0C31AD108E108F108058404C0CC0CCD
:10145000DD1CEE1CFF1C0A94D2F786859785A089B7
:10146000B189C80ED91EEA1EFB1E81E08093310FA0
:10147000C0923411D0923511E0923611F0923711AA
:1014800080E092E0E4E3FFE0DF019C011D92215047
:101490003040E1F701E0E98DFA8D8481081790F47E
:1014A00024E33FE0B701A601400F511D611D711DEE
:1014B0008091320F9091330F0E948E898823E1F042
:1014C0000F5FE9CFC12C82E0D82EE12CF12C0584EE
:1014D00004C0CC0CDD1CEE1CFF1C0A94D2F7498919
:1014E0005A896B897C894C0D5D1D6E1D7F1D498B52
:1014F0005A8B6B8B7C8B812FDF91CF911F910F913A
:10150000FF90EF90DF90CF900895CF93DF93EC01A1
:1015100041E0611101C040E06C857D858E859F852D
:101520000E943493882341F0888920E2829FC00181
:1015300011248C5C904F02C080E090E0DF91CF914D
:10154000089530E020E04EE2DC015C91503271F011
:10155000383029F4FB01E20FF11D40832F5FFB01BE
:10156000E20FF11DDC015C9150832F5F3F5F01961C
:101570003B3051F7FB01E20FF11D10820895CF932C
:10158000DF93EB01FC012381211102C080E010C038
:101590002250223020F48FE28883198208C060E054
:1015A0000E94858A009791F3BE010E94A18A81E082
:1015B000DF91CF910895FB012BE030E23193215070
:1015C000E9F7DC0190E027E03A2FEB2F8D918111B4
:1015D0000AC0DA013C931196EC9381E0FB01908103
:1015E000903239F525C08F32A1F38E3219F0E2E83E
:1015F000F0E108C02A30E1F098E02AE0E5CF31962A
:101600003817B1F034913111FACF291788F03FED36
:10161000380F3E3568F431E0390FFB01E90FF11D59
:101620009FE9980F9A3108F480528083932FCCCF92
:1016300080E008950F931F93CF93DF93EC018B010C
:101640008B81882311F080E042C0FB0187898031C3
:1016500039F18032C1F783E08B83F801428D538DDD
:10166000648D758D4D8B5E8B6F8B788F9E012F5E99
:101670003F4FC8010E94ED93882329F31A8F098FE9
:1016800081E089831C821D821E821F821886198632
:101690001A861B861C861D861E861F86188A17C002
:1016A00082E08B831D8A1E8A1F8A188EFB01408D63
:1016B000518D60E070E095E0440F551F661F771F65
:1016C0009A95D1F7498B5A8B6B8B7C8BD7CFDF9157
:1016D000CF911F910F9108952F923F924F925F9259
:1016E0006F927F928F929F92AF92BF92CF92DF9232
:1016F000EF92FF920F931F93CF93DF93EC015B0167
:101700006A018B81811103C08FEF9FEFC9C089816E
:1017100080FFFACF49895A896B897C8988859985A8
:10172000AA85BB852601612C712C8A019B01081BAF
:10173000190B2A0B3B0B041515052605370518F464
:101740006A01C81AD90A76013E0124E0620E711CB2
:10175000E114F10409F477C0488559856A857B85D1
:101760004A0181E098222B811A012B01E9E056946D
:10177000479437942794EA95D1F7898D9A8DFC0187
:10178000223049F4628D738D848D958D620D731DA9
:10179000841D951D3DC014811150122181149104A6
:1017A000C9F4111117C0452B462B472B49F48D89DD
:1017B0009E89AF89B88D8C839D83AE83BF830AC019
:1017C0004C815D816E817F8193010E946D9388239E
:1017D00009F49ACFE98DFA8D6C817D818E819F818C
:1017E0006250710981099109058404C0660F771F51
:1017F000881F991F0A94D2F7268537854089518919
:10180000620F731F841F951F610F711D811D911D34
:1018100020E032E02819390987012E153F0508F428
:1018200089010115F2E01F0769F52091341130910B
:1018300035114091361150913711621773078407A3
:10184000950719F41FC0C6012BC09501AB01BC015F
:101850008091320F9091330F0E942E89882309F4D2
:1018600053CFA00EB11E88859985AA85BB85800FB0
:10187000911FA11DB11D88879987AA87BB87E01A90
:10188000F10A66CF40E00E943493882309F43CCFEC
:10189000B4016C5C704FA801C5010E94C5F2E1CF94
:1018A000DF91CF911F910F91FF90EF90DF90CF903C
:1018B000BF90AF909F908F907F906F905F904F9070
:1018C0003F902F900895CF93DF931F92CDB7DEB74F
:1018D00041E050E0BE016F5F7F4F0E946C8B01972B
:1018E00019F4898190E002C08FEF9FEF0F90DF9194
:1018F000CF910895AF92BF92CF92DF92EF92FF9275
:101900000F931F93CF93DF936C01EB017A01DC01FE
:1019100013968C911397823070F018960D911D914B
:101920002D913C911B970F71112722273327012BF3
:10193000022B032B11F08FEF59C04115510511F007
:10194000F70110821DE040E250E0BE01C6010E9496
:101950006C8B9C018032910531F081E0232B09F4DE
:1019600080E0819543C088818823C1F1853E59F389
:101970008E3249F3E114F10461F19B859F739F302E
:1019800041F54A8D5B8D452B21F58F719FEF980FA7
:101990009230F8F490E00197189F9001199F300D54
:1019A0001124FE0180E090E05701A20EB31E8530A5
:1019B000B8F46181A501480F591FDA016C930196B3
:1019C00032968D30910599F7888186FF02C0F50126
:1019D00015868B8583FDB7CF822F08C080E006C0B7
:1019E0008B3010F46481E6CF6681E4CFDF91CF9134
:1019F0001F910F91FF90EF90DF90CF90BF90AF902D
:101A000008951F93CF93DF93EC018B81823018F4FC
:101A100080E090E024C0488559856A857B85A5E0F3
:101A20007695679557954795AA95D1F7142F1F700E
:101A3000CE010E94638C97FDEBCF488559856A855E
:101A40007B85415E5F4F6F4F7F4F488759876A871D
:101A50007B8720E2129FC00111248C5C904FDF91A4
:101A6000CF911F9108954F925F926F927F92AF92A4
:101A7000BF92CF92DF92EF92FF920F931F93CF937B
:101A8000DF93EC016A017B012B81222349F08989D4
:101A90009A89AB89BC8984179507A607B70710F404
:101AA00080E06CC0223009F464C0C114D104E104A8
:101AB000F10449F41C821D821E821F821886198639
:101AC0001A861B865AC088859985AA85BB85E98DAB
:101AD000FA8DE585F0E03996AC01BD014150510920
:101AE000610971090E2E04C0769567955795479543
:101AF0000A94D2F797018601015011092109310991
:101B000004C03695279517950795EA95D2F70417DF
:101B100015072607370720F0892B8A2B8B2B49F4D2
:101B20008D899E89AF89B88D8C839D83AE83BF8359
:101B300004C0041B150B260B370B280139015E016D
:101B400084E0A80EB11C411451046104710489F0B1
:101B50004C815D816E817F819501898D9A8D0E9476
:101B60006D9391E0491A5108610871088111EBCF1A
:101B700005C0C886D986EA86FB8681E0DF91CF91D1
:101B80001F910F91FF90EF90DF90CF90BF90AF909B
:101B90007F906F905F904F9008950F931F93CF9316
:101BA000DF93EC018B818823E1F1898187FF33C0CA
:101BB00061E0CE010E94858A8C01009791F1FC01C1
:101BC0008081853E71F18B81823040F449895A8948
:101BD0006B897C89448F558F668F778F4D895E899D
:101BE0006F89788DF801538F428F758B648BE091EC
:101BF0002B0FF0912C0F309759F0B8016A5E7F4F90
:101C0000C80148960995F801808D918D938B828B40
